:020000024000BC
:10E000006FF0C171000000000018011800280128FD
:10E0100002280328002901290229032904290529A6
:10E02000062907290829002A012A022A032A042A84
:10E03000052AA62ADCDE0600880905004204002025
:10E04000BC040020CA0300209C03002032030020EF
:10E050002A0B05006A0B0500080D0500880F050056
:10E060006C100500E80705009A0705008C020020E7
:10E070003602002026150500D0070020000B050001
:10E080002E120500E6970600C6990600309A060093
:10E090003A5C0600725C060072150600A80A0600CB
:10E0A000689206005E120500686206000CAE05006C
:10E0B0009CAE0500F6AE0500461D0500841D05005A
:10E0C000041C0500767005009A6B0500480A0020C4
:10E0D000AC7C050012800500C85E05006C5E050082
:10E0E0002A620500145F05004C5E0500C25E050053
:10E0F000025E05008C5F0500E45F0500945F05008B
:10E10000985F05002E600500EC5F05001C600500AF
:10E11000D6640500DA640500885F0500905F05009D
:10E120002C600500D8640500DA6005003266050041
:10E130006C8D0500E08D05001A8E0500C272050089
:10E14000D67205000A730500F45305001A5605003F
:10E15000F65605002E3A0500C4340500024B0500B2
:10E160004035050080460500C4C0060070B90600B1
:10E1700032BE060036D3060022D2060090D5060035
:10E1800080D5060088D50600CAD50600C8AB0600B3
:10E19000000000000000000000000000000000007F
:10E1A0003AD6060028D00600C6CF060000000000C0
:10E1B000000000000000000000000000000000005F
:10E1C000467B06006C6A0600C26D0600AA6B06005C
:10E1D00084750600C092060000000000FCAB06003B
:10E1E000A2160500825C0600486206004063060035
:10E1F000000000000000000000000000867605001E
:10E20000847A06000000000000000000000000000A
:10E210001C6A0600BA090020EE5C0600B6D50600AE
:10E22000000000000000000084D50600120F050069
:10E23000FA730500BED50600327D0600967E060004
:10E24000027F060070BE0600BAD50600C2D50600E1
:10E25000340A0600C6D50600341B00203C240020EA
:10E2600000000000000000000000000000000000AE
:10E27000000000000000000000000000000000009E
:10E280006373B60082801C419105110523AEF5FE33
:10E29000C5BFB727002037370020938707501307E3
:10E2A000C7BC6373F700828023A007009107D5BF26
:10E2B000411122C4B747024006C603A4C72023A6C3
:10E2C00007200F10000011C199E5B747024023A6AF
:10E2D0008720014545A093073500C207C183F19B04
:10E2E000C207C183130740036366F7023727002084
:10E2F0000325077837270020832687776391A602B6
:10E30000373700200327C78069D3C207DD8D054555
:10E31000029765BF372700200325C777E1BF7A2121
:10E3200031EF5A21636CF704B72600203306F7401B
:10E330002148938686786375C8028328050003D830
:10E340006600138687001D8F2A9661175AA2232024
:10E3500016012313060010C15EA1130788FFFAA25D
:10E360006EA1EE222105B387F540FEA2B747024019
:10E3700023A68720B2402244410182800841BDBFCC
:10E38000B747024003A8C72023A607200F100000AC
:10E3900001E523A607218280B727002003AE077876
:10E3A000B727002003A387778146F28763FE6708BB
:10E3B00083A80700636DF50863EBA808138787003F
:10E3C0006364E508F223216705076319E600372631
:10E3D00000200347065A05072300E65A3726002087
:10E3E00013058678CE237A212393070013068678B7
:10E3F0002E97420741837AA16383C7033725002004
:10E400000325C577630DF500EA2211E9DE2223A07A
:10E4100016012107BE95A105CEA27AA2B687984320
:10E4200063046702B726002083A6C677630ED70071
:10E43000762399EAD6234E231843A106AE96D6A397
:10E4400098C37E22A1077EA2B747024099B7BE8635
:10E45000C687A9BFB7270020B726002083A7077863
:10E4600003A686772A87B305B5406314F6003A857C
:10E4700029A8938687009C43E369D7FEE377F7FEDC
:10E480002E85E3E4D5FEE3F2F5FE828023AC05FEA3
:10E490001C4181E70CC18280BA8703A787FF6DFF0B
:10E4A00023ACB7FE8280411126C24AC0B744024065
:10E4B00006C622C403A9C42023A604200F1000000E
:10E4C00009E923A62421B240224492440249410191
:10E4D00082802A842105BD654205C18D4181C93BE9
:10E4E00011C9FD572320050042A17CA123A62421A8
:10E4F0002105D1BF23A624210145F1B701114AC846
:10E500004EC6B747024006CE22CC26CA83A9C720F2
:10E510002A8923A607200F10000037250020032496
:10E5200045788144014609E889ECA1654A85971040
:10E5300005E0E780A0CC25A08347E4FF639D270387
:10E54000A1C0A68513054578970005E0E780404AFD
:10E5500069DCA1654A85971005E0E7804084F240B8
:10E560006244B747024023A6372126854249D24458
:10E57000B2490561828091E02286032484FF65B759
:10E58000A284E5BFB727002083A7477D99E33E8596
:10E590008280BA236315B7009823E30AA7FEDC47FD
:10E5A000F5B7B747024003A7C72023A607200F10DF
:10E5B000000001C599C1814711E6B747024023A673
:10E5C000E7208280B386F50003C80600B306F50095
:10E5D000850723800601E317F6FEC5B737470240DB
:10E5E0008327C720232607200F10000019C191C1DF
:10E5F00011E6374702402326F7208280910503A7C2
:10E60000C5FF11057D16232EE5FEDDB73747024015
:10E610008327C720232607200F10000001C53307DA
:10E62000C50011E6374702402326F7208280050502
:10E63000A30FB5FEE31DE5FEF5B7B747024083A67D
:10E64000C72023A607200F10000081473307F500DD
:10E650000307070019E7374702402326D7203E85E6
:10E6600082808507E5B7011126CA4AC8B74702402C
:10E6700006CE22CC83A4C7202A892E8623A6072073
:10E680000F100000131506019305F004418132C6F6
:10E6900005312A8401C53246CA8521372285F240D8
:10E6A0006244B747024023A697204249D2440561FD
:10E6B0008280B747024003A7C72023A607200F1078
:10E6C000000001C599C1814711EAB747024023A65E
:10E6D000E720054582808507E309F6FE3308F5004B
:10E6E000B386F500034808009422E306D8FEB74736
:10E6F000024023A6E72001458280B747024003A7D6
:10E70000C72023A607200F1000009307F6FFBE9531
:10E710002A966317C500B747024023A6E7208280E8
:10E72000FD159C310505A30FF5FEE5B737470240FF
:10E730008327C720232607200F10000001C53307B9
:10E74000C50019E6374702402326F720014582809D
:10E7500005058346F5FFE397B6FEE31BE5FE374765
:10E7600002402326F72005458280797126D2B724FE
:10E77000002022D403A4447D06D64AD04ECE52CCEB
:10E7800056CA5AC85EC662C455C4372A0020372903
:10E790000020B7390020814BB72A002037CBC901B0
:10E7A000130A8A7D13098978938909823E2099EF9B
:10E7B0005C44639A0B0023AAF47C032CC4002285DA
:10E7C000C1366284A9A823A6FB00C5BF83A7CA7C63
:10E7D00082971C443307F5406376F50003A7490090
:10E7E0001D8F2A979306FB3763EAE6062328090064
:10E7F0002E200820970005E0E780605A5C405844CE
:10E80000B1C70C4403A64900AE97BE8663E4B700C7
:10E8100063E4C700B386C74014C4A28B3A8459F49A
:10E82000B727002093878778984B854663FCE604DA
:10E830007D1798CBB250225492540259F249624A41
:10E84000D24A424BB24B224C4561828063950B0009
:10E8500023AAE47C9DB723A6EB0085B703278A0291
:10E8600019CB63EDA7003385A740832709016374A3
:10E87000F5002328A900A28B404455B703A74900FF
:10E88000BA97D5B723A8070075B701114EC6B74789
:10E89000024006CE22CC26CA4AC852C483A9C72049
:10E8A00023A607200F1000003734002093070482AE
:10E8B000C843DC2713040482B9CFB73700209387FD
:10E8C000879803D7870A21CB83A4470A6385A404CA
:10E8D000B727002013878778184B138A8778630F30
:10E8E000A70E372900208327C97C829763E5A40EF1
:10E8F0008327C97C898C829703270A0163F3E4008C
:10E900002687B307A7003E85544063E4E70063E42D
:10E91000D7003385D740B747024023A637215C4054
:10E92000639DA702B7240020938484789848B72772
:10E93000002083A7C77C6315A70A82975440B74776
:10E9400036FE938707C8B6973387A7003A85636476
:10E95000F7006364D7003305D740B73400209387AE
:10E96000C4ACDC539384C4AC99CBB737002083A6E6
:10E9700087B43707CDFF7D179C46F98F9CC611E100
:10E9800048408547DCC4B737002083A707808297BB
:10E9900005E1DC5089CFDC4499CB976006E0E78045
:10E9A00040D7975006E0E780205623A60400753B29
:10E9B000DC5091CBB737002003A787B4B7063300EC
:10E9C0001C47D58F1CC7F2406244D2444249B24929
:10E9D000224A056182805C40BE9419BF268525BF0E
:10E9E000829794485840B387A6003E8563E4D700D9
:10E9F000E3E5E7F63385E7408DB7B727002023A08E
:10EA0000A75011C5B727002005472382E750828011
:10EA1000B727002003A70750411122C406C613845C
:10EA2000075011C30297B727002083C7475093F7B9
:10EA3000F70F99E323200400B24022444101828071
:10EA4000011126CAB734002022CC4AC89387048219
:10EA500006CE4EC652C456C2DC2737290020938406
:10EA600004821304497B95E3B73700209387C7AC32
:10EA7000D833058B19CBF8339946639BE60AA382FA
:10EA80000700EF1060415C4482971C4491C3829759
:10EA900037240020B72900209307847803A7097D35
:10EAA0009033130A84788347847893961700BA9634
:10EAB0009622C9CA8347847863EEC7082304047882
:10EAC000373400209307C4AC9C371304C4AC639163
:10EAD0000710B727002083A7C77CF5C3DC40232895
:10EAE000FA006131B737002083A70780E9CB7C307B
:10EAF00011476366F70CB7370020938787B1DC278F
:10EB0000918BD5EFB727002083C7475093F7F70FB6
:10EB1000DDE783461A0003A6097D63C7D70C62446C
:10EB2000F240D2444249B249224A924A0561B1BBFD
:10EB3000F8339D46E39BE6F4A3820700EF10C0354F
:10EB40001C4899B7850793F7F70F2304F478E3EC93
:10EB5000C7F48DB786073E970E23231007000345A1
:10EB60008478B727002083A7077B13172500B72ACF
:10EB70000020BA979C4323940A7C829783D78A7C8F
:10EB80000347847893C7F7FF7D8D9317170003A77A
:10EB9000097D3E971E235D8D0AA38347847881C734
:10EBA00085072304F4788327497B81C78297232A2A
:10EBB000097A0347847883471A00E371F7F0F2403B
:10EBC0006244D2444249B249224A924A0561828053
:10EBD0007C3093F7F70FE39E07EEA30404009750F1
:10EBE00006E0E7806062F5B51397170032971A23A5
:10EBF00079F785071DB7374702408326C720F1778D
:10EC0000FD17F58F2326F72001000100B72700200C
:10EC100093878778C84F832787262326D7206A05BE
:10EC200093C7F7FF99835D8D8280B727002083C744
:10EC3000B77889CFB737002083C7C78291CBB73762
:10EC4000002003A307836307030002830545828036
:10EC5000094582801305F00F8280B737002003C674
:10EC60000798B727002003A7075781476315F600C9
:10EC7000814636858280BA8613078702835587FDD1
:10EC8000E389A5FE850793F7F70FCDB7B7370020C7
:10EC900003C71798B727002083A7C7582A860507F8
:10ECA00081463E859E236388C700850693076500DD
:10ECB000E3E9E6FE01458280B727002003A7475815
:10ECC00019E3014615A81C4703D8A700636B05018B
:10ECD00083584700B38608016355D5008146639485
:10ECE00016011843F1BF3E86C10703D3A7FF631780
:10ECF000A30099C123900501328582808506C20652
:10ED0000C182F1BFB737002003C60798B73700208C
:10ED100003A7079281476315F600814636858280F6
:10ED2000BA861307C703835567FCE389A5FE8507E9
:10ED300093F7F70FCDB7032785116DCB411122C48F
:10ED400006C65C258345E5042A8493F7C70F5CA5B6
:10ED50001437522713958601618563F7C506635101
:10ED60000506082793F6F60714B7054693E627002D
:10ED70006314C50093E6170054A45C4389075CC381
:10ED80004CB8032504112E864C430905EFF07F8112
:10ED9000832784115038D443DA27B296118FD4C315
:10EDA000DAA789473CBCB72700200347640383C721
:10EDB000A77E6371F7045C2493E707015CA41DA898
:10EDC00093E717005CA46DBF9376F60F63590502B5
:10EDD0000827854513E627006314B50013E61700DE
:10EDE00050A454B8A304070085473CBC8327841172
:10EDF0009C43D5FBB240224401454101828093E708
:10EE000017005CA454B8A3040700032504114C4365
:10EE10000905EFF00FF9832784115038D443DA271E
:10EE2000B296118FD4C3DAA78D47C1B7054582804A
:10EE3000B737002083A7C7AA411122C406C6858B15
:10EE40002A84D5E34165130525F5971006E0E78090
:10EE5000603E51C93C253EA583270412ADE3232023
:10EE6000A4122322A41285472311F40423200500B1
:10EE70007C2854415EA5583418A5054718B5373786
:10EE80000020032707AF1385170215811C437D154A
:10EE90001375F50F9CC25C43DCC21C479CC65C47E3
:10EEA000DCC61C4B9CCA5C4BDCCA1C4F9CCE5C4F26
:10EEB000DCCE19CD9386060213070702C1BF832754
:10EEC000441288C3835724042322A412850769BFF0
:10EED000B7370020938787989A2705079AA7B240EB
:10EEE0002244410182805C2423090400054593C724
:10EEF00047005CA4EDB71C2D93F7E70FC5EB1C3D55
:10EF0000D5E73029542509CA3727002083456503F2
:10EF10000347B77E63E7E50013F7060149CB0147D6
:10EF200009C6C18A0357E51B81C68356251C36973F
:10EF30003DCFB737002003D587821307C712374666
:10EF40000F00B335A702411113060624814622C4DF
:10EF500026C206C67D543305A70297D006E0E78097
:10EF600020AAB727002083C7F77EB384A700B7374E
:10EF7000002003A787A18327070963F387003E8446
:10EF8000184375FBB727002083A7C77C829781476A
:10EF90006364A400B307A440B2402244B3B797000F
:10EFA00093C7170092443E854101828081473E8588
:10EFB0008280B737002003A747AF7C53FDFF8280D4
:10EFC00001114EC6B73900209387899822CC03A43B
:10EFD000870926CAB7340020938704829E274AC82F
:10EFE000035964080325040906CE3309F902B7471B
:10EFF0000F001387F7239387072452C456C25AC0C1
:10F0000093898998938404823A993359F902636DFC
:10F010002503372A00208327CA7C3309254182979C
:10F020006367A9023309A9406346090283570404B0
:10F03000A30F040085072310F4048347041463948A
:10F0400007102285CD2511A2DC403E95D9B7DC40C2
:10F050003E99C9BF8327CA7C829703278408636FC0
:10F06000E508198D7E3C9A248E07B387E7021307C3
:10F07000003293870719B3D7E70263E5A708B74AB9
:10F080000F00138BFA23938A0A24835704048507FD
:10F090002310F4048347041499E32285692522850B
:10F0A000970006E0E780007E631D0524832604099F
:10F0B0008327C408D840B6973E8563E4D70063E44D
:10F0C000E7003385E7407C3C035964082328A40803
:10F0D00085077CBC9E243309F9025A993359590398
:10F0E000636C2505330925418327CA7C82976369B0
:10F0F000A9043305A940E34A05F80DBFDC40998F08
:10F100003E958DB7A1452285970006E0E780C06F48
:10F11000A305A402B737002003A3C7806303031E1F
:10F120006244F240D2444249B249224A924A024BD6
:10F130008945154505610283330927412A996DB731
:10F14000DC403E997DB7228551252285970006E057
:10F15000E78040736317051A8A2483576408B7460B
:10F160000F001386F623B387A7029386062403278E
:10F170000409230B040283AA4400B297B3D7D70231
:10F18000636BF718B307F7408326C4082324F408F9
:10F19000014BB387E6003E8963E4D70063E457017F
:10F1A000338957411E3023282409A1CB83560404F8
:10F1B0005A3037460F0056B03387E640B387E70230
:10F1C0003A301306062481468145BA97C207C183A7
:10F1D0003385A7023EB097D006E0E780608211CD6C
:10F1E0004A95333925012E99AA8763142B0163644C
:10F1F0005501B30755412328F4088327CA7C829719
:10F200002A898327CA7C8297E30D25FF8327CA7C3E
:10F210000329840882976365A9103305A940630A0E
:10F22000051083DA84008357640837490F001307F9
:10F23000F923B387570313090924BA97B3D72703D0
:10F24000372700200347F77EBA9763E4A70EB3354C
:10F250002503035A2402568681463305250397C0A9
:10F2600006E0E780E079330BAA0033055A033746FE
:10F270000F00130606248146814597C006E0E7800B
:10F2800020780DC1B337250356868146B305B902F0
:10F290003305A902BE9597C006E0E7806076330586
:10F2A000AA402AB03545975006E0E780400323ACDA
:10F2B000890838348547631DF700930700FD7CA457
:10F2C000B737002003A587ABDC24B1CFEFF0EFF216
:10F2D000B736002003A646AFB73700209387C7ACE8
:10F2E0001547F8B35846F977FD17F98F5CC60F102C
:10F2F000000083A746AF8966060B94C723A2670761
:10F30000D8C7F2406244D2444249B249224A924AA2
:10F31000024B05618280B3065701B387F640ADB555
:10F32000DC403E99DDBD8145970005E0E7800005A2
:10F3300045B7DC2423AC090885C3B737002003A5F3
:10F3400047AB970005E0E780003EB7E700E03707EE
:10F35000000223A2E72075B78347940285456244E3
:10F36000F240D2444249B249224A924A024BB395F2
:10F37000F500C205C18101450561170305E067007D
:10F3800003A2011122CC4AC84EC606CE26CA52C4D8
:10F3900056C25AC0383585472A842E8983290509E3
:10F3A0006315F71E83570508035BC503373A002032
:10F3B00093060A8283DA8600130A0A8263FF6719BA
:10F3C0001429639CE618032785116318071803277F
:10F3D000450A6314071874351D476390E6182A3DE3
:10F3E000330BFB409307204E330565038324440908
:10F3F00037460F001306062481463305F502B7276A
:10F40000002083C7E77EB3549502B3B5AA02BE9429
:10F41000C204C180231394083385AA0297C006E072
:10F42000E780005EAA9933B5A9002E954E87832701
:10F430004A0019E163E4F9003387F940B3845403C7
:10F44000B7460F009387F623938606242320E9000E
:10F45000BE94B3D4D40293171B00A6976369F70E2A
:10F460001D8F2320E900B729002083A7C97C8324AE
:10F470000900829763EEA4103385A440635D050AFA
:10F4800083A7C97C373B0020130B0B82829703278D
:10F4900009006365E510198D7E3C03578B008E07CC
:10F4A000B387E7021307003293870719B3D7E70240
:10F4B00063EBA70E374A0F00930AFA23130A0A24B4
:10F4C0008357040485072310F4048347041499E345
:10F4D0002285912C2285970006E0E780A03A6DE115
:10F4E000832604098327C40803274B00B6973E856B
:10F4F00063E4D70063E4E7003385E7407C3C835452
:10F5000064082328A40885077CBC83578B00B38438
:10F51000F402D694B3D444036363950CB3049540CA
:10F5200083A7C97C23209900829763EEA40A3385C0
:10F53000A440E34705F8B727002083C7F77E63E2BE
:10F54000A708B737002023A087A201459DA88326DE
:10F550004A00B387F6403E9729B783576408374778
:10F560000F00B38457039307F723A6979304072448
:10F57000B3D4970263E79900B3849940232099009C
:10F58000DDB583274A00BE99C5BF23A03501E1BD83
:10F59000B737002083A74782BE94F9BD83274B006D
:10F5A000998F3E95D5BDA1452285970006E0E7805D
:10F5B000A025A305A402B737002083A7C78081EF49
:10F5C0007D55F2406244D2444249B249224A924AAD
:10F5D000024B05618280894515458297D5B7B304F2
:10F5E0009740AA9435BF83274B00BE9489B721CD9D
:10F5F00001116C0022CC06CE2A84613339C1FD573B
:10F600006307F502B72600209386867DFC3A945660
:10F61000324791C285836360F702B307F7403EC665
:10F62000B24503459402970005E0E780208DF24043
:10F63000624405618280B736002083A646823697F1
:10F64000E9BFBD3AEDB78280B737002079711387E3
:10F6500087984AD00329070906D622D426D24ECE4F
:10F6600052CC56CA094763000906B7340020938A72
:10F6700087989387C4ACFC3395469384C4AC0D47FC
:10F680006383F604DC442A8A99CB975006E0E7802E
:10F690004008975006E0E780208723A60400FD5924
:10F6A0006C004A85F93915E937150020130505D591
:10F6B000EFF0AFB4A147DCA0B737002083A747AF76
:10F6C0000947F8D30D47B250225492540259F249D7
:10F6D000624AD24A3A854561828063743501324478
:10F6E000AA8903290900E31D09FAFD571307F00F42
:10F6F000E38BF9FC914763F187029307B4FF232062
:10F70000FA0023A2FA0A0147DDFFB737002083A7DA
:10F7100047822320FA0045BFB737002083A74782DE
:10F72000ED17A297E9BF797126D206D622D44AD026
:10F730004ECE52CC56CA5AC85EC6834755030344C0
:10F740007513AA843E941374F40F9307400263F672
:10F7500087001304B4FD1374F40F03AA841383AA5F
:10F76000C413A38B841222865285D68597C006E0E7
:10F77000E7804026058915E503CBD412014981496C
:10F78000337B6403930B50024A865285D68597C01B
:10F7900006E0E7802024058915C563916903137489
:10F7A000F90F238B8412B250225492540259F24919
:10F7B000624AD24A424BB24B456182808509E209D6
:10F7C00093D989410509E31179FDE1BF83278509B3
:10F7D00003560504797193D60701BD8EC206C18216
:10F7E000358E1357764093575640898B058B5D8F26
:10F7F00093573640918B5D8F93571640A18B5D8F49
:10F8000093171600C18B5D8F9317360093F707028D
:10F810005D8F931756009355860093F707041E06D5
:10F820005D8F1376F60F518F93D7554013D6354021
:10F83000118A898BD18F13D67540D18F13D615407D
:10F84000218AD18F13961500418AD18F13963500E6
:10F8500013760602D18F13965500137606049E0583
:10F86000D18F93F5F50FCD8FA20745465D8F3307F6
:10F87000C70222D42A8426D252CC56CA032A841321
:10F88000832AC4135AC806D6369742074183935732
:10F890007740135557400989858BC98F13553740D9
:10F8A0001189C98F135517402189C98F1315170066
:10F8B0004189C98F1315370013750502C98F1315B8
:10F8C000570093558700137505041E07C98F1377DA
:10F8D000F70FD98F13D5354013D755401189098BB0
:10F8E000498F13D57540498F13D515402189498F0C
:10F8F000139515004189498F13953500137505023D
:10F90000498F13955500137505049E05498F93F58E
:10F91000F50F4D8F2207D98FB387C7024AD04ECE3D
:10F920005EC662C4B697C207C18313D7774013D5AA
:10F9300057400989058B498F13D537401189498F65
:10F9400013D517402189498F139517004189498F95
:10F950001395370013750502498F1395570093D5FA
:10F960008700137505049E07498F93F7F70FD98F0A
:10F9700013D5354013D755401189098B498F13D5BD
:10F980007540498F13D515402189498F139515006E
:10F990004189498F1395350013750502498F1395D9
:10F9A0005500137505049E05498F93F5F50F4D8F8E
:10F9B0002207D98FB387C702130650025285D68516
:10F9C000B697BD8E93940601C18033F6C402137BB3
:10F9D000F60F97C006E0E780E0FF05890DED83474D
:10F9E000D41201498149B3849702130C5002C1809B
:10F9F0004A865285D68597C006E0E780A0FD058936
:10FA0000937BF90F11C563863403850993F9F90FC8
:10FA10000509E31F89FD230B6413B250225492544D
:10FA20000259F249624AD24A424BB24B224C4561DA
:10FA300082805E8BCDB70111B737002022CC03A4A2
:10FA400087A426CA4AC84EC606CEAA841309250032
:10FA5000854905C09C303830858B6304F700405CD5
:10FA6000CDBF1946930544004A85EFE09FC4E318D3
:10FA700035FF2285F2406244D2444249B2490561D1
:10FA800082804111B737002022C403A487A426C274
:10FA90004AC006C693042500054901E82285B24004
:10FAA00022449244024941018280A6851305A402A2
:10FAB000973006E0E780E0E0E30225FF405CF1BF1D
:10FAC0004111B737002022C403A487A426C24AC02C
:10FAD00006C693042500054901E82285B240224468
:10FAE0009244024941018280A6851305A401973002
:10FAF00006E0E78000DDE30225FF405CF1BF011175
:10FB0000B737002022CC03A407A426CA06CE2AC4F5
:10FB10002EC6854419E40145F2406244D244056191
:10FB200082809C841830858B6304F7000044DDB725
:10FB300019469305A10013052400EFE09FB7E317D2
:10FB400095FE0545D1BFB736002083A7C6AB130786
:10FB5000001098C323A0070018310348250022078E
:10FB6000420842970348050042970348350062085F
:10FB7000429798D7583103486500220742084297B8
:10FB80000348450042970348750062084297D8D75A
:10FB900018350348A500220742084297034885000C
:10FBA00042970348B5006208429798DB58350348EE
:10FBB000E5002207420842970348C500683542978E
:10FBC00062052A97D8DB9831A821220742052A9797
:10FBD00088212A97A83162052A9798CFD831E82141
:10FBE000220742052A97C8212A97E83162052A97F9
:10FBF000D8CF9835A825220742052A9788252A9725
:10FC0000A83562052A9798D3D835E82522074205FA
:10FC10002A97C825EC352A97E2052E97D8D3D843E2
:10FC2000759BD8C3D84313671700D8C3984313678D
:10FC3000170098C303A7C6AB5C43858BBDE71C4F79
:10FC400001451CA283A7C6AB9C4FA1831CB283A70E
:10FC5000C6AB9C4FC1833CA283A7C6AB9C4FE1833C
:10FC60003CB283A7C6ABD84F58A2D84F218358B215
:10FC7000D84F418378A2D84F618378B2985318A6A1
:10FC80009853218318B69853418338A698536183BB
:10FC900038B6D85358A6D853218358B6D853418381
:10FCA00078A6DC53E1837CB68280010061B7B73768
:10FCB000002003A747AF1605136505083C4B93E7E3
:10FCC00007083CCBB737002083A7C7AB03A7450E77
:10FCD00088C398CB03A7850E0145D8CB03A7C50BD6
:10FCE00098CF03A7050CD8CF03A7450C98D303A73B
:10FCF000850CD8D303A7C50C98D703A7050DD8D773
:10FD000003A7450D98DB03A7850DD8DB03A7C50D19
:10FD100098C703A7050ED8C798431367070498C36D
:10FD20008280B737002003A747AF16051365050883
:10FD30003C4B93E707083CCBB737002083A7C7AB02
:10FD400003A7C50E88C398CB03A7050F0145D8CBE1
:10FD500003A7C50B98CF03A7050CD8CF03A7450C65
:10FD600098D303A7850CD8D303A7C50C98D703A7AE
:10FD7000050DD8D703A7450D98DB03A7850DD8DB64
:10FD800003A7C50D98C703A7050ED8C798431367E7
:10FD9000070498C3B73700209387C7AC130700F850
:10FDA000F8A38280B736002003A706AC41114AC0F1
:10FDB0001C5F06C622C4998326C2858B3689B5CFBF
:10FDC00093070006373400201CDF8347C4AC93043C
:10FDD000C4AC93F7070489CFB727002083A7C77C5B
:10FDE0008297C8CC8347C4AC93F7F70B2306F4ACD7
:10FDF0008347C4AC93F7070285C38347C4AC373746
:10FE00000020032747AF93F7F70D2306F4ACDC4837
:10FE1000A16614C786077CD7DC2093F7070491EF0F
:10FE20008547DCB0B737002083A747AF096798C77D
:10FE3000130700FCD8A09848F8D3032709AC1C5F2F
:10FE40009183858B89CBC1471CDFB737002093870F
:10FE5000C7AC8546D4A31C5F9D83858B91CB93074C
:10FE600000081CDFB73700209387C7AC0547D8A32D
:10FE7000B737002083A7C7ABD8430583058B19C7C5
:10FE8000D843759BD8C3D843799BD8C3B24022448A
:10FE90009244024941018280B7370020B7360020E2
:10FEA00003A647AF9387C6AC03C7C6AC058B19E75B
:10FEB0009833058B01E7785265FBD833A38207009E
:10FEC000828037380020032708AC1C5F9583858B20
:10FED000BDE701C61C5BBD831CA29DC6832708AC81
:10FEE000985B4607935767016356070093E707C07F
:10FEF000C207C18303970600C207C18709C7BA9723
:10FF00000947B3C7E7029EA285C11C3191CF3E9538
:10FF10001C350547194593F6F7066393E602E20799
:10FF2000E187394563CE0700832708AC37370020C7
:10FF300001459C5FED838D8BA30BF7AC828005455B
:10FF40008280411122C406C63734002026C203270E
:10FF500044AF3DE5AE877453FDFEB7340020938473
:10FF6000C4AC3E85B28523810400974006E0E7805B
:10FF7000C00DB737002083A707ACB70680009843B1
:10FF8000558F98C3D857719BD8D7832744AFA38286
:10FF90000400A3800400094798C3832644AFB73701
:10FFA00000209387C7ACB823058B11E7B833058BC6
:10FFB00019E3F8526DFBB240224492444101828021
:10FFC0008D47631FF500B737002083A707ACB7063E
:10FFD00080009843558F98C3D857719BD8D775BF69
:10FFE0008547E31CF5FA5447F977FD17F58F5CC791
:10FFF0000F100000032744AF8967130600F81CC7E1
:020000025000AC
:10000000B73700209387C7ACD0A3B737002083A7AA
:1000100007AC9C43B1838D8B91E7930760197CD328
:1000200054C7A5BF9307E01BDDBF5D7152DC373AB3
:10003000002003270AAC86C6A2C4A6C2CAC04EDEF0
:100040001C43B73900203739002093F7F7E793E7CF
:1000500007081CC383A689B43707CEFF7D179C46CB
:10006000130680022A84F98F9CC6832749AF280093
:10007000AE8423A8070493051008EFE02FD9354577
:10008000974006E0E780A02583270AAC9376F41F0B
:100090003706330023A40700984B370FFCFF4E8828
:1000A0001367F70398CBF84FCA88130510F8137736
:1000B00007E0558FF8CF9843F576FD16758F98C3F6
:1000C00037370020832649AF1307C7ACA3020700C8
:1000D000A3000700054798C29843D285B7020400E1
:1000E0001377F7E798C39843930380251149137753
:1000F000F7E71367071098C303A789B47D1F8549E5
:100100001C47930F8002D18F1CC793079005BCCA70
:1001100001473400135337002693834703001376B7
:100120007700B3D7C740858BE1C383A705AC832E87
:1001300088B4239C07042390070603AECE02137EE7
:10014000DEFF23A6CE0383AE0700137EF70793FEE0
:100150000EF833EECE0123A0C70103AE4702336E83
:100160005E0023A2C70383AE48AF014E23A27E06E2
:1001700003DA070663074E0303AE0703038A06008C
:10018000135EFE00620E135E8E416358CA0103AE19
:100190000703135EFE002380C60103DE0706137EFD
:1001A000FE0F03AA4E0663060A0003DA8705E37F03
:1001B00049FB03AE4702337EEE0123A2C7038387C8
:1001C0000600635CF400034E03003396C900134637
:1001D000F6FF3376C6012300C3003E8663D3A70033
:1001E0002A8613158601618505071377F70F8506A3
:1001F000E312F7F3B640264496440649F259625A90
:1002000061618280B737002083A747AFD847931634
:10021000170163D2060298479316170163DD0600A3
:100220007D57B8D73727002013078778544F8506A6
:1002300054CF116798C798470D83058B11CF373777
:1002400000201307C7AC342393E6160034A39306AB
:1002500000F854A3214798C79847058B19CB373727
:1002600000201307C7AC143393E6160014B30547F8
:1002700098C798470983058B09E798470583058B3D
:1002800031CB373700201306C7ACA30206009447D2
:10029000B735002083A505AC8982858AE5C69441DF
:1002A000B1828D8AE9EEA84B54521376050294323E
:1002B0004DC2F9E29306D005D4CF8346C7AC93E68E
:1002C00016002306D7AC114798C7D855719B136702
:1002D0001700D8D598479316370163D406023737ED
:1002E00000209306879803C6060713078798418A5C
:1002F00045C203C70607136707022388E60605679A
:1003000098C798479316270163DF06003737002008
:100310001307C7AC5423E206E18663D40600854682
:1003200054A3096798C798479316070163D206023A
:10033000373700201307879883461707858AADCA89
:100340008346170793E62600A308D706216798C7B8
:100350008280ADD205466395C60093061006A9BFFC
:1003600009466395C60093065006B9B70D466395D6
:10037000C6009306900689B79306B00635BF93066C
:10038000C0061DBF38321367170038B209472DBFAA
:10039000834607070946BD8A6388C6008346070768
:1003A0000D46BD8AE39DC6F491462308D70681BF5A
:1003B00083461707918AD9DA8346170793E68600A2
:1003C00061B7B737002083A747AFB7360020138740
:1003D000C6AC904710CF90470D82058A11CA3023D2
:1003E0001366160030A3130600F850A3214690C7E9
:1003F0009047058A19C610331366160010B30546D8
:1004000090C790470982058A09E690470582058AC8
:1004100031C6A30207009047B735002083A505AC7D
:100420000982058A59CA904131820D8A41E6A84B5A
:10043000505313750502103221C935EA1306D00551
:10044000D0CF03C6C6AC136616002386C6AC914651
:1004500094C7D455F19A93E61600D4D594471396D1
:100460002601635B06005423E206E18663D406009E
:10047000854654A3096798C798479316070163D424
:100480000600216798C7828055DA05456315A600E6
:100490001306100675B709456315A6001306500626
:1004A00045B70D456315A6001306900651BF130608
:1004B000B00679B71306C00661B7343393E6160069
:1004C00034B3894671B737370020B736002013861A
:1004D00086AF130787B15C372C3E484AAE97FD8B39
:1004E000B355F5001CB25CB785898DE9183B814690
:1004F00013080002B3F7E7020147B355E500858909
:100500009378F70F89C96395D700A30016018280FD
:10051000850693F6F60F0507E31107FF8280B737CC
:1005200000209387C7ACDC3393F7F70FD1EBB727E5
:10053000002083A7C77C411122C44AC006C626C238
:10054000829737390020930789B18047130989B111
:100550006302A40663688504018DB7340020938785
:1005600084AFBC2F13545500938484AF6364F404A8
:1005700085676371F404813FBC2C0327890093963F
:10058000570036971D8C2324E900E376F4FE2244BD
:100590008830B2409244024981454101174306E048
:1005A0006700E31AB737002083A747823384874068
:1005B000229565B7B24022449244024941018280AB
:1005C0008280B727002083A7C77C011122CC26CACE
:1005D00052C406CE4AC84EC68297B73400209387CD
:1005E00084B18047014A6300A406938484B16365A3
:1005F0008506018D37370020930787AFBC2F135432
:100600005500137AF501130987AF636BF402B7390C
:10061000002093890982453D8346A90103A88400EF
:1006200083A54900139756004297158C3A86636458
:1006300007016364B7003306B74090C4E37DD4FC80
:100640001604336A4401F24062445285D24442495E
:10065000B249224A05618280B737002083A74782CA
:1006600033848740229579B7B737002003A747AF77
:100670008567938707777CD3B737002083A787B434
:1006800083A60709139656006358060083A6070938
:1006900013966600634406007453FDF282800000E6
:1006A000EFE00FB7730000000000000097020000A9
:1006B0009382820C0383020023800200630F0300F5
:1006C000F32510342EC0970500009385A5FD739087
:1006D0001534EFF01FCF7300203086DCEFF09FB2AF
:0806E000E650828000000000DA
:1006E800B72700203727002083A7077803278777B5
:1006F80001456313F7008280F62399E2D6233695E5
:100708009C43C5BFB727002083A5877D37270020D6
:100718009387877D138605222320C778DA2393875A
:1007280085FFB72600204111BA97056523ACF676F8
:1007380006C61D05935637006374E500930600202E
:100748003307D60037250020232EE57623A0E5229F
:10075800E11656A2231306001CC3998FE1175EA366
:1007680023130700B53FB240B72700202397A77887
:1007780041018280184183A785FF6319B7001CC116
:10078800FD5723AC05FE238FF5FE8280232CF6FE51
:10079800C5BF411122C426C23744024006C683247D
:1007A800C420232604200F10000009E923269420E2
:1007B8001545B24022449244410182800347E5FF37
:1007C8009307F00F6306F700232694201145D5B749
:1007D8009700FB1FE7808093014523269420D1BF13
:1007E800411126C24AC0B744024006C622C403A922
:1007F800C42023A604200F10000089E523A6242185
:10080800154515A0B727002083C797782A842E8519
:100818006375F400894763EE8700A53FB747024038
:1008280023A627210D45B2402244924402494101A2
:10083800828083A785FF99E703C7E5FF9307F00F39
:100848006308F700B937B747024023A627214DBFF1
:1008580037250020238F85FE130545789700FB1F59
:10086800E780809BA16522856D2C014523A6242164
:100878005DBFB727002023A207788280BDCD79719C
:1008880022D406D626D24AD04ECE01444147B3D709
:100898008540858BB1CF1205314722953305E50296
:1008A800B737002003A987818544B3948400C20424
:1008B800C180BE892A990327090011C70325490069
:1008C8002EC60297B24531473304E40283A78981D3
:1008D8003E941C4489E72320090023220900B250D2
:1008E8002254A58D02599254F2492E854561828081
:1008F8000504E31EE4F88144DDB72E8582804111AA
:100908001397050122C406C626C24AC041872E8411
:10091800635107029700FB1FE780009711C1953DBF
:10092800A1673D8C2285B24022449244024941018C
:100938008280EDD9AA8701474146B356E440858AAB
:100948009DCA9207BA97B146B387D702B736002037
:1009580003A986818544B394E400C204C1803E990A
:1009680083270900032549008297232009002322B1
:100978000900258C45BF0507E311C7FC8144D5BF95
:10098800411126C2B747024006C622C483A4C72025
:1009980023A607200F100000B727002083A7C77FD2
:1009A800372400201304044D91C782971C403E95BC
:1009B80008C031A0B727002083A7C77CFDF71C40DB
:1009C800374703001307D73FB387E70237A7260047
:1009D800130737ECB240BA971CC0B747024023A6AA
:1009E800972008402244924441018280797126D29E
:1009F800B747024006D622D44AD04ECE52CC56CA69
:100A08005AC85EC662C483A4C72023A607200F1055
:100A1800000005E123A697200945B25022549254BC
:100A28000259F249624AD24A424BB24B224C4561C2
:100A38008280B727002083A7C77CBA8A368AB28B00
:100A48002E8BAA898297B737002003A787813E8912
:100A58000144B146C147330CD40233068701104222
:100A680059E2C165938505F0414597F0FA1FE78083
:100A7800E05C19EDB737002083A7C78081C781459F
:100A880011458297B747024023A697202D4571B795
:100A9800B727002003A7477D39E323AAA77C2300B3
:100AA800050083278981054733178700232605001A
:100AB800232475013AA123225501E29723A0370187
:100AC80023A2670123A4570163040A0023008A00B4
:100AD800B747024023A69720014581B73E875C4768
:100AE800F5FF48C76DBF0504E317F4F6B7470240A2
:100AF80023A69720214515B7B737002083A7C781BC
:100B0800411122C406C6372400201304847889C7FB
:100B180082975C483E9548C84848B2402244410103
:100B28008280B747024083A6C72023A607200F105C
:100B3800000037270020034797786370E5023726BF
:100B48000020131715000325067D3A951A21D98D23
:100B58000EA123A6D7200145828023A6D7200D45C4
:100B68008280B747024083A6C72023A607200F101C
:100B7800000037270020034797786372E50237267D
:100B88000020131715000325067D93C5F5FF3A9538
:100B98001A21F98D0EA123A6D7200145828023A60C
:100BA800D7200D45828001114AC83747024006CE3A
:100BB80022CC26CA4EC652C40329C72023260720A2
:100BC8000F100000130705FF1377F70FFD4763E3C6
:100BD800E70AB146B306D502B737002003A78781D5
:100BE80036971C43C1CB9354450005443D893315C2
:100BF800A400131405014180AE892685A28597F0CB
:100C0800FA1FE780E0702A8A29C9A2852685913FC4
:100C1800B727002083A7C77CB734002093840482B9
:100C280082979E242A848146B3853703130600647D
:100C3800B3B7370313850532B335B500BE95EFC09A
:100C48007134B30785003E87D44063E4A70063E4AA
:100C5800D7003387D7402324EA00B747024023A6AA
:100C680027210145F2406244D2444249B249224A0E
:100C780005618280B747024023A627210945DDB7D1
:100C880001114AC8B747024006CE22CC26CA4EC632
:100C980003A9C72023A607200F100000BD4763EB58
:100CA800A70431473307E502B737002083A78781B8
:100CB800BA979C43A1C305443314A400420441805D
:100CC800AE840145A28597F0FA1FE7806064AA897F
:100CD80011C5A2850145713523A49900B747024083
:100CE80023A627210145F2406244D2444249B24931
:100CF80005618280B747024023A627210945E5B749
:100D0800797126D252CCB744024006D622D44AD0B2
:100D18004ECE56CA5AC85EC603AAC42023A60420CB
:100D28000F100000B727002083C797786378F50075
:100D3800B727002083ABC77C63970B00B7470240F7
:100D480023A6472199A03739002013090982AE8AC2
:100D5800032B490083558900B74736FE938707C898
:100D68003E9BB387C5022A84B2898146B3B5C502C2
:100D780013850732B337F50013060064BE95EFC03C
:100D880071206370AB0223A644210145B25022545E
:100D980092540259F249624AD24A424BB24B4561D7
:100DA8008280829B83558900AA8413060064B387D6
:100DB80035038146B3B5350313850732B337F500DC
:100DC800BE95EFC0311CB3079500BE8403274900C8
:100DD80063E4A70063E4E700B384E740D68522858F
:100DE80097F0FA1FE780C05201C904C5B74702400F
:100DF80023A64721054559BF936504F0C205C18163
:100E0800414597F0FA1FE780602311E9B7370020C2
:100E180083A7C78085D7A2851145829705B737274D
:100E280000208327477D99EF232AA77C854723261F
:100E3800050004C52311550100A11CB1232205009A
:100E480075B7BA87D84775FFC8C7CDB779714ECE81
:100E5800B747024006D622D426D24AD052CC56CA28
:100E68005AC85EC662C466C26AC083A9C72023A6E0
:100E780007200F10000025C141443689B28A2E8A06
:100E8800AA84B14C373B0020054D130C0003B30B6B
:100E9800940303278B815E971C43B9EF9375F40085
:100EA800B315BD0013554440C2055686C18113755C
:100EB800F50FB93531C183278B81DE9784C323A20F
:100EC80047016304090023008900B747024023A6AD
:100ED8003721014521A023A637210945B2502254C4
:100EE80092540259F249624AD24A424BB24B224CBE
:100EF800924C024D456182800504E31A84F9B74794
:100F0800024023A637212145D1BF011122CC26CA90
:100F18004AC84EC6B747024006CE03A9C7202A844E
:100F2800AE89B28423A607200F100000D13B22858A
:100F3800CE8597F0FA1FE780A03D2A8405C5B7370C
:100F4800002083D58782130600648146B387950203
:100F5800B3B5950213850732B337F500BE95EFC0D8
:100F6800710248C013351400F2406244B74702408A
:100F780023A62721D2444249B2490E050561828041
:100F8800011122CC4AC84EC6B747024006CE26CA2F
:100F980083A9C7202A892E8423A607200F100000C2
:100FA80097F0FA1FE780C036AA8419C123110500FB
:100FB800A2854A857D36B727002083C7877863993D
:100FC8002701B727002003D7877C598C2394877C77
:100FD800B747024023A63721014591E01945F24061
:100FE8006244D2444249B24905618280011126CA4D
:100FF8004AC8B744024006CE22CC4EC603A9C42034
:1010080023A604200F1000009307F00263E6A7044C
:10101800B1473304F502B739002083A78981A29725
:101028009C439DCB9377F5008545B395F500C205A4
:10103800C1811181B13783A789810145A29723A076
:10104800070023A2070023A62421F2406244D244C9
:101058004249B24905618280B747024023A6272149
:101068000945E5B7411126C206C622C4B747024062
:1010780083A4C72023A607200F10000097F0FA1FAB
:10108800E780002919E90145B2402244B7470240E8
:1010980023A69720924441018280B727002083A786
:1010A800C77C00458297B73700209387078263671C
:1010B800A402D843B74636FE938606C83305A44033
:1010C8003697E372E5FC13070064B335E50292270F
:1010D80081463305E502EFC0E16A7DB7D8433A940B
:1010E800C9BF4111B737002006C623AEA7800295B5
:1010F800B240B727002023A0A77A0145410182808A
:10110800914763E9B700B72700208A059387477B93
:10111800BE9588C18280B727002023AA077C37257F
:101128000020B7370020411123AE07805146B7276A
:10113800002081451305457B06C623A6077C22C4EB
:1011480026C23724002097F0FA1FE780E024130511
:10115800847813068002814597F0FA1FE780C02340
:10116800EFF04FDAB727002083C7D77E13048478BF
:10117800854513D527008D8B3E958D473305F502A0
:101188009947B734002039051375F50F28A03305A2
:10119800F5021305052497F0FA1FE78020EA23AC2F
:1011A800A4802DCD3020994781453306F6021306D9
:1011B800062497F0FA1FE780201E83A78481382031
:1011C800B7240020938707240A0723A8F47ABA973C
:1011D800372700202328F77CEFF0AFE939291C30A6
:1011E80083A6047B37160500139727003697130646
:1011F800468810C3138717001377F70F0A073716A7
:10120800050036971306669010C3138737008907C1
:1012180093F7F70F8A0718B0B69790C3B2402244E5
:1012280092444101828037270020130787781C33B6
:10123800342363FFD700B726002083A6067B1386D6
:10124800170010B313972700369708C33E8582808E
:101258009307F00FE5BF1C41F1CF41777D8FB706AB
:10126800002089476319D70C5A2171C7411126C23A
:101278001946AA849305F00F610506C622C497F0A3
:10128800FA1FE780602305478D47630FE5089C44F4
:1012980091C7985C994749CBD85C59C73724002037
:1012A8001306000481451305847D97F0FA1FE78033
:1012B800A00E13060004A6851305847D97F0FA1F77
:1012C800E780E0069307847DDA2701E7130700101B
:1012D800DAA7F82719E30547F8A79A2B19E36D470A
:1012E8009AABF83719E31547F8B7B82B19E3054750
:1012F800B8ABB83B19E3F837B8BBD82B19E3254787
:10130800D8ABF82801E71307C003F8ABDC5791C73F
:101318008297B72700202398A778B73700207D57F2
:10132800A386E7BACD3B8147B240224492443E852A
:101338004101828089473E85828001114AC8373938
:1013480000208327098206CE22CC26CA52C456C260
:101358004EC68297130A0064B33545031309098200
:10136800835A89008146568633054503EFC081417B
:10137800B727002013878778004FAA8401456306A2
:1013880094029389877833858440636E940003259B
:10139800490056868146B335AA023305AA02EFC032
:1013A800613E018D269523AC9900F2406244D244F7
:1013B8004249B249224A924A05618280011122CCEF
:1013C8002E84B7E506000A854146938505BD06CEFD
:1013D800EFC06174180806043A94B7370020035523
:1013E80004FF83D7A782F2406244AA9737450F00CB
:1013F800130505243355F50205618280B7370020AF
:1014080083D7A78251471D45637CF7027947194561
:101418006378F7021307200315456373F702130770
:10142800B0041145637EF700130740060D45637944
:10143800F7001307600909456374F70013B5B70F80
:101448008280011122CC06CE2A842EC6EFF04FD31B
:10145800B245F240818D33A5A502229562441375E9
:10146800F50F05618280011122CC06CE2A842EC692
:10147800EFF00FD1B245F240818D33A5A502229538
:1014880062444205418105618280011122CC06CE69
:101498002A842EC6EFF0CFCEB245F240818D33B507
:1014A800A5022295624405618280B737002023A8EF
:1014B800A7828280B72700201387877D585739CFA6
:1014C800411122C426C24AC006C61389877D0297E5
:1014D800B7270020138787781A272A849384877868
:1014E80005CBBA876373A700AA87C207C183BA86E8
:1014F8006373E400A286C206C182958F514763597F
:10150800F7008327090391C38297EF40F16282A411
:10151800B2402244924402494101828082800111F2
:1015280022CC372400209307847D9C5B06CEAA85B5
:101538001304847D81C72AC68297B245C9C19C41DC
:101548000545B5CBDC41A5CB9E25B5C7BE25A5C7AE
:10155800DC2589CB5C3813F737008983BA970947AC
:10156800634BF7043735002041461305058297F091
:10157800FA1FE780C0DBB737002083A6078237272A
:1015880000202326D77C78380DE3938707828A27A3
:101598009307805737460F003305F50213060624D4
:1015A80081468145EFC0011E68B83715050013054F
:1015B8002534053E0145F240624405618280B72723
:1015C8000020938787783717002023AE070013077A
:1015D8006798B737002023A0E782378732009387C0
:1015E8000782FD56130727A1D4C398C7238607008F
:1015F800B747024023A4D726BDBF011122CC372408
:1016080000209307847D884706CE26CA4AC801E988
:101618000545F2406244D244424905618280130480
:10162800847D1C5CF5D7585C65D77000854582972A
:101638001844B247E30EF7FC4A249305E004B724A4
:10164800002097F0FA1FE780609F1387847808D3FB
:101658009384847855DD52249305F00F014997F05F
:10166800FA1FE78060D37C249050634DF9003285DF
:1016780097F0FA1FE78080A9014523A0040223A25E
:10168800040241BF4E240844585CB387250389816E
:1016980005093E9508C20297F9B701114EC6B72948
:1016A80000209387897D9C4726CA4AC852C406CE23
:1016B80022CC56C25AC02A8AAE8432896388071E51
:1016C8009389897D03A78903630207121307F01F13
:1016D8006360A7123724002013078478832A07023F
:1016E8001304847863980A0803D5C900956593851F
:1016F80015E097F0FA1FE780609408D02A867DC528
:1017080083D5C90083A7890303A5890089818297A6
:1017180083A78900832A04025CD089476314FA08E6
:10172800C1476395F40C83D5C9009147938505FC9F
:10173800B3C5F5028A05D695B8219307A0056313AA
:10174800F70A9E216390470B4A852686910597F0F4
:10175800FA1FE780C0BD1C50568563915713014599
:10176800F2406244D2444249B249224A924A024B68
:10177800056182805850E382E7FA03D5C900956570
:10178800938525E097F0FA1FE780408BAA8A39CD28
:1017980083D5C9002A8683A7890303A5890089817F
:1017A8008297A5BF8D47631BFA00C1476390F40475
:1017B80083D5C900938545FDF199B5BF9147631855
:1017C800FA006395440383D5C900A115F5B79307BB
:1017D8000010631DFA00A14763EA970083D5C9008A
:1017E800C115D9BF1C505685639D570B29458DBF20
:1017F8009D6A637A5509930A05E01947B3CAEA0254
:1018080003D7C900372B0020B38AEA02BE9A930790
:101818008B78DC53130B8B786395570103240B02E9
:101828001DE003D5C9009305E00497F0FA1FE7808F
:10183800E0802A8445DD83D5C90083A789032A86E9
:1018480089815685829791451307A00589819397C9
:101858002500A297B4236391E6049623639C46036C
:1018680085058A052686A2954A8597F0FA1FE7809E
:1018780000AC83270B02E38487EE228597F0FA1FDA
:10188800E780C088E9BD21677917E361A7F6B30A45
:101898005541BDB7AC335DBF83270B02E38887F49E
:1018A800228597F0FA1FE780608689B7B72700205E
:1018B80083A5877A85DD91479306A00589831397C9
:1018C80027002E973023E313D6F21223631C460118
:1018D80085078A072686BE954A8597F0FA1FE7800E
:1018E80000A5B5BD3C33D9BFB72700209387877DB6
:1018F800984721C3D85F15CF8546631CD50241118F
:1019080022C43724002013048478105006C611CE50
:10191800CE27485089810297085097E0FA1FE78040
:10192800E07E2320040223220402B2402244410123
:1019380082808280011122CC372400209307847D85
:1019480056C283AA870026CA4AC84EC606CE52C4C3
:101958002A89AE84B2891304847D638D0A1A5C5C7B
:1019680099EB2945F2406244D2444249B249224A9D
:10197800924A056182801C5CEDD79307F01F63E1F2
:10198800A70C372A002093078A789C53130A8A7871
:10199800A9C7084483274A02639CA704894763139D
:1019A800F906C147E39FF4FA4A249147130505FC59
:1019B8003345F5029317250003250A022686CE85AE
:1019C8003E959307A0053CA123102501110597F02A
:1019D800FA1FE780C095014571B74A249305E004D2
:1019E80097E0FA1FE78080652320AA025DF195BF82
:1019F8004E241C5C03260A02898182971C442322F8
:101A0800FA0269BF8D47631BF900C147E39BF4F4F1
:101A18004A24130545FD9377C5FF79BF914763179E
:101A2800F900E39024F54A242115F5B7930700102F
:101A3800E319F9F2A147E3E697F24A244115E1BF19
:101A48009D676375F506930705E01947B3C7E70275
:101A58005A24372A0020B387E702BE9A93078A7868
:101A68009C53130A8A78B1CB83274A02639257079B
:101A780003250A0291461308A0059305F00F93D792
:101A88002600139727002A973023631206078358E6
:101A98000700303363992805B306D64063C496041B
:101AA80085078A072686CE853E9515B7216779175B
:101AB800E369A7EAB307F54061BF4A249305E00448
:101AC80097E0FA1FE78080572320AA0251FD51BDF5
:101AD8004E241C5C03260A0289815685829723229C
:101AE8005A0379B70EA393160601C18249BF52243F
:101AF800B38596009105130606FCE3F4C5E6138644
:101B08003400719A1106B2962301070123102701A8
:101B180034B379B7372A002093078A789C53130A7D
:101B28008A7895CF03250A0291461308A0059305E4
:101B3800F00F93D72600139727002A9730236310B6
:101B4800060583580700303363972801B306D6404B
:101B5800E3D896F40EA393160601C182D9BF682470
:101B68005E249305E0043305F5024205418197E0C0
:101B7800FA1FE780A04C2320AA024DF5DDB35224BA
:101B88006C24B385C502338696001106E3EBC5DCE9
:101B9800BDB7014582809C211CA1BE211CB1BE217C
:101BA800A1833CA1DC213CB111458280B7270020EC
:101BB80023A60750B727002023A4075082800DCD05
:101BC800411126C206C622C4AA8401458DC12E84AD
:101BD800B7E5060022854146938505BE97E0FA1FC2
:101BE800E780E0749C2005455CA49C305CB4B2405E
:101BF800224492444101828001458280011122CC15
:101C080026CA06CE0947AA8432846381E504414680
:101C18008147639BC500638FE6006397B6000DA8F4
:101C280041478147638EE600F2406244D2443E85D4
:101C3800056182808A852285593741468A8519A897
:101C48008A85B53F41468A85228531A0E39AB6FC4C
:101C58002E86A285268597E0FA1FE780407EAA8710
:101C6800E1B7B727002023A4A7508280B727002018
:101C780023A6A7508280011122CC622106CE26CA53
:101C88004AC84EC62DCC83298500AE842A8803C94C
:101C98000900814713178901618763550702B14716
:101CA800054563F787045114420403552800418011
:101CB80033878900A2864E868545EFA0C020B337BA
:101CC800A00085077D14135569004204058913791E
:101CD800F90341809CA088B023812401C2A0014758
:101CE80019C01387190098C409476383E7000145A1
:101CF800F2406244D2444249B249056182800545B6
:101D0800C5BFC167F917630AF502D94763F7B70278
:101D1800011122CC2EC606CE2A84EF701028B245B7
:101D28006368B50022856244F24005616F90A0198E
:101D3800F240624405450561828005458280C1679D
:101D4800F9176314F5006F705025411106C6EF901E
:101D5800000611E15D45B240410182809147639DD3
:101D6800F5001C211CA23C211831A207D98F3EA2E4
:101D78003C3101455CA28280114582804111814538
:101D880022C426C206C6AA84BD232A8409E9B72725
:101D9800002083A7875081C7F94526858297228529
:101DA800B240224492444101828039714ED656D2C3
:101DB8005AD006DE22DC26DA4AD852D4AA8A2E8BDA
:101DC800B28951EB36C6A53F9145EF70B02BAA8476
:101DD8004D493DC5B246054A238034010544630A8E
:101DE8000B00B68513851400029B05051314050125
:101DF8004180E20993D9894163D30902C1455685D7
:101E0800EF904009654915E533868400A28526854B
:101E1800EF90505D2A8911ED3104420441809147C9
:101E28002C085685FC8426CEE085EF8010222A896E
:101E380001C963070A00268597E0FA1FE780002D8D
:101E4800F25062544A85D2544259B259225A925A8F
:101E5800025B21618280BA84014ABDBF011122CC94
:101E680026CA4AC84EC606CE2A893284B689353F64
:101E7800AA840DE1B727002083A7C75081CF054763
:101E88006317E40003C4090005041374F40FA28562
:101E98004A858297F240624426854249D244B24933
:101EA80005618280AE86B725050001470546938502
:101EB800E5B96DB79E211CA19E21A1831CB10945DE
:101EC80082809E211CA19E21A1831CB1BE213CA120
:101ED800BE21A1833CB1114582809E211CA19E2177
:101EE800A1831CB1BE213CA1BE21A1833CB1DC3140
:101EF8005CA1FC215CB18A251905420541818280DB
:101F08009E211CA19E21A1831CB1094582809E218E
:101F18001CA19E21A1831CB1BE213CA1BE21A1838D
:101F28003CB111458280CA21060542054181828063
:101F38009E211CA19E21A1831CB1AA21090542054D
:101F4800418182809E211CA19E21A1831CB1BE21BA
:101F58003CA1BE21A1833CB1CA21110542054181A2
:101F680082809C211CA1054582809E21411122C4AA
:101F780006C61CA19E212E841105A183A30EF5FE81
:101F8800BE219505230FF5FE83D7D5FFA183A30FA7
:101F9800F5FE03C6F5FF97E0FA1FE78040394820B1
:101FA800B240224411054101828089476399F500B6
:101FB8001C3118210145A207D98F1EA28280114524
:101FC80082809A21D94763FDE702011122CC06CE0F
:101FD8002EC62A84EF70607CB2469E22636DF5009F
:101FE80022856244F240B7250500014709469385DA
:101FF800C5EB05615DBBF24062440945056182801D
:1020080009458280914785C51421FD15C20585477C
:10201800C1816390F60213D725008D89914781E924
:10202800914711C7050534A21AA248C281473E85C7
:10203800828009479147E39CE6FEC94733D7F502FA
:10204800B3F5F502E1BFAE86B72505000147114695
:102058009385A5EC99BB93F7350089EB8981914766
:1020680081C50EA248C281473E8582809147EDBF57
:10207800D8218947631CF702011122CC2A84C8455C
:1020880006CEAE86014709C92EC69D4597E0FA1FC0
:10209800E7800015B2462A8722856244F240B725B8
:1020A80005001946938525EE056101B3094582802F
:1020B80099E1114582801C2105473EA2E37BF7FE8A
:1020C800FD1593F5F50F33D7F502B387E702E392D1
:1020D800F5FE050548C21AA201458280DC210947A0
:1020E800AE866385E70041476399E700B725050099
:1020F80001472146938525F74DB9094582800EA2EF
:1021080091E1014548C201458280AE86B7250500A8
:1021180001472946938585F049B90EA291E1014509
:1021280048C201458280AE86B72505000147314681
:10213800938565F19DB90EA291E1014548C201451B
:102148008280DA21854763FFE702011122CC2A84C5
:10215800884106CE1DC12EC6854597E0FA1FE78047
:1021680020082A8722856244B246F240B725050036
:1021780039469385E5F205610DB9F2406244094597
:102188000561828009458280914785C518218D4661
:10219800914763F0E602FD15C205C181B3C6E502A9
:1021A8003308D70263970501050516A23AA248C26B
:1021B80081473E858280DC210947AE866385E7003A
:1021C80041476399E700B7250500014741469385D4
:1021D80025F7E1BE09458280B335B0001395250087
:1021E8008280011122CC26CA06CE98258547AA846A
:1021F8002E844946631FF70099363E204915130679
:10220800200963C8A700F2406244D2440945056129
:102218008280183485476314F70013660604484023
:1022280001C98D4532C697E0FA1FE78060FB324648
:10223800A2866244F2402A872685D244B725050043
:10224800938585F3056195B68D4763F8B7021C3110
:102258001821F115A207D98F1EA23C313821C205D9
:10226800A207C181D98F3EA24EA289C5110508C611
:102278000145828023240600E5BF114582800111B3
:1022880022CC2A84884506CEAE8601C92EC695453D
:1022980097E0FA1FE780C0F4B2462A872285624495
:1022A800F240B725050059469385C5F40561F5BC8C
:1022B800B335B000139525008280AE86B72505009A
:1022C800014761469385A5F6CDB48547114563F06E
:1022D800D7021C320C22A207CD8F1EA39387E6FFDC
:1022E8003EA389476386F600090650C301458280EC
:1022F80023220700E5BF014781467946814575B429
:102308009E211CA19E21A1831CB109458280BC216C
:1023180005471CA18A216397E7000A0505054205C0
:1023280041818280C9473305F502CDBF8A210A055C
:10233800420541818280BE211CA18A21BE2133052C
:10234800F50205054205418182808A2182808A2121
:1023580082808A218280BE211CA18A21BE21330568
:10236800F50205054205418182809E211CA19E211E
:10237800A1831CB1BE213CA1BE21A1833CB1CA21CD
:1023880011054205418182809E211CA19E21A183C5
:102398001CB1AA210905420541818280894711455E
:1023A8006398F6001C3214220145A207D58F1EA39C
:1023B80082809A21D947AE8663F9E700B7250500E0
:1023C80001470D469385853051BC094582801145EA
:1023D800639DA6001C3214220145A207D58F1EA3B7
:1023E8003C323422A207D58F3EA38280BC21054708
:1023F800FD1793F7F70F6361F7049E2195CF01113D
:1024080022CC2A84C84106CE1DC12EC6894597E034
:10241800FA1FE780E0DC2A8722856244B246F24050
:10242800B7250500154693856531056105BCF24061
:1024380062440945056182800945828095471145B6
:1024480063F1D706411122C426C24AC006C61C320F
:10245800BA841822A2073284D98F9EA03C3238222F
:1024680093054400A207D98FBEA08947DCA009467E
:1024780013855400368997E0FA1FE78040EB9307ED
:10248800A9FF9EA49947631BF90023A60400B24044
:102498002244924402490145410182801904C0C482
:1024A800FDB782809E2195CF011122CC2A84C84194
:1024B80006CE1DC12EC6854597E0FA1FE78040D29B
:1024C8002A8722856244B246F240B72505001D4698
:1024D80093854533056159B2F24062440945056167
:1024E8008280094582809947639DF6028947411198
:1024F80006C65CA31C321422B285A207D58F1EA380
:102508003C3234225023A207D58F130557003EA32F
:10251800910597E0FA1FE78080E1B240014541014B
:102528008280D14711456394F600C147C9B78280BC
:102538009E219DCF011122CC2A84C84106CE05C513
:102548002EC6894597E0FA1FE78080C92A87228529
:102558006244B246F240B725050025469385E53327
:1025680005616FF0BF8FF2406244094505618280C2
:1025780009458280894711456398F6001C32142268
:102588000145A207D58F1EA38280011122CC2A847F
:10259800C84106CEAE86014709C92EC6854597E0D3
:1025A800FA1FE780E0C3B2462A8722856244F240D8
:1025B800B72505002D469385253505616FF01F8ADF
:1025C8001145639DA6001C3214220145A207D58F30
:1025D8001EA33C323422A207D58F3EA3828001116C
:1025E80022CC2A84C84106CEAE8601C92EC68545AE
:1025F80097E0FA1FE780C0BEB2462A872285624468
:10260800F240B725050035469385653505616FF0BD
:10261800FF8493F71600114581EB89476386F6001E
:10262800858256A310C301458280011122CC2A84D9
:10263800C84106CE05C52EC6854597E0FA1FE78036
:1026480020BA2A8722856244B246F240B72505009F
:102658003D469385A53505616FF05F80F240624481
:102668000945056182809E219DCF011122CC2A84D3
:10267800C84106CE05C52EC6894597E0FA1FE780F2
:1026880020B62A8722856244B246F240B725050063
:1026980045469385E53505616FF04FFCF24062448D
:1026A80009450561828009458280854763F6D7021E
:1026B80008A70CB71C320C22A207CD8F1EA3938744
:1026C800E6FF3EA389476386F600090650C3014525
:1026D800828023220700E5BF114582800147814699
:1026E8004D4681456FF08FF78D47114563F4D7024A
:1026F8001C320C22A207CD8F1EA33C322C22A2072B
:10270800CD8F3EA39387C6FF5EA36386A6001106FE
:1027180010C70145828023240700E5BF011122CCA0
:102728002A84884506CEAE8601C92EC6954597E00F
:10273800FA1FE780E0AAB2462A8722856244F2405F
:10274800B72505005D469385253705616FF00FF1C4
:10275800854711456395F6001C2201451CA382801C
:1027680001478146654681456FF04FEF011122CC44
:102778002A84C84106CEAE86014709C92EC68D45B2
:1027880097E0FA1FE780C0A5B2462A8722856244EF
:10279800F240B72505006D469385053905616FF050
:1027A800CFE0011122CC2A84C84106CEAE8601476B
:1027B80009C92EC68D4597E0FA1FE78060A2B24688
:1027C8002A8722856244F240B7250500754693851D
:1027D800053905616FF06FDD011106CE2EC6EF8059
:1027E800205919C5B245F2402A2105616FC0402D14
:1027F800F240494505618280B7270020A38C075223
:10280800B7270020238C0752B727002023A00752A0
:10281800B727002023A20752B727002023A4075276
:10282800B727002023A60752B727002023AE07505A
:10283800B727002023AC0750B7370020239A078416
:102848001306403893874785B2B371761307400B58
:10285800130606B8BAA3D2B311671D46930600053E
:102868009305000A1305007DDAA3F2B34147054634
:10287800130810F8BAA7DAA7BAABDAABFAAB9AAF73
:102888009AB723960703EEA38EA7F6A796ABAAAF2F
:10289800239E0700239F070023900702B2B72397C0
:1028A80007021308F007239807022392E7042393EB
:1028B800E704239FE7042390E7062391E706239282
:1028C800E706239907031307C01CD2BBF2BB239C5E
:1028D8000702239D0702239E0702239F07022390D6
:1028E80007042391C7042394070423950704239618
:1028F800C7042397D7042398D7042399A704239AB6
:102908000704239B0704239C0704239DD704239EC5
:10291800D7042393A706239407062395070623962F
:1029280007062397B7062398B70623990706239A1D
:10293800E7067D57239B070623900708239107087E
:102948002392E7088280011126CAAA84214522CC55
:1029580006CE2E8432C636C43AC297E0FA1FE78004
:10296800408D0DC5A24612473246930700FD1CA1B3
:10297800994704B13CA174A178B152A1AA852285D6
:102988006244F240D24405616FD09FE5F240624450
:10299800D24405618280B727002023A4A7528280F1
:1029A800B727002023A6A7528280011122CC4AC84B
:1029B80006CE26CA2A890144B30489006368B40094
:1029C800F2406244D2444249056182802EC6EFD06B
:1029D8003FFB93170501C183A183B2459CA09307D0
:1029E800140093F7F70F850463F8B700CA97090432
:1029F80088A31374F40FC9B73E84C9B7411122C420
:102A080037340020130444836A20C16706C6FD17C3
:102A1800630EF500B737002003C68797B725002057
:102A280093850553EF800018FD577EA0B2402244DD
:102A38004101828009C925151375F50F1335850ED7
:102A48001345150082800145828023900500C1C688
:102A5800797122D426D24ECE52CC5AC806D64AD044
:102A680056CA5EC63684328AAE892A8B814463F29E
:102A78004407B30794009C23138914004209939ACE
:102A8800070193DA0A011359090163840A04CA97F2
:102A98006341FA04B307240183CB07005E85593FDD
:102AA8000DC99387FAFF2390F90063906B03130510
:102AB80019002295B250225492540259F249624A9E
:102AC800D24A424BB24B45618280D694C204C1803F
:102AD80079BF0145C5B701458280011122CC373441
:102AE800002026CA4AC84EC69307448306CE2E89BC
:102AF800D0CB8CCBC8C7AA8441469305F00F4A8532
:102B080097E0FA1FE780409B8549130444836319C3
:102B180035030848C145513D41469305F00F2685C8
:102B280097E0FA1FE7804099054963152503484453
:102B38006244F240D2444249B249C1450561B5B543
:102B4800414681454A8597E0FA1FE780E096E315FC
:102B580035FDC1B741468145268597E0FA1FE780D4
:102B6800A095E30625FDF2406244D2444249B249A9
:102B780005618280411122C43734002026C24AC030
:102B8800AE842A891306000281451305448306C6CC
:102B980097E0FA1FE780408093074483A3812701C9
:102BA800B7370020238E9796EFB0D073854719C1A9
:102BB80081474945230AF482B2402244924402499B
:102BC80041018280814791C909C985476319F50088
:102BD800DC3193E707FCDCB185473E858280894775
:102BE8006316F500DC3193F7F703F5B70D47854712
:102BF800E315E5FED8311377F70313670704D8B157
:102C0800E9BF814785C119CDD8319306000C8547A6
:102C18001377070C6308D700930600048D476303F6
:102C2800D70089473E858280411122C4005D06C6CF
:102C380026C21DC8AA84085009C597D0FA1FE78084
:102C4800E04C485009C597D0FA1FE780204C08543B
:102C580009C597D0FA1FE780604B228597D0FA1FE5
:102C6800E780C04A23AC0402B240224492444101A6
:102C7800828019E9B737002083C7678391C7372552
:102C88000020130505518280373500201305C584BF
:102C98008280B737002003C567838280B73700205A
:102CA80003A507848280B737002003A54784828064
:102CB800B737002083A7878488438280B7370020EE
:102CC80093874783D44B9842050798C2A833930744
:102CD800F00F6305F50091656FD0BFE482800111A4
:102CE80022CC06CE2E8432C6EF8020199147B245F9
:102CF8006310F502B727002083A7C75295C303A323
:102D08000700630F030022856244F24005610283D5
:102D1800B727002083A7475281C703A34700D5B729
:102D2800F2406244054505618280011122CC2A8463
:102D38004A2106CE26CA4AC84EC697E0FA1FE7803F
:102D480020D52DC52A8904218349C500F13D4A852E
:102D5800EF80E0504A20EF80800D372900201309CA
:102D6800895383470900B9C763969704B72700209A
:102D780083C5975326858D3419E1230009004A201D
:102D8800EF80A00F9147631CF500B73700209387A9
:102D980047835620FA236394E6007D57FAA3F2404E
:102DA8006244D2444249B249056182808149930410
:102DB800F00F65B79307F00FE383F4FC74205220FB
:102DC80028204E87A68541365DBF79715EC6AA8BDD
:102DD8002E8552CC56CA5AC806D622D426D24AD0F4
:102DE8004ECEAE8A328B368A97E0FA1FE78040CA09
:102DF8007DC1045D2A89E5C09C50614599C31305CE
:102E080040039C5481C751054205418163050A006E
:102E1800710542054181DC5081C75D05420541814C
:102E280097D0FA1FE780E0402A8455C5614681455E
:102E380097D0FA1FE7804056B737002083C94788E4
:102E48006394090083490900930700FD1CA0A94762
:102E5800A30074013CA0230364018C502312540185
:102E68001305840191C908C47146930A440397D095
:102E7800FA1FE780C04B56858C5491C948C4514607
:102E8800930A450197D0FA1FE780604A5685630C7C
:102E98000A0008C87146D285930AC50197D0FA1F5F
:102EA800E780E0485685CC5099C548C85D4697D01C
:102EB800FA1FE780C047A2854E85EFD07F92225443
:102EC800B2509254F249624AD24A424BB24B4A85B6
:102ED8000259456191BBB250225492540259F249A9
:102EE800624AD24A424BB24B4561828001114EC6BA
:102EF800AA892E854AC806CE22CC26CA2E8997E0F2
:102F0800FA1FE780E0B839C5B737002083C447887F
:102F180091E00421194597D0FA1FE78080312A846F
:102F280015C98145194697D0FA1FE780E0469307EF
:102F380000FD1CA0B947A30034013CA023122401C2
:102F4800A2856244F2404249B2492685D2440561CD
:102F58006FD01F89F2406244D2444249B2490561A8
:102F6800828039715ECEAA8B2E8526DA4ED652D44F
:102F780056D25AD006DE22DC4AD8AE84328BB68AC4
:102F88003A8ABE8942C697E0FA1FE78060B039C91D
:102F98002A89414597D0FA1FE780A0292A8439C198
:102FA8004146814597D0FA1FE780003FB737002098
:102FB80003C5478819E103450900930700FD1CA0D4
:102FC800BD473CA0B247A300740146A02304640196
:102FD800A304540123054401A30534015CC4A2855C
:102FE800EFD01F80F2506254D2544259B259225A3B
:102FF800925A025BF24B21618280797126D2AA84AF
:1030080039454AD04ECE06D622D42EC6B289368944
:1030180097D0FA1FE780E0210DCDB2459307000D48
:103028001EA1B1472A844EA13CA1CE851905194697
:1030380097D0FA1FE780A02F23062401A2852254E7
:10304800B2500259F24913F5F40F925445616FD00A
:103058002FF9B250225492540259F24945618280A4
:10306800411126C2B734002093844483B83006C681
:1030780022C44AC09307F00F6308F7042A89394528
:1030880097D0FA1FE780E01A2A841DCD930700FD28
:10309800B73500201CA1A300250123010500938555
:1030A800C5840D05194697D0FA1FE78040289E244D
:1030B800A285A8303EA49C305CA42244B24092442D
:1030C800024941016FD0CFF1B240224492440249F3
:1030D8004101828001115AC02A8B314526CA4EC649
:1030E80052C456C206CE22CC4AC8AE84B28A368AA8
:1030F800BA8997D0FA1FE780C0132DCD2A84268578
:1031080097E0FA1FE780C09809C55825A1476311C1
:10311800F704B737002003C97783930700FD1CA085
:103128009D47A30064013CA046A023135401231427
:10313800440123153401A2856244F240D244B249C5
:10314800224A924A024B4A85424905616FD04FE9AB
:10315800B737002003C9D797E3110BFCB727002026
:1031680083A7075E9C47D5DBCE865286D685268503
:10317800829765B7F2406244D2444249B249224A32
:10318800924A024B05618280011122CC2A84214592
:1031980006CE2EC697D0FA1FE780A00915C5B245FE
:1031A800930700FD1CA1C5473CA1BC313CB1DE2101
:1031B8005EA1FC217CA1FC31AA857CB122856244F8
:1031C800F24005616FD0CFE1F24062440561828030
:1031D80001114AC82A89614526CA4EC606CE22CCA4
:1031E800AE89B28497D0FA1FE780A00425C193075F
:1031F80000FD1CA1BC302A84938584001CB195472E
:103208003CA1FC3011051946A30FF5FE97D0FA1F13
:10321800E780E011DE2023063401A2853EA4BE2CFF
:103228004A857EA4DE2C1EA8FE2C3EA883C7040275
:103238005CA883C714025CB8BE30F240D2447EA8B2
:1032480062444249B24905616FD08FD9F240624465
:10325800D2444249B24905618280411122C43734BF
:103268000020130444833C2006C626C285CBB7241D
:103278000020AA8519461385045197D0FA1FE780C4
:10328800000B282093850451EFF0DF932244B240CD
:1032980013850451924441016FB09005B240224415
:1032A8009244014541018280411126C2B734002071
:1032B8009387448306C622C44AC0B8339307F00FE5
:1032C800938444836301F7042A89294597D0FA1F18
:1032D800E78020F62A8405C9930700FD1CA1A147B1
:1032E800A30025013CA1BC20B725002093850551EA
:1032F8003CB11946110597D0FA1FE7804003A83062
:10330800A285EFD0EFCDB8208D476311F702B7271C
:10331800002083A7875299CB03A387006308030083
:103328002244B2409244024941010283B2402244FD
:103338009244024941018280797122D406D626D26C
:103348004AD04ECE52CC56CA09444DCD2A890A21BC
:10335800AE89514497D0FA1FE7808073AA845DC173
:103368003737002093078797DC238546BA8AFD17ED
:1033780093F7F70F494463F7F6085825A1476314F4
:10338800F700639109089C5C4544ADEF916593850E
:1033980045711305C00297D0FA1FE78020CA88DC60
:1033A8002A8A4D4425C11306C002814597D0FA1FC9
:1033B800E78080FE8357090093064A00368523116B
:1033C800FA0071469305490036C697D0FA1FE78080
:1033D80000F689472300FA00C824B24603560900BC
:1033E80083C58A97611513351500EF8070212A84EB
:1033F80063860900CE852685EF80401401C42685A2
:10340800EFF09F822285B250225492540259F24919
:10341800624AD24A45618280B737002083C7C7977E
:103428000547FD1793F7F70F6377F708894749C6EC
:10343800011122CC26CA4AC84EC652C406CEAA8951
:10344800368AB2842E8997D0FA1FE78060642A846E
:10345800D14731C5485509C597D0FA1FE78000CB39
:10346800F145268597D0FA1FE780A0F848D4CD47C4
:103478001DC5542421478147639DE600630B0A005C
:10348800382D122993062501AA854E85EF806011F3
:10349800AA875820630E09001367670058A0F240F6
:1034A8006244D2444249B249224A3E85056182803B
:1034B80013674700E5B7C9473E8582809307100424
:1034C80063EAA700B73700209387478506053E952E
:1034D8000A21828041657D158280011122CC2A84CF
:1034E8002E8526CA06CEAE8497D0FA1FE780405AAA
:1034F8000DCDB7470F009387F723094563E287028D
:1035080081450A85414697D0FA1FE780E0E8A685FD
:1035180060800A8541804081A3010100EF80E07A44
:10352800F2406244D244056182804945D5BFB7372D
:103538000020238DA79682806F80F006797152CC87
:103548002A8A328522D426D24AD04ECE56CA5AC8A2
:103558005EC606D662C4AE8BB28A368BBA843E8902
:10356800C289468497D0FA1FE78080520DC92A8CF9
:1035780063130A0213774B005C2115CF93E72701E9
:103588002302FC008DEC631C0902639A090205E81A
:10359800ED9B2302FC00832B8C0363910B08B25034
:1035A800225492540259F249624AD24A424BB24BCF
:1035B800224C45618280F59B93E70701D1B793E7D9
:1035C80047002302FC0001CC1C484146A285232465
:1035D800FC0213058C0197D0FA1FE78040D563934E
:1035E8000B02D5D80325CC0209C597D0FA1FE7806E
:1035F800E0B1F145268597D0FA1FE78080DF2326C2
:10360800AC0251BFE30909F80325CC0209C597D0DC
:10361800FA1FE780A0AFF1454A85F1BF9DC483A793
:103628000B0299EB916593853571714597D0FA1F17
:10363800E780C0A023A0AB0203A50B0219C5714601
:10364800A68597D0FA1FE78080CE6388090283A7F2
:103658004B0299EB9165938525715D4597D0FA1FCB
:10366800E780C09D23A2AB0203A54B0219C55D46A6
:10367800CE8597D0FA1FE78080CB1DC483A78B0225
:1036880099EB916593851571514597D0FA1FE7809D
:10369800E09A23A4AB0203A58B0219C55146A28563
:1036A80097D0FA1FE780A0C82254B2509254F2492A
:1036B800B24B224CCA865A860259424BD68552854D
:1036C800D24A624A45616FF04FF0011126CA52C4CE
:1036D80006CE22CC4AC84EC62A8AAE8497D0FA1F94
:1036E800E780003B35C1AA89394597D0FA1FE780A2
:1036F80040B42A8431C9B737002003C94788631406
:10370800090003C909009307000D1EA0AD473CA09E
:103718009385690013053400194697D0FA1FE7808E
:1037280000C193F71400858085885CA444B42315F0
:103738004401A2856244F240D244B249224A4A85F1
:10374800424905616FD0CF89F2406244D244424970
:10375800B249224A0561828001114EC652C456C23E
:1037680006CE22CC26CA4AC8AA8A2E8AB28997D0FF
:10377800FA1FE780E0312DCD2A891305C00297D0C2
:10378800FA1FE78000AB2A8425C5B737002083C419
:10379800478899E0834409009307000D1EA0E94774
:1037A8003CA09305690013053400194697D0FA1F09
:1037B800E780E0B7D285231554011305C4004146BC
:1037C80097D0FA1FE780A0B6CE851305C4014146FD
:1037D80097D0FA1FE780A0B5A2856244F24042491B
:1037E800B249224A924A2685D24405616FC05FFFDA
:1037F800F2406244D2444249B249224A924A05619F
:103808008280411122C437240020130484510840C7
:1038180006C619C597D0FA1FE780408F23200400F9
:10382800B240224441018280011106CE22CC26CA30
:103838004AC82EC697D0FA1FE780802531CDB245F9
:10384800B737002003C947880CD5AA846314090038
:1038580003490500414597D0FA1FE780809D2A84D7
:1038680005CD9307000D1EA1A5473CA1DC3093852B
:1038780064001105A30FF5FE194697D0FA1FE780DB
:1038880000AB9C54A285F2405CC46244D2444A8591
:10389800424905616FC0DFF4F2406244D2444249B4
:1038A800056182801D71A2CC86CE2A842EC697D04F
:1038B800FA1FE780E01D15C954251147AA87494515
:1038C8006391E6029C5FB24591C3EC2BB7D6050025
:1038D8002308B1009386C6C9100889452285EF7070
:1038E800103DF6406644256182805145DDBFB737FB
:1038F800002083C7C7970547FD1793F7F70F637A2B
:10390800F704894721CA411122C426C24AC006C603
:10391800B2842E8997D0FA1FE78080172A84D1476E
:1039280015C1630609005C2193E727005CA14146A5
:10393800A6851305840197D0FA1FE780409F9C480D
:103948001CD48147B2402244924402493E85410139
:103958008280C9473E858280797122D406D62A841E
:103968002EC697D0FA1FE780A01201CDB245228556
:10397800230EB1006C08EF701039B2502254456123
:1039880082805145DDBF6F702044C1671387E7FF10
:103998006395E502B727002083A7475291EB494575
:1039A80082804945B24022449244024941018280C2
:1039B80003A30700E30503FE0283411122C426C2C4
:1039C8004AC006C6FD172A892E84B284639AF50276
:1039D800B727002083A7475291CF9C4381CF829776
:1039E80011E9B7270020238C2753B7270020A38C81
:1039F80097524DBFA6854A85EFE01FDE45F5D5B73E
:103A08002E8597D0FA1FE780A00841DD1C210D45BF
:103A1800E39A27F922852244B2400249A6859244B6
:103A280041016FB0E0099307100463E1A706411153
:103A3800C16722C406C626C2FD172A8409456381C8
:103A4800F502C547AE846312F4022E85EFB0800EEE
:103A5800373500201305458506042A9406A001453C
:103A6800B24022449244410182809307A003631626
:103A7800F4002E85EFB08005E1BF9307B003E3198A
:103A8800F4FC13F5F50FEFB0A004D9B7094582800F
:103A9800011106CE2AC6EFE03FD6EF10401BEF908B
:103AA800E16FB737002093874783130700F0BAA365
:103AB80023820700B7370020324513878797FD56C2
:103AC80034A3F240238CA796954505616F50305674
:103AD80075719397050126C306C722C54AC1CEDE74
:103AE800D2DCD6DADAD8DED6E2D4E6D2EAD0EECE26
:103AF800C187AE8463D007563734002003458497C6
:103B080037390020372A002097C0FA1FE780C0778E
:103B1800AA8C22CCB72A0020372B0020372D002072
:103B280013044983372C002063930C022165258DEB
:103B3800BA402A449A440A49F659665AD65A465B04
:103B4800B65B265C965C065DF64D4961828083C74C
:103B58000C001307200A639CE7008349340003D54F
:103B68002C00C1656686FD15EFF06F9785A2624748
:103B78001307879783492700130710096394E716EB
:103B880083C71C0015476391E7026685EFF0EF993C
:103B98006685EFC01FC0E24703C5879797C0FA1F25
:103BA800E780806EAA8C49B739476395E71603D535
:103BB8004C008567A5076316F50483A58C0083CBA5
:103BC8000500639D0B00850591C93735002019460E
:103BD8001305C58497C0FA1FE780607503474983BA
:103BE80085476311F71063880B00230A09825E85F5
:103BF800EFF00FC771BF8947230AF982EFA0106F52
:103C080041BF8967138727006318E50483AB8C00DD
:103C1800638A0B0C83C70B0099EB83C72B0003C780
:103C28001B00A207D98F1EA483C73B001CB0034703
:103C3800498389476318F70A83C70B0091C7230A8A
:103C4800098203C50B006DB70C300A248D47230A7F
:103C5800F982EF509040F5B795076318F50083A7F0
:103C68008C008823EFF04FE425B7F9771387A7FF77
:103C78002A9742074183914663F1E6049387A7FC9C
:103C8800AA97C207C18371476371F70289671387CF
:103C9800B7006310E50483A70A52E38B07EE9C4341
:103CA800E685E38707EE829715A037070018130704
:103CB800F770B357F700858BA1CB83278A52E38926
:103CC80007EC9C43E38607EC66858297E31205ECD4
:103CD80011A81387C7006310E50283A78C009C23F3
:103CE800E38807EA9307F00FE384F9EAE6854E854F
:103CF800EFC01FAF4DB5B9076318F50083274C52C5
:103D0800E38807E8DC4369BF896793871704E304FE
:103D1800F5F8C9BF3D476398E70403D54C008967A8
:103D28001387D700E30CE5FC13879701E308E5FC4C
:103D3800CD07E319F5FA7A20C167FD17631DF7006F
:103D480083274C52E38607E4DC43E38307E40965F1
:103D5800E6854D0589BFB727002083A7C752E389A9
:103D680007E29C43DDB71307E003E39DE7F683C74B
:103D78002C000547639EE71283C76C003727002095
:103D8800930D87516398071083A70D00638107106F
:103D980083CB0700A14903C57C0013878C00BA8533
:103DA8003ACEEFE01FE6A383AC001306400281453C
:103DB800681097C0FA1FE780205E83C73C007247EF
:103DC8001946A307F10283C77C00BA854818A309DE
:103DD800F10297C0FA1FE780805583D74C00701016
:103DE800CE852318F10283D7EC005E852313F104F6
:103DF80083D70C012314F10483D72C012315F10474
:103E080083C74C012306F104FD57A306F104FD57AF
:103E18002317F104EFF0CFBB83C73C0072478DE74F
:103E2800DD4783D80C0103D8EC0083C67C0083D51A
:103E38004C003EC283D72C013EC00546CE875E8526
:103E4800EF70801AA381AC0083A70D0081C71145CC
:103E5800EFF03F9B03458B53930B8B53E30A05D23B
:103E680083459D53EFE05F97E30405D283C63C008A
:103E780093071003638AF60003D64C0083C50B0032
:103E88004E873685EFE03FAC23800B0011B3834BA0
:103E9800340009B783278A52834B34009149E38C55
:103EA80007EEDC43E38907EE814501458297E5B5D6
:103EB800130790026397E70883C76C003727002031
:103EC800930D8751B9EB83A70D00A9C783CB0700D2
:103ED800A14903C57C0093772500A1CF05891387E5
:103EE8004C01A383AC006686CE855E853ACEEFF0A2
:103EF8002FAE83C73C007247A1FBDD4783D8CC01B6
:103F080003D8AC0183C67C0083D54C003EC283D75E
:103F1800EC011DB7834B340065BF83278A52834B5E
:103F280034009149DDD7DC43CDD7814501458297DF
:103F38004DB713878C00BA853ACEEFE09FCC724715
:103F48004DB70947639CE70083A70A52E38207C479
:103F5800DC43E38F07C2668582971DB92D476398B6
:103F6800E70083A70A52E38507C29C47DDB70D47E0
:103F78006397E70066868D4503D54C00F5B619476B
:103F88006395E7069305A10213051031EF90E12828
:103F98006C1013052031EF90412803D66C0083572D
:103FA800C10203D54C0063E8C70083D68C000357D1
:103FB800A10263F7E60093050002EFA0B036C9BE80
:103FC8006374E6002393EC0063F4D7002394FC00A9
:103FD80003D7CC0083D6AC0003D68C0083D56C0005
:103FE80001488147EFA0D03365B61D47E38CE7CE83
:103FF80031476395E7006686B145BDBF354763988D
:10400800E70083A70A52E38507B8DC4799B7494711
:10401800639DE70083278A52E38607CCDC43E3836A
:1040280007CC81450545829775B94D47639CE700E4
:1040380083278A52E38807CADC43E38507CAE685F3
:104048000945D5B713076002E39EE7C8668693055E
:1040580060021DB793F7150089CFB727002083A703
:10406800075289C7DC4399C30145829713C51400D9
:10407800C1B493F7250091CFB727002083A78752B3
:1040880091C7DC4381C781450545829713C5240044
:1040980045B493F745000145E38C07A8B7270020EE
:1040A80083A7C751373400201304448389CF854739
:1040B8005CA0B727002083A7875291C7DC4381C73C
:1040C80081450545829748446C10EF70B02C681004
:1040D800EFF0AF98B737002083D7678781CF1306F3
:1040E80000643386C702B737002003C58797914518
:1040F800EFC01FC113C5440025BC411122C4372499
:1041080000200325C45106C619C597C0FA1FE780C9
:10411800E0FF232E0450B240224441018280757191
:1041280022C5372400208327C45106C726C34AC1A5
:10413800CEDED2DCD6DADAD8DED6E2D4054563891B
:10414800070E9305F1051305F041EF70F101930592
:10415800F1051305F041EF703101B737002093875F
:104168004783BC230347F105B337F00011C3890720
:104178000327C451BEC6283393054700EFE09FA428
:104188000327C451AAC40D452C23AEC2EFF00FB3C8
:10419800AAC01145EFF08FB20324C4512ADE654549
:1041A8003824034CB4003ADCEFF04FB1AA846945D7
:1041B800EFF0CFB02A897145EFF04FB0AA896D456D
:1041C800EFF0CFAF2A8A7545EFF04FAFAA8A79454D
:1041D800EFF0CFAE2A8B13050004EFF02FAEAA8BB9
:1041E80013051004EFF08FADE2042648B647625776
:1041F800F256064696451375F50F93FBFB0F137B96
:10420800FB0F93FAFA0F137AFA0F93F9F90F137950
:10421800F90FE1842AD05ECE5ACC56CA52C84EC68F
:104228004AC426C262C0930844000545EFA0501155
:10423800BA402A449A440A49F659665AD65A465BFD
:10424800B65B265C49618280011122CC06CE26CA63
:104258008D472E84631AF504B831B7340020E94736
:10426800CA21938444836315F700FE206389A70459
:1042780097D0FA1FE780C08119C17E207EA53A2415
:10428800162472204E202830EFE0DFE45A20FE206A
:104298006309F7008547F2406244D2443E850561D0
:1042A8008280FD57FEA0FDB78967CD07631CF50026
:1042B800BC2131476385E7004547E39DE7FCEFE014
:1042C800EFF3C9BFB1476319F500B737002003C53D
:1042D800D797EFE07FEB7DBF41677D178147E31CF0
:1042E800E5FAD4314947E398E6FACC212A20300090
:1042F80023140100EF60700771BF411122C43724F5
:1043080000208347A45326C206C64AC01307E00FFD
:10431800AE846382E7041307F00F1304A453638485
:10432800E702114597C0FA1FE780A0F009CD93076F
:1043380000FD1CA189473CA1854704B13CB1AA8571
:104348000820EFC0EFC9F9571CA0B240224492449C
:104358000249410182802A89114597C0FA1FE780E6
:1043680040ED65D5930700FD1CA189473CA104B128
:10437800A30125012244B7270020B24092440249F4
:10438800AA8503C5B75341016FC08FC579714AD05B
:10439800372900208327C95122D406D626D24ECEEB
:1043A80052CC56CA4544C5EBB7340020938784974E
:1043B800DC234944958BC5C3B72700202E8A916515
:1043C800A38DA752AA8993857571314597C0FA1FA5
:1043D800E780C0C6232EA9504D4435CD23003501B2
:1043E800A30005002946D285090597C0FA1FE78072
:1043F80000F48327C9519146B82363E9E60835E7F5
:104408004D47B8A3B82313670701B8A393057100F4
:104418001305F041EF7041559C83F1E7B737002051
:1044280003C767838D476310F70CEFE03F872C00C5
:10443800EF7040762800EFE05FE24545EFF00F8827
:10444800014411C9130600643306C50203C58497E5
:104458009145EFC0FF8A2285B250225492540259E6
:10446800F249624AD24A4561828085466314D70080
:10447800754741BF89466314D700494759B78D46E8
:104488006314D7004147B5BF5547A5BF9546CA8AAB
:10449800630DD70099466315D7000947B8A331A023
:1044A8001D466312C702238107006545EFF00F819F
:1044B8009307F007E30CF5F403A7CA513C2393E7ED
:1044C80007043CA3A1B721466314C7000547F9B701
:1044D80025466314C700B4A3C9BFA9460544E31C15
:1044E800D7F6114765BF25392A8435D53931A5B79F
:1044F800011126CAB724002083A7C45122CC06CEB6
:104508004AC84944B9C39C230D446390A70437396A
:104518000020034589978945EFC09FA603458997E1
:10452800B72700209145239E0752EFC07FA583A798
:10453800C4510147814680B31306F100854785457C
:104548000145DC87EFA0A0642A842285F2406244FA
:10455800D244424905618280011106CE22CC26CA86
:104568004AC88547631AF506372400201304C45344
:104578001E20B9C7373700200347878331E3130765
:10458800B003636BF702B734002003C584978945ED
:10459800EFC01F9F12209307006403C5849733065A
:1045A800F6028945EFC0CFF523100400F2406244BB
:1045B800D244424905618280938747FC1EA0FDB71B
:1045C800B727002083A7C751F5D36244F240D244ED
:1045D80042498823056129BFB724002083A7C45115
:1045E800F1D7373700201309879783474900918B04
:1045F800D5DF89476310F5062D452EC697C0FA1FEB
:10460800E78020C32A845DD1B245930700FD1CA131
:10461800E547A30005003CA1BC3115051946230F49
:10462800F5FEDC219505A30FF5FE97C0FA1FE7807C
:1046380000D0034559009307F00F6315F50083A7D1
:10464800C4518823A2856244F240D244424905619C
:104658006FC00F99034587978945EFC07F926244E1
:10466800F240D2444249B7270020239E07520561F1
:104678006FF0BFA849458280B737002083C7C79726
:10468800958B638C07129307C01C63FCC700094510
:104698008280F2406244D2444249B24909450561E8
:1046A8008280B727002083A7C75163880710B727E0
:1046B80000209387A75303C807001307E00F631E62
:1046C800E80E011122CC4AC806CE26CA4EC688A3D7
:1046D800130586004205368932844181A5C9916552
:1046E8009385657197C0FA1FE7804095AA8955D1CF
:1046F800B724002003A544549384445409C597C0A3
:10470800FA1FE780A0A01385890023A0A9002286AC
:10471800814523A0340197C0FA1FE780E0C79C4079
:104728002286CA85884397C0FA1FE78040C09C400C
:10473800A286F240C2A36244D2444249B249984395
:1047480005468D45054505616FA0E0439165938554
:10475800557197C0FA1FE780608EAA891DD9B724C2
:10476800002003A5C4549384C45409C597C0FA1FF4
:10477800E780C0991385890023A0A9002286814576
:1047880023A0340197C0FA1FE78000C19C4022860D
:10479800CA85884397C0FA1FE78060B99C40A28603
:1047A800F240C2A36244D2444249B2499843054602
:1047B8008D45054505616FA0403D494582809307B9
:1047C800C01C63FCA700094582800945F240624489
:1047D800D2444249B2490561828055C9011122CCAF
:1047E8002A8421054EC64205AE8991659385657177
:1047F80041814AC806CE26CA97C0FA1FE7800084BE
:104808002A8961D5B724002003A5445493844454CD
:1048180009C597C0FA1FE780608F13058900232018
:10482800A9002286814523A0240197C0FA1FE780AA
:10483800A0B69C402286CE85884397C0FA1FE780A1
:1048480000AF9C40C2A3B727002083A7C75185CFDC
:10485800B737002083C7C797958B85CBB72700202C
:1048680083A7475491CF9843D6236244F240D24459
:104878004249B24905468D45054505616FA0A030FE
:1048880001478146DDB7014591B7494581B7B7274B
:10489800002083A7C7518DC7B737002083C7C797A4
:1048A800958B8DC3B727002083A7475499C7984392
:1048B800D62305468D450545D1B701478146D5BF65
:1048C80001458280494582809307C01C63FCA7008C
:1048D800094582800945F2406244D2444249B249BE
:1048E8000561828055C9011122CC2A8421054EC652
:1048F8004205AE8991659385557141814AC806CEB6
:1049080026CA97B0FA1FE78060732A8961D5B72451
:10491800002003A5C4549384C45409C597B0FA1F52
:10492800E780C07E130589002320A90022868145DF
:1049380023A0240197C0FA1FE78000A69C40228686
:10494800CE85884397C0FA1FE780609E9C40C2A32B
:10495800B727002083A7C75185CFB737002083C763
:10496800C797958B85CBB727002083A7C75491CFCE
:104978009843D6236244F240D2444249B24905469C
:104988008D45054505616FA0402001478146DDB78B
:10499800014591B7494581B7B727002083A7C7517B
:1049A8008DC7B737002083C7C797958B8DC3B727A7
:1049B800002083A7C75499C79843D62305468D4539
:1049C8000545D1B701478146D5BF01458280494594
:1049D80082809307C01C63F4A7000945828079711F
:1049E80022D44ECE06D626D24AD0AE892A8425C1F4
:1049F80021059165420593857571418197B0FA1F2C
:104A0800E780C0632A89094563040908B7240020A0
:104A180003A584549384845409C597B0FA1FE7808A
:104A2800E06E130589002320A9002286814523A072
:104A3800240197C0FA1FE78020969C402286CE85E5
:104A4800884397C0FA1FE780808E9C40C2A3B7278F
:104A5800002083A7C751014585CFB737002083C7FA
:104A6800C7974945958B8DC76C001305D030EF80EB
:104A7800C17AB247014593F7070F99CBB7270020B2
:104A880083A787548D4505459443D223EFA0601032
:104A9800B250225492540259F24945618280B72794
:104AA800002083A7475489CFD2238C43411106C6DF
:104AB80097C0FA1FE780A087B24001454101828074
:104AC80009458280B727002083A7475485C7B727A1
:104AD800002003A7C754894719CF52230C4341111B
:104AE80006C697C0FA1FE7808084B24081473E859A
:104AF8004101828089473E858280797106D622D419
:104B080026D24AD04ECE52CC8D4763FCA7008944AA
:104B1800B2502254268502599254F249624A45619C
:104B280082803739002003474983C144E312F7FEE6
:104B38009307F5FF9309498393F7F70F8546AE84EA
:104B48002A8403CA29001309498363EAF6068DE11A
:104B580099452800EFD07FE5B739002003C589972C
:104B6800914523018900EFC0AFC135E481444DB7B9
:104B780019468145280097C0FA1FE780E081194649
:104B88002C00268597C0FA1FE780608B49F11946EB
:104B98009305F00F280097B0FA1FE780E07F1946C9
:104BA8002C00268597C0FA1FE78060892DF11946E9
:104BB800A685280097B0FA1FE780607771BFE31DCC
:104BC800E5F803A5C9002C00EF60D07CAA8449D57C
:104BD8002381490135BF2800EFE02FE8AA8405EDBD
:104BE800930571001305F041EF6011588483BDFCF3
:104BF8008D47E31DF4F64545EFE05F8C25D9B7777F
:104C08001800938707A03306F50203C589979145D5
:104C1800EFC0AFAFF5BD23014901DDBDB7370020B7
:104C280083C7C797918B8DC3372500204111130582
:104C3800055406C6EFD0DFD6B240B73700207D57FF
:104C4800239DE7824101828001456FD07FD5B72738
:104C580000207D57A38DE752B72700207957238D71
:104C6800E752B7370020238D078CB7270020239EF3
:104C78000752B727002023A20754B727002023A6EE
:104C88000754B727002023A4075437570500B72730
:104C980000209387875E1307E7E598C33747050029
:104CA80013070756D8C3374705001307671298C775
:104CB800B747050037270020938707252320F75497
:104CC8008280411126C2B724002083A7C45106C69A
:104CD80022C49DCB2A840D4597B0FA1FE780605502
:104CE800AA8501CD930700FD1CA18D4700B13CA109
:104CF80083A7C4518823EFB0BFAE19C42244B24081
:104D0800924441016FF06FBFB24022449244410186
:104D18008280797152CC372A00208327CA514AD021
:104D280006D622D426D24ECE56CA0149A1C703C9F7
:104D38001700B73400208547AA8993844483630504
:104D4800F904DC2005499DE70D4597B0FA1FE78077
:104D5800404EAA8509CD930700FD1CA19147A300E9
:104D680035013CA18327CA518823EFB07FA7EFF014
:104D7800CFB80549B25022544A8592540259F24993
:104D8800624AD24A45618280B727002083A74754E8
:104D9800D28A85E30145EFE06FF22A8601CAB73768
:104DA800002003C587978945EFB09FF583A7CA51AF
:104DB800B1A09443D2239305E1000545EFD0FFC885
:104DC80071D91C21858BF9D70545EFE02FEF9307A3
:104DD800B0032A8463FEA702B737002003C587976C
:104DE8005D66130606708945EFC02F92B72700202D
:104DF800130444FC239E87528327CA51094798B35A
:104E0800DC2081C723820400B5B74E855D3D9DB780
:104E1800130600643306C50251B7411122C42A841F
:104E28000D4506C697B0FA1FE780A0400DC193074D
:104E380000FD1CA1CD473CA100B12244B7270020AA
:104E4800B240AA8503C5B75341016FB07F99B240FC
:104E580022444101828056210111896706CE22CC65
:104E680026CA138667002A876398C6001C4701452F
:104E78008C23EFF08FC81DA8138687006396C600A1
:104E88001C4705458C23F5B7138697006392C60225
:104E9800B727002083A7C751014595C318470823A2
:104EA80071E5054798B30545EF90D044054501A83D
:104EB8001386A700639AC6001C478823993DF240D1
:104EC8006244D2440561828013866703E380C6FA90
:104ED80013867703E386C6FA13868703639AC608A0
:104EE8001C45372400201307E00F84238347A4536D
:104EF8001304A453638BE7021307F00F6384E702DC
:104F0800114597B0FA1FE780C032AA8501CD9307F3
:104F180000FD1CA1894704B13CA1A301050008209C
:104F2800EFB01F8CF9571CA051B7B727002003A773
:104F3800C7513E84014541D78DE885447D45448568
:104F4800EFE0CFD7688613050002EFE02FD783275D
:104F5800C451C8851307B10084B374001306A100B7
:104F680085450545EF90B04291B72685993B3DBFF1
:104F780013869703E382C6F41386E7036396C60095
:104F88001C4509458C23F5B59387F7030145E3983C
:104F9800F6F21C4788231DE56C001305D030EF801E
:104FA800C127B247414793F7070FE381E7F093051D
:104FB800B10013056031EF80412688858545EF9063
:104FC800903DEDB5993DDDB5B737002083C7C7974C
:104FD800411106C6958B99CB372500201305855EB0
:104FE800EFD07F9B4D45B240410182800145EFD013
:104FF8009F9A0145CDBF9821937625009377D70FC7
:1050080099C293672700131885011358884113F72D
:10501800F7076354080013E707089376850093772A
:10502800770F99C2936787001377050293F6F70DF8
:1050380019C393E6070294A1634508009377A50274
:1050480091C71C2293E7C7001CA282807DFD1C2209
:10505800CD9BDDBF2D45631B0710882109476313CE
:10506800E51001114EC6BE89DC4122CC26CA4AC8C9
:1050780006CE98339C23B68422075D8F42078D663F
:105088004187938736A032842E89630BF70A63C061
:10509800E702938716A06307F70863CAE70A9386AF
:1050A80006A0630BD70423900400054559A09387F5
:1050B80066AA630EF708938786B86301F70A938692
:1050C80046A0E312D7FEDC45C1C321479AA09A2324
:1050D80018A29A23218318B2BA2338A2BA232183AB
:1050E80038B2DA2358A2DA23218358B2FA2378A2F5
:1050F800FE23A1837CB22DA8C84597B0FA1FE7808C
:10510800802C420541814E86637335012A8692A020
:10511800420641828325C900228597B0FA1FE7809D
:10512800002139A0DC459E238AA01CA2A1831CB2C1
:105138000145F2406244D2444249B2490561828045
:1051480099479EA01946F9B723900400D5B785471B
:105158009EA08327C9009C231CA0D9BFE1479EA01D
:1051680061464DBF2390060005458280828083C832
:1051780005008947639BF816DC41797122D406D66D
:1051880026D24AD04ECE52CC56CA03C817009C230A
:105198002E8422083368F80042088D6713580841A6
:1051A800138327A0630F68102A8A3A89B684B285C8
:1051B800634C0301138707A0630BE802938717A0CA
:1051C8006301F80A854711A8138737A06300E80C24
:1051D800138767AA8D47E317E8FEB250225492540A
:1051E8000259F249624AD24A3E8545618280484462
:1051F80032C697B0FA1FE780001D420541819D47DE
:10520800E36D25FDB72A0020938A3A5583C70A0023
:10521800B3099900B24563D43701B5477DBF484407
:105228002686C2094A9597B0FA1FE780401003C640
:105238000A00484493D909010506330636418145D9
:105248004E9597B0FA1FE7802015B727002083A74F
:10525800875599E3814751B79C438145E5DF5285DE
:1052680025A0AD47E31B09F6E39916FB1C3214226F
:105278005844A207D58F1EA3B727002083A78755B8
:10528800F1DB9C43E1DB85458297E9B7B72700202E
:1052980003C7C7558D4731D3AD47E31009F4994784
:1052A800E39DF6F64844194697B0FA1FE7802008B0
:1052B800B727002083A78755D1DF9C43C1DF8D45E1
:1052C80079BFB727002083C5474E8D47A18991D55F
:1052D800AD4701F78547E392F6F4182293070008D3
:1052E800E3EDE6EE5C4498A3B5B785473E8582803A
:1052F800B7270020411123AC0754B727002022C448
:10530800238B07540944B7270020A38B874CB72762
:105318000020A3890754B7270020238A874CB72782
:10532800002023980754B72700202382874E37256B
:105338000020B72700202147238E07541946B72796
:10534800002081451305055606C6A382E74E97B08F
:10535800FA1FE7806004B7270020238D874C3707A2
:10536800A000B72700209387C74D1307070598C3E8
:105378003707E803D8C3B7270020238B874C054796
:10538800B7270020A38AE74CB72700202383874E3E
:1053980037250020B7270020238307566146B72703
:1053A800002081451305855F238C874C97B0FA1F31
:1053B800E78080FEB7270020A38C874CB727002002
:1053C800A38A075437570500B727002093878747D4
:1053D8001307C70598C3B24022443757050013077F
:1053E8006717D8C323A40700410182809547630249
:1053F800F51A797122D426D206D64AD04ECE52CC8E
:10540800B2842E8463E4A7048947630DF51463EF1F
:10541800A7004DC50547630FE5120945B250225450
:1054280092540259F249624A456182808D47630469
:10543800F5149147E313F5FEA1476395F508372561
:1054480000202146A6851305C54D3DAA93072004D3
:105458006305F51663E1A7029D476306F514A147A6
:10546800E31DF5FA8547639FF5041822B727002046
:10547800A38AE754F1A8930710086309F514930762
:105488002008630DF51493070008E318F5F885471D
:10549800639AF502B727002083C747551387F7FF9C
:1054A800B72500209385056112072E97920750476C
:1054B8008820A107BE95EFF01FB459A89307800F65
:1054C80063F4B700614599BF372A002083464A55DF
:1054D800B7270020138707619206369748479389B4
:1054E8000761130A4A5509C997B0FA1FE78000C235
:1054F800B7270020A38907541306140091659385E4
:105508000571328503490A0032C697B0FA1FE78051
:10551800E0B283470A0012094E9992072326A90090
:10552800CE97C84745D13246814597B0FA1FE780E4
:10553800A0E683470A002286A6859207CE97C84729
:1055480097B0FA1FE780A0DEB7270020A389875409
:105558000145E9B5E398F5F61A22B7270020239804
:10556800E754FDB78547E39FF5F41822B7270020D5
:10557800238EE754F1BF9947E396F5F437250020C9
:105588001946A6851305055697B0FA1FE78020DA55
:10559800C1B78547639DF5061822B7270020014546
:1055A800A38AE74C8280E147E39EF5F03725002087
:1055B8006146A6851305855FC1BF8547E394F5F06D
:1055C8001822B72700202382E74E59B78547E39B67
:1055D800F5EEB727002083C72755C9B58547E3935C
:1055E800F5EE082293772500E39E07ECB727002005
:1055F80083C7D755B7250020938505611387F7FF23
:10560800120792072E97A1075047BE956DB56145C1
:1056180082804111AA8706C611472E856386E70A4C
:105628006361F7020547638EE706A9C709476381E7
:10563800E7080D476384E7088947B2403E85410182
:1056480082801D47638AE708636AF7001547E39578
:10565800E7FEB727002083C7574DB9A821476383C2
:10566800E70813072004E399E7FCB727002083C75E
:10567800474E99A0B727002083C74755139747007F
:10568800B727002093870761BA97CC478947D5D5B4
:10569800B727002003C6375597B0FA1FE78020C9FF
:1056A80031A0B727002083D707559EA1814771B73E
:1056B800B727002083C7C7551CA1CDBFB725002039
:1056C800194693850556C9BFB725002021469385FD
:1056D800C54DEF804144D9BFB72500206146938569
:1056E800855F5DBFB727002083C75755F1B7630FA4
:1056F8000538B7270020938767559823631807381C
:1057080085463728002094A309479307086198A382
:1057180037E706001307C728D8C337E7060013077B
:105728008725D8C794A7239507007D57630DE534CF
:1057380013771500854539C3B7E606009386862694
:10574800D4CBB72600209386764D0947D4CFB72609
:10575800002098AB238AE6542380E70237E7060047
:1057680005461307072790AF239D0700D8D3238446
:10577800C7022395070223A607028D451377250044
:105788002DC313974500B7E606003E9793868626F5
:1057980054C3B7260020894805469386464D54C70A
:1057A8002300170110A723150700138715004207C8
:1057B8004183B72600202389E6541207B7E606007E
:1057C8003E979386062654C38905B72600209386FC
:1057D8000655C2052300170110A72315070054C753
:1057E800C181137745002DC313974500B7E606001E
:1057F8003E979386862654C3B726002089480546D7
:105808009386464E54C72300170110A72315070097
:105818001387150042074183B7260020A38EE6545C
:105828001207B7E606003E979386862854C3890573
:10583800B72600209386C655C2052300170110A776
:105848002315070054C7C1811377850021CF13970B
:105858004500B7E606003E979386862654C38546DC
:1058680014A7B726002009469386564E54C710A39E
:105878002315070013871500420741831207B7E66F
:1058880006003E979386462954C3A14614A7890566
:10589800B726002093860656C20510A323150700D5
:1058A80054C7C1811377050129CF13974500B7E67F
:1058B80006003E979386862654C3B726002089485B
:1058C80005469386A64D54C72300170110A7231534
:1058D800070013871500420741831207B7E6060041
:1058E8003E979386462854C38905B7260020938699
:1058F800C64DC2052300170110A72315070054C77A
:10590800C1811377050229CF13974500B7E6060032
:105918003E979386862654C3B726002089480546B5
:105928009386664D54C72300170110A72315070057
:1059380013871500420741831207B7E606003E9712
:105948009386462654C38905B72600209386564D6C
:10595800C2052300170110A72315070054C7C181EA
:105968001377050429CF13974500B7E606003E973D
:105978009386862654C3B726002089480546938611
:10598800664E54C72300170110A723150700138775
:105998001500420741831207B7E606003E97938633
:1059A800062954C38905B726002093866656C20582
:1059B8002300170110A72315070054C7C1811377C7
:1059C800050821CF13974500B7E606003E97938652
:1059D800862654C3D14614A7B726002009469386C5
:1059E800864D54C710A323150700138715004207D7
:1059F80041831207B7E606003E979386462754C3AD
:105A0800854614A78905B72600209386865FC205B8
:105A180010A32315070054C7C1811375051039C990
:105A280013974500B7E606003E979386862654C32B
:105A3800B7260020094505469386964D08A310A76A
:105A48002315070054C7138715004207418312071F
:105A5800BA9737E7060013074727D8C389053727BA
:105A6800002013075755C20588A390A72395070060
:105A7800D8C7C181B72600209386864741461305BB
:105A880008616F30202E130530037DB101458280F7
:105A9800011106CE22CC0546638CC5021146094485
:105AA800639EC5023EC63AC436C2EFD0AF8C2A8484
:105AB80092462247B2471DE13E86BA853685EFD029
:105AC800CF81EFF06FD0EFF06F95EF60E06639A00F
:105AD800EFD04F8A2A8419E1EFF00FCF2285F240E8
:105AE80062440561828079714ECEAE896C0022D401
:105AF80026D24AD006D62A89B284EF0090682A8432
:105B08000DE1CE854A85EFC04FE02A8419E9324578
:105B1800B72605002687938666102D468145EF1027
:105B280020002285B250225492540259F24945610C
:105B3800828079714ECEAE896C0022D426D24AD0AA
:105B480006D62A89B284EF00D0632A840DE1CE8577
:105B58004A85EFC00FE92A8419E93245B7260500BE
:105B680026879386061E4D468145EF00707B228569
:105B7800B250225492540259F249456182803971D7
:105B880026DAAE844C0022DC4AD84ED652D406DE41
:105B9800AA893289368AEF00D05E2A8421E9A6854F
:105BA800630D09009E202C007C84BE207C85930711
:105BB80020307C86930780025C874E85EFC00FD229
:105BC8002A840DE55946A6851305A1002304210161
:105BD80097A0FA1FE780A0751245B72605005287DF
:105BE8009386860B25462C00EF0090732285F25091
:105BF8006254D2544259B259225A21618280797131
:105C080026D2AE846C0022D44AD04ECE06D6AA89BB
:105C18003289EF0010572A840DE1A6854E85EFC022
:105C28008FD02A8419E93245B72605004A8793861A
:105C380026123546A685EF00B06E2285B250225452
:105C480092540259F24945618280BD47638CF5063A
:105C580063E9B702A5476387F50663EDB70099477F
:105C6800638CF5049D47638FF5049547638CF504B1
:105C780001458280B5476387F50463E1B704AD4702
:105C8800F5B7DD47638EF50263EAB700C947638B52
:105C9800F502D9476386F502C547C9BFF54763834F
:105CA800F50263E4B700ED47D1B793072005638B8E
:105CB800F5009307200D5DBF48458280084182802A
:105CC80008458280484182809307F00F630FF506EC
:105CD800011126CAAA841305000222CC4AC84EC65E
:105CE80052C456C206CE3A89B689B28A2E8A97A07D
:105CF800FA1FE78000542A844D450DC8930700FB1E
:105D08001CA0A300540123114401230234011305EC
:105D18008400614663050902CA8597A0FA1FE780D7
:105D28000061A2852685EFA0BFAB0145F240624421
:105D3800D2444249B249224A924A05618280814549
:105D480097A0FA1FE7804065E9BF094582800111E5
:105D580022CC06CE2A844C86D08697B0FA1FE780DC
:105D680020D305C15425B73700202147938787974B
:105D7800639DE600E82378009306E0070146A285C4
:105D8800A137F24062440561828078009306E007FB
:105D98000146A285C833EDB7930700643306F602BF
:105DA8006FB0CF8A15C5182185469307270093F74A
:105DB800F70F63FFF600411122C42A843A8506C60C
:105DC800EFB0CFA2FD571CA0B2402244410182800F
:105DD80082801A219307000B6310F7025C21494760
:105DE800639AE700183985476398E7002A218545B3
:105DF8006F30501B6D47CDBF828001116C846C00E1
:105E080022CC26CA4AC806CE2A89B6847085EF00F5
:105E180050372A840DE12C004A85EFC0CFA22A848E
:105E280019E93245B726050026879386C600154628
:105E38002C00EF00F04E2285F2406244D2444249E1
:105E4800056182807971930720306C8470857C8627
:105E58002C0093078002014606D65C870D33B250AA
:105E680045618280C177797185073EC4894726D20A
:105E78007C86AE84930780024C0022D44AD006D692
:105E88002A895C87EF00F02F2A840DE12C004A85CF
:105E9800EFC06FB22A8419E91245B7260500268794
:105EA8009386061945462C00EF0090472285B2508C
:105EB80022549254025945618280B2860546C1B186
:105EC800797126D2AE846C0022D44AD04ECE06D642
:105ED800AA893289EF00F02A2A840DE1A6854E8529
:105EE800EFC02F8E2A8419E93245B72605004A8764
:105EF800938626FB0D46A685EF0090422285B25078
:105F0800225492540259F24945618280797193076B
:105F180020206C8470857C862C00930780020146C3
:105F280006D65C87EFF0BFC5B2504561828001118B
:105F380022CC06CE2A842EC632C436C297B0FA1FA7
:105F4800E78000B50DC94825B7370020A1469387DB
:105F5800879712472246B245631AD500E823B286CE
:105F68002E86A2856244F2400561B9BBB286C83369
:105F78002E86A285C5BFF240624405450561828030
:105F88006FF07FB66FF03FB66FF07FC76FF03FC717
:105F980079714ECEAE896C0022D426D24AD006D66C
:105FA8002A89B284EF00F01D2A840DE1CE854A8546
:105FB800EFC02F992A8419E93245B72605002687AC
:105FC8009386E6133D468145EF0090352285B25011
:105FD800225492540259F24945618280B2860146A0
:105FE8006FF0FFB9011122CC2E846C0026CA06CEB0
:105FF800AA84EF001019DD476309F5009307101014
:106008001EA4A2852685EFC0CF9DF2406244D244EB
:1060180005618280239405009E2599E36FF07FB186
:1060280009458280C5BFB727002003C7E7598547C0
:1060380063F8E702011122CC2E846C0026CA06CE32
:10604800AA84EF00101401E9930700101EA4A2858A
:106058002685EFC00F99F2406244D24405618280E0
:1060680059458280B727002023A4A7568280B727E6
:10607800002023A6A7568280011122CC26CA06CE6C
:106088002A84AE8497B0FA1FE78080A0A68522856F
:10609800EFB03FC705E92285648697B0FA1FE7800D
:1060A800209F0DC15425B737002021479387879734
:1060B800639FE600E82378009306F0070146A2856F
:1060C800EFF09FC0F2406244D24405618280C83339
:1060D800DDB7011126CA06CEB68422CCDD4663E3BD
:1060E800B608D94663FFD50AA5466382D50A63EF89
:1060F800B6049546638DD50899466388D50A054444
:1061080041687D18631706093AC6EFB05FC33306C6
:106118008540324742064182420441803305C4002B
:106128004205BA85418132C6EF30C075AA8751C190
:1061380099C0324692A0B30580406244F240D244EE
:106148003E85056117A3FA1F67008309C54663806A
:10615800D504C9460D44E394D5FAC167FD17E31D7C
:10616800F6FA5DB7F5466380D50463E4B600ED46FC
:10617800D5B7930620056388D5029306200DE390D2
:10618800D5F8C167FD170D446319F600B5BF09447A
:1061980085BF9306200DE391D5F83106420641826A
:1061A800A5BF15445DBF0D444DBFC167FD171D4414
:1061B8007DB7F2406244D24405618280011122CC4D
:1061C80026CA06CED0212E8413070002814699459F
:1061D800AA8401372AC621C51E20502093055400E1
:1061E8007C803E207C8189477C82930780025C8387
:1061F80097A0FA1FE780A0135C208A8526857C84F7
:10620800EFB01FE72A8411C5324597A0FA1FE7802F
:10621800E0EF2285F2406244D244056182804D4419
:10622800CDBF5D7186C6A2C4A6C2CAC04EDE89476C
:106238006306F600C14709446318F6040144A9C57A
:106248002E894C0832C6B689AA84252F2A8432465C
:1062580005EDC1778507CA851305D1013ECC230E0C
:10626800C10097A0FA1FE780800C2C082685B93753
:106278002A8419E95245B72605004E879386E60514
:106288001D462C08EF00D0092285B64026449644C6
:106298000649F25961618280797122D436844AD0E4
:1062A8004ECE52CCB2892E8A3A8981461307100203
:1062B8002286D94526D206D6AA84213D2AC621C1DE
:1062C8002286CA856084231241012313310197A0D5
:1062D800FA1FE780C0054C002685EFB05FFA2A84D4
:1062E80011C5324597A0FA1FE78040E22285B250D7
:1062F800225492540259F249624A456182804D44BF
:10630800F5B7011122CC26CA06CE4AC8DD472A8431
:10631800AE846389F50281470A206C005C86EFB081
:10632800DFF905456380A4080824B165938505B89D
:10633800EFA07F87E5473CA0B72705009387872B09
:106348005CC085A058393149B286330627031849FD
:106358009C4232971043E310F6FCDE225223E31CE2
:10636800F6FA8C46084797A0FA1FE780400D45D5F6
:106378005C385828850793F7F70F5CB863FAE7028B
:10638800B387270318480A20BA979847D623B22319
:106398008E23193749F10824B165938505B8EFA014
:1063A8009F805945F2406244D24442490561828047
:1063B8007C289DB7011122CC26CA06CEDD472A8447
:1063C800AE846393F5060A21EFB07F97522C3628E6
:1063D8005A286D162A9642064182B307D640C2074C
:1063E80052ACC18363F9E7069305C5FF3308F7404C
:1063F8006358B802BA96918EC206184C0E280A2025
:10640800C1823E97513D0DE10824B165938505B8D9
:10641800EFA06FF95945F2406244D2440561828089
:106428006D1593160501D1BF81470A206C005C8663
:10643800EFB0BFE80545E380A4FE0824B165938565
:1064480005B8EFA04FF6E5473CA0B72705009387AE
:10645800872B5CC0C1B78547C9BF397126DAAE84BE
:106468002C0022DC4AD84ED606DE2A89B289112BA6
:106478002A8431E54A85EFB09F8CD6206D1563C517
:10648800A60093160501C1829844B2208E204A8541
:1064980021352A840DE53146A68508082306010022
:1064A80097A0FA1FE780A0E8BE202245B72605007E
:1064B8004E87938606255D466C00FC8695252285C9
:1064C800F2506254D2544259B2592161828071B754
:1064D80069B7797126D206D622D44AD04ECE52CC8C
:1064E80056CA5AC88944D1C949CA2E842A89BA8A3F
:1064F800368B328AEFB0BF8493054400814771150B
:106508009A21635DA708850793F7F70FB105E3198B
:10651800FAFE8A854A85B521AA8425E131453305E5
:10652800AA02916593851570CD4497A0FA1FE7805C
:10653800E0B0AA8939C131463306CA02A28597A0BC
:10654800FA1FE780C0DE1844562032200E204A8504
:10655800A133AA8415ED0245B7260500854756875D
:10656800938606255D464C005C824EC42306410195
:10657800A3060100230761016523B2502254268532
:1065880002599254F249624AD24A424B456182808A
:106598004E8597A0FA1FE78060B7C5B7ED44F1BFF5
:1065A80079714ECE37E60600AE89C16526D201471D
:1065B800AA8489461306C629FD15054522D406D6A0
:1065C8004AD0EF10A078054429C92A891307300258
:1065D80081461146F5452685EFF0BFAF2AC65544DA
:1065E8000DCD8357A900CE8601467C8491477C85D2
:1065F80085471CA1B2472C002685A3800700324797
:10660800FD573CA332473CB3EF10C0692A8411C53B
:10661800324597A0FA1FE78060AF2285B250225416
:1066280092540259F24945618280411106C6EFF041
:10663800CFE119C5B240410117A3FA1F670003ADA6
:10664800B24041018280011106CE2AC6EFB00FD6B2
:106658003245B727002023A40756B727002023A6D2
:1066680007569145B7370020A38CA796EF30201C1A
:10667800F24005616F2070037971939705014AD044
:1066880006D622D426D2C187014963DB070AB73769
:10669800002003C597972E8997A0FA1FE780C0BEF0
:1066A8002A8441CD18219307000A6315F708854706
:1066B8004C08DC85EFB02FDCAA8405ED8347610127
:1066C80071476376F708138717FE1377F70F93065A
:1066D800000263F5E608858BCDC7B727002083A79E
:1066E8008756994499C72A201306B1004C08829707
:1066F800AA849C8599C7084409C597A0FA1FE78012
:10670800E0A095E05247B7070001938707F07D8F17
:10671800B707120093870710630EF700034761015C
:10672800ED476319F7002A208545EF30A007CD47CC
:106738006388F4002285EFA0CF85A1673349F9006B
:10674800B25022544A8592540259456182803707D3
:10675800301405073357F700058B35DF372700203E
:106768000327C75659D70347510141F75C86994714
:106778002308F1002A206C0023170100EFB08FF2E4
:106788008DBFB727002083A7C7568DC32A201306BD
:10679800B1004C08829731DDAA8483475101B1FBCF
:1067A80083476101230891005C86E9B79944F5B7EE
:1067B800397122DC26DA06DE4AD84ED652D456D2B1
:1067C8005AD0A5472A84B2846398F50E83474502B8
:1067D8001A22835A260085072302F5029307F7FF3A
:1067E800B387FA025442C207C183B69703C9170098
:1067F8009C23542522093369F90085476390F602E2
:1068080033075703231006008149014A130B35014A
:10681800931A070193DA0A0163EA5905C167FD175C
:106828006303F90A1E286370F90A0509420954240A
:10683800135909012317240105470A209305E40089
:10684800639CE6007C85930720307C869307800252
:10685800231421015C872C00EFB05F880824B16500
:10686800938505B8EFA02FB45945B9A8B620DC40E8
:106878002C28ED1613865900C206C1823E965A8509
:10688800EFB0CFB705C5630B3A01C840B220B305D6
:106898003501529597A0FA1FE78060A9BE203E9A5D
:1068A8009E20420A135A0A0185079EA0BE20BE995F
:1068B800C20993D909018DB75822A9476310F70275
:1068C8008347450281CF0145F2506254D254425960
:1068D800B259225A925A025B2161828034281309E4
:1068E800340137E506004A8689451305C528EFB007
:1068F800EFB019C10545C9BF342837E506004A86F7
:10690800894513058529EFB06FAF6DF5342837E554
:1069180006004A86894513050528EFB02FAE79F998
:10692800342837E506004A86894513058526EFB0E1
:10693800EFAC69F1D820BD47E3EEE7FAA567938786
:106948004712B3D7E700858BD5D78347440285071D
:106958002302F40203D92400D1B5011106CE2EC6B4
:1069680097A0FA1FE780200811C93C25B245138774
:1069780017006395E50093F707F83CA5F240056119
:106988008280011106CE2EC697A0FA1FE780A005C7
:106998001DC1B24591C188C11C251307E00F5D4593
:1069A8006388E7001307F00F01456383E700594543
:1069B800F240056182800945E5BF411122C42A845D
:1069C800210506C626C24AC0EFF0CFBD3C20A51758
:1069D80093F7D70F89EB58248547631EF7041C48A3
:1069E80081443149A1E3FD57230104001CB423026B
:1069F80004021305C4002244B2409244024961468D
:106A08008145410117A3FA1F67000399B38724033F
:106A18003E95084509C59790FA1FE780206F8504C1
:106A280093F4F40F5C280848E3E2F4FE9790FA1F09
:106A3800E780C06D4DBF084C75F975B7411122C488
:106A4800416406C626C29307E4FF6301F502AA84DF
:106A58009DE197A0FA1FE78000F909E91305F4FF03
:106A680097A0FA1FE78020F811C106A1B24022447E
:106A780092444101828085476391F50497A0FA1FEB
:106A8800E78060F62A847DD1FD571EA11C241307D8
:106A9800F00F6381E7021307E00F6389E7003420F2
:106AA800083401475146A685EFF00FA222853137F9
:106AB800FD571CA42305040055BF8947E398F5FA40
:106AC8008545EF40203D5DF1268597A0FA1FE780B8
:106AD80080F12A8445FD59BF39C118259307F00F65
:106AE800630FF702011122CC06CE2A8434210E212D
:106AF800083501475D46EFF02F9D3820E1476318C0
:106B0800F7000A206C0023060100EFB00FFBF957CD
:106B18001CA422855D35F240624405618280828032
:106B28009307F00F6306F706011122CC26CA2A84C0
:106B38004EC6AE84B689AA859306850037750500CA
:106B48004AC852C43A89328A130505AE794606CE38
:106B5800EFF08FA4A304240123014401232234016C
:106B680085C01305C4006244F2404249B249224A32
:106B7800A685D244614605611793FA1F6700237BF7
:106B8800F2406244D2444249B249224A05618280B5
:106B98008280B7270020238AA7568280954763946E
:106BA800F50683474502854685072302F5021E221E
:106BB80058423022FD17C207C1836312D6048A07E0
:106BC800BA9798339C232207D98F7A2563F5E7046F
:106BD800411106C622C485075EA52A849305C5000F
:106BE8000A21EFB04FC60824B165938505B8EF9028
:106BF8009FFBB2402244D9473E8541018280C94665
:106C0800B387D70275BF5422294785476396E600A4
:106C18000347450211C381473E8582809D47639B98
:106C2800F50483474502762585072302F5021E22CF
:106C38005842FD178A073E971C331823A207D98F9D
:106C4800014763F2D704411106C622C485072A8486
:106C58005EA59305C5000A21EFF04FD60824B1655B
:106C6800938505B8EF903FF4B240224459473A85DE
:106C7800410182805422A94705476396F6000347DD
:106C88004502133717003A858280411122C406C68F
:106C980026C2B5472A846395F50483474502B28422
:106CA80085072302F5020A21EFB06F899E2013079A
:106CB800F5FF014563C1E7027A240A209305C40061
:106CC800BA977EA4EFB02FC60824B165938505B89E
:106CD800EF907FED5945B2402244924441018280B1
:106CE80058229D470545E318F7FE0345440213352E
:106CF8001500D5B7C5476396F5061E223A22FD173B
:106D0800B387E7020347450205072302E502584215
:106D1800C207C1833E973C333823A207D98F416706
:106D28007D176395E70081473E85828013871700AA
:106D38005AA57A25E3F9E7FE411122C49305C50057
:106D48002A840A2106C6EFB00FC70824B1659385C7
:106D580005B8EF905FE5B2402244D9473E8541012E
:106D68008280542229478547E390E6FC0347450281
:106D78005DFB5DBF011122CC26CA4AC852C406CEAB
:106D88004EC6BC2115472A8AAE8432843689639957
:106D9800E7043686A28526851135AA895DE18547EF
:106DA8006311F40A03474900A9476300F7028834CE
:106DB8004A8785460146D285EFE01FF119E58545EA
:106DC8004A85EFE09FE813341500B4208834014762
:106DD8006946D285EFE05FEF2685EFF01FBEB5A8C4
:106DE8001D476397E7003686A2852685053D75B75A
:106DF80025476398E7003686A2852685EFF05F9BD6
:106E080069BF35476397E7003686A2852685B53D75
:106E180069B745476397E7003686A2852685D93D39
:106E2800ADBF5D47639EE700D82585473686A285B6
:106E38002685631DF702EFF0CFCC8547631AF5046A
:106E48008549A5476317F402835709009DE3054464
:106E5800E38D09F6D947E391F9F82285F2406244B7
:106E6800D2444249B249224A05618280EFF08FD468
:106E7800E9B788344A87A2860146D285EFE0DFE485
:106E880079F5A2854A85EFE05FDC13341500C9B7B0
:106E98000544E1B7397122DC06DE26DA4AD84ED637
:106EA80052D456D29E211944B9E783C925002A89AC
:106EB800328A938759FE93F7D70FAE84DDE3B7275D
:106EC800002083C647571307F00F938A4757194482
:106ED8006383E602F5476395F90497A0FA1FE780F4
:106EE80080B0AA891DCD30250DCE93178601E18784
:106EF80063DD070001442285F2506254D25442599E
:106F0800B259225A925A21618280F5454A85EFE0AA
:106F18001FE483C7A90093E707F82385F900D9BFC1
:106F28008149D62090448C3088203800EFB0EFB9E2
:106F38002A8471F1B42003C50A0038000146CA85C5
:106F4800EFE09FD82A8445F9B24799C323000A0085
:106F5800BC207547E390E7FAE38E09F82385F9002A
:106F680059BF97A0FA1FE78000A8AA8A41D585478C
:106F7800639FF908CE2088443000EFA03FDE2A84C2
:106F88003DF903C72A00C54763FFE708DD47630DDE
:106F9800F70AB737002003C59A0083C79797639805
:106FA800A70A014403C72A008D47631EF7043C84DF
:106FB80003D7CA0063F4E7002396FA0083D5CA0012
:106FC8004A85EFF06F8BB727002083D7877E6D4700
:106FD800637BF70283D5CA005D476376B7021387E0
:106FE800350091056349F7001307B00FBE85637438
:106FF800F7009305B00F1166C20513060629C18173
:107008004A85EF70702C5685EFF03F9BEDB53C211B
:107018001144E39237EF5C41E38F07ECCE208844BC
:1070280030008297A9BFB72702009387072AB3D7F2
:10703800E700858BB9DFB0203400D6854A85EFF0AC
:107048007FD32300AA0045BD83A70A01E5B7B42072
:1070580038000146CA85EFE03FC72A8421F5AC20F5
:107068002800EFE09FBE15DD23000A0025BF0111AF
:1070780022CC3734002006CE26CA4AC84EC652C48F
:107088009309849703C589009307800291653305A6
:10709800F502938565703729002093040957979066
:1070A800FA1FE780A0F903C689009307800281458B
:1070B8003306F60288C09790FA1FE780E02D9C40BF
:1070C8004D459DCF93048497130909570144130A2A
:1070D8008002FD599C24636DF40237750500130581
:1070E800C5E9EFE03FF83775050013052596EFA0D1
:1070F8005FB737750500130545A4EF30B05001455B
:10710800F2406244D2444249B249224A056182802F
:10711800B307440303250900614681450504137438
:10712800F40F3E9523103501230105002314350182
:10713800230505002302050231059790FA1FE78011
:10714800A02549BF01458280B737002083C617981C
:10715800814763E5D70001473A8582802E879105EC
:1071680003D6C5FFE30AA6FE8507E5B70DC93C218E
:107178000547890793F7F70F6373F702411122C494
:1071880006C62A840E2128310147F9465D46EFE0FC
:10719800BFB3F9573EA0B2402244410182808280A9
:1071A800B737002003C71798FD56814763E3E70008
:1071B800828016A12301050085071105C5BF014579
:1071C8008280372600201306764F930700021CA200
:1071D80037270020FD57230BF74E372700202304BD
:1071E800F74E37270020A303F74E8545B727002021
:1071F800239AB74EB7270020239B0756B7270020AE
:1072080023A00758B727002023A80758B72700202E
:1072180023A20758B7260020B7E706009386C64E74
:107228009387C727DCC2B7270020238C0756B727C8
:10723800002093874748094798A298A398AB2380D2
:10724800E7022388E70237E706001307C726D4C7F3
:10725800D8DBB7E606000D47238CE702938686261F
:1072680037270020D4CB0327C75737E50600B7E6F2
:1072780006001305C5289386C629C8C38CA723957D
:1072880007008CAF239D0700D0CFD4D323840702F7
:107298002395070223A60702239D0702D8DFB727F5
:1072A8000020377705009387474C1307273623A01C
:1072B8000700D8C323A407008280411106C6693598
:1072C80009C52821B240410182800145E5BF41112D
:1072D80022C426C24AC006C6AA842E893284AD3585
:1072E80001E94165CA857D158535C54701C506A1F2
:1072F80020A18147B2402244924402493E8541017F
:10730800828029E389483547639F1603011106CE19
:1073180022CC26CA1832102293C7F7FF2207598EAB
:10732800F18F32C69DE3C4452A84A6857937324653
:107338000147630EA60022856244F240A685D24426
:10734800056171B72D473A85828013070008F2401E
:107358006244D2443A850561828083C805000948A1
:107368006394080303A845008347180003480800EE
:10737800A207B3E70701C2070D68C1871308289061
:10738800639407018947B5BF05458280011122CC66
:10739800372400201304844E182006CE26CA4AC873
:1073A8004EC69307F00F630FF702AA892945B284E6
:1073B8002E899790FA1FE780C0E70DC59307100B39
:1073C8001EA123020500231135012313250106A55B
:1073D800AA8508206244F240D2444249B249056174
:1073E8006F900FC0F2406244D2444249B2490561ED
:1073F80082804111B727002026C2AE8483A5C757D3
:1074080022C406C62A84553D098909C92285224411
:10741800B240A685924441016FF08F98B240224451
:107428009244054541018280411122C426C24AC0C6
:1074380006C6AA84130445001309850B1E209DC3A4
:10744800084409C59790FA1FE78040CC2285314649
:1074580081459790FA1FE78020F43104231A04FE2F
:10746800E31E24FDB2402244FD579EA002499244E7
:1074780041018280B737002003C61798B72700203C
:1074880003A7875881476315F600814636858280B1
:10749800BA861307870B835587F4E389A5FE85070A
:1074A80093F7F70FCDB7B727002083A7075981CBEC
:1074B800DA236314A700884782809C43CDBF014527
:1074C8008280411106C6C53709C50845B240410149
:1074D80082800145E5BF011126CA9384450022CC6C
:1074E8004EC606CE4AC852C456C25AC026878149DB
:1074F8000144814681473D45122345CABDEE4223DA
:107508003E23B286A297C207C18385093107E39556
:10751800A9FE35C42E89916593854570228597907B
:10752800FA1FE780A0B12A8B39C9814A014A8C44E5
:1075380095C1D22033054B019790FA1FE78020DFD1
:10754800DE2088443E9A420A135A0A019790FA1F8D
:10755800E780C0BB63890A0031468145268597903C
:10756800FA1FE78060E3850AB104E3E23AFD2326C7
:10757800690123148900054521A0630DD600014542
:10758800F2406244D2444249B249224A924A024BEA
:10759800056182803223E314F6FE52233294B297B7
:1075A8004204C2074180C1838DB70545E37A35FDA2
:1075B8008DB7B727002083A7475899E301458280F4
:1075C80098473A276315A7001385470082809C4394
:1075D800EDB7411106C6F13F09C50A21B240410184
:1075E80082800145E5BF411106C6E13709C528215A
:1075F800B240410182804145E5BF411122C42A843D
:107608002E8506C6CD37AA8505462285EF308068C7
:1076180095476305F500BD476313F5002145B24062
:107628002244410182804111B727002022C406C6A6
:1076380003A4475881469387475821C018443227E6
:1076480018406317A60285CA98C22E8581C92146AB
:10765800930544009790FA1FE78060CD22859790A4
:10766800FA1FE780A0AA0145B24022444101828066
:10767800A2863A84D9B798C3C9BF0545F5B7372755
:10768800002083270759014613070759A1C703D8C4
:1076980047009443631BA802011106CE22CC26CAD8
:1076A80005CA14C2AA843E852E849790FA1FE780E3
:1076B800E0A52C002685853F01E519C0B2471CC00E
:1076C800F2406244D244056182803E86B6877DBF1F
:1076D80014C3C9BF05458280411122C42A84090503
:1076E80006C6EFE02FECFD573CB0B2402244410102
:1076F8008280411122C4416406C626C29307E4FF72
:107708006301F502AA849DE19790FA1FE780C030D3
:1077180009E91305F4FF9790FA1FE780E02F11C1DC
:1077280006A1B24022449244410182808547639178
:10773800F5049790FA1FE780202E2A847DD1FD5703
:107748001EA13C201307F00F6381E7021307E00F27
:107758006389E70028300147F9465146A685EFE0DE
:10776800AFD62285953FFD573CA02302040055BFA4
:107778008947E398F5FA8545EF30C0715DF12685B4
:107788009790FA1FE78040292A8445FD59BF1D714B
:10779800A6CACEC686CEA2CCCAC8D2C4D6C2DAC0C1
:1077A8005EDEAE84AC21F947AA896396F50497900A
:1077B800FA1FE78060262A8411ED01442285F640ED
:1077C8006644D6444649B649264A964A064BF25B71
:1077D800256182803C210547890793F7F70FE37EEF
:1077E800F7FC28310147F9460146CE85EFE0CFCDB9
:1077F8002285DD35D9B703AB0400B70700019387AD
:1078080007F037071200B377FB0013070710B28A97
:107818000149638BE7022EC69790FA1FE780C01FC5
:107828002A89B24515C1502105C293178601E187FF
:10783800E3C507F84E85EFE08FD18347490093E70A
:1078480007F82302F90095BF372A002003476A4F3B
:107858009307F00F130A6A4F1944E301F7F6E1475B
:10786800E3EEB7F493D71500FD1713973700B7E782
:107878000600938707BFBA9703A80700E30008F438
:1078880083AB4700E38C0BF2420B135B0B016305E0
:107898000B00C947E394F5F2D62090448C30882039
:1078A800380802982A8419F92C084E85829B2A8464
:1078B80031C19C30E39407F0BC20230AA10039476A
:1078C8002308F1006396E70262471C331823A207D6
:1078D800D98F0C084E85FC81EFA0CFDCE30F05ECB7
:1078E80014080546D9454E85EFE06FE42A84F9B5BA
:1078F800BC84C5B7B4209147E381F6EC03450A0080
:1079080038080146CE85EFE02FBC2A84E31805EA43
:10791800AC202808EFE06FB319C123800A00984013
:10792800B7070001938707F07D8FB7071200938789
:107938000710E304F7E8E30209E8BC202302F90092
:10794800B5BD011106CE2EC69790FA1FE780C00C70
:1079580011C95C21B245138717006395E50093F7B9
:1079680007F85CA1F24005618280397152D42E8AF1
:107978004ED69305E101AA89528522DC4AD856D20F
:1079880006DE26DA328936C63AC4BE8A9790FA1FCE
:10799800E780400B054435C1AA84A8873944EFF035
:1079A8009FB021CD03284500630908042247B24649
:1079B800D6874A86A6854E8502982A841DED9307A8
:1079C800E00F638CFA02982089476318F702D840C1
:1079D8001C331823A207D98FC2070D67C187130765
:1079E8002790639CE7008347190003460900D28566
:1079F800A2075D8E4E85EFF07F992285F250625482
:107A0800D2544259B259225A925A216182807971CC
:107A180022D422214ECEAA89228556CA06D626D23B
:107A28004AD052CC5AC85EC662C4AE8AEFF09FA450
:107A380001E92285EFA0DFD2594429E5014499A044
:107A480003C789008547AA8401446316F702AA85FB
:107A580013858900EFF03FA821C9FA209624D04465
:107A6800CE2003D52900E1470937D9472A8463186E
:107A7800F50223A604002685EFF01F9B41C0D947D5
:107A8800E30EF4FA2285B250225492540259F24974
:107A9800624AD24A424BB24B224C4561828061DD38
:107AA800DE202390FA00C1BF13894400014AB94B74
:107AB800594C3D4B83550900DDDDE14763067A01EA
:107AC8000357C90011C3D9470357290083564900F2
:107AD8000326890003D52900EFF03FE92A846319BA
:107AE800850123240900050A3109E3156AFD61B7F8
:107AF8007DD9835709002390FA00F5B703D52900EB
:107B080015BF011170879307E00F1306E1000147C5
:107B1800894606CEEFF07FE5F240056182807971F3
:107B280022D42A840A2526D2AE849305210106D6BA
:107B38004AD09790FA1FE780E0F079C51C252AC63D
:107B480093F707029DC7A881EFF0BF97AA87B245B0
:107B580011E91E2439459EA0B2502254925402596C
:107B6800456182802A204946829701C51E249EA02D
:107B7800E5B7035924004A85EFF0DF8F01ED416531
:107B88007D15EFF03F8F09E51E2425459EA0E9B736
:107B980023102501130745008147BD46122339EEFE
:107BA8003147B387E702130984003146CA85910734
:107BB8003E959780FA1FE78080773146CA85480846
:107BC8009780FA1FE780A07652242A2041478146F1
:107BD800DD45EFE00FD02ACE09E51E2445459EA0DD
:107BE800A5BF0C4852249780FA1FE78040742A20CA
:107BF8004C08EFA0BFB22DD15945B9BF8507310751
:107C0800E39ED7F825459DB705458DB7797122D4F0
:107C18002A840A2526D2AE849305E1014AD006D6E5
:107C280032899790FA1FE780E0E12DC91C2593F768
:107C3800070295EF18389307200511E35C203624D6
:107C480050440E242A200147EFF03FD2AA8729E1A9
:107C58001C3891E72A20EFA07FA8D94711E1814776
:107C6800B2502254925402593E85456182802AC6F8
:107C7800A887EFF01F85AA8705C5B2452A2049467F
:107C88008297AA8745D91A249AA0183869FBC9BFD0
:107C98005947E31AE5FE23000900D1B78547E5B740
:107CA800B947D5B7397122DC4AD84ED652D406DE48
:107CB80026DAAA892E8A32C636899790FA1FE78073
:107CC800A0D509440DC53C211307E00FAA845D44E3
:107CD800638FE7001307F00F5944639AE7003246B1
:107CE80005E2D2854E85EFA0DFAB2A841DCD228523
:107CF800F2506254D2544259B259225A21618280B8
:107D080003550A009305E101231F01009790FA1F0C
:107D1800E78040D3A887EFF01F8DAA8505464E85DA
:107D2800EF2050772A8455DDD9B79307F00FE30089
:107D3800F9FC37750500938624007946A685130556
:107D48004517EFE06F85A381240155B73971B7272F
:107D5800002026DA83A4475852D45AD05ECE62CC8B
:107D680006DE22DC4AD84ED656D266CA2A8BAE8B9D
:107D7800328C368A99E08149A9A0804483DC44008A
:107D88000149835AA400631499018440E5B73E244D
:107D9800A28963F8670105094209135909014104D9
:107DA800DDB7E3EAFBFE630B0A000C204840D286ED
:107DB80062863AC6EF909FE4324771DD19C32310FB
:107DC8005701F25062544E85D2544259B259225A40
:107DD800925A025BF24B624CD24C216182809A210A
:107DE800B621854763E5E60439C34111D42126C28B
:107DF80037E506009384550022C426862E84130591
:107E0800C528894506C6EF907FDFC14719C95420A8
:107E18002E200A2001472686EFF05FF3814711E103
:107E2800A947B240224492443E85410182803E8562
:107E380082802E860A22AE21854763E1A50219CDEC
:107E4800542241110147150606C6EFF03FF081475D
:107E580011E1A947B2403E85410182803E8582807A
:107E68002E860A22AE21854763E1A50219CD542248
:107E780041110147150606C6EFF05FED814711E194
:107E8800A947B2403E85410182803E858280397192
:107E98004ED6BE2183D9050006DE22DC26DA4AD872
:107EA80052D456D25AD05ECE62CC66CA6AC863EA49
:107EB8003715854763880912416BAE8A2A8A2314CD
:107EC800010002C6014401497D1B894B054CC94C80
:107ED800054D83D52A000147814601464E85231367
:107EE8000100EFF0BFE6AA84630B050E09EC130747
:107EF8002002930661005A8695455285EFE06F9DF2
:107F08002A846302051038849C2041CB18856305B8
:107F1800A70741476385E7022C005285EFA00FCDE4
:107F280009CD34001546D9455285EFE04F8011C57B
:107F380032459780FA1FE780601D814765A0BE24FF
:107F48004146130524001CA0BE24A1831CB0CC40CC
:107F58009780FA1FE780A03D49043C848507C20743
:107F6800C1837C8463FD2707BE24638A670785096C
:107F7800C20993D90901B1BFE39077FBBE24094632
:107F8800130524001CA0BE24A1831CB0CC409780FC
:107F9800FA1FE780C0391104C9B722C60359610026
:107FA800B82413052400638F7701335999032305F7
:107FB800710118A0BE244146A1831CB0CC4013799E
:107FC800F90F79B72305810118A0BE241359290098
:107FD8001379F90FA1831CB00946CC404DBF3C84EE
:107FE80085FFA947F2506254D2544259B259225AD5
:107FF800925A025BF24B624CD24C424D3E85216153
:1080080082808547C5B7C547F1BFB727002003C79A
:10801800E759854763F4E706011122CC26CA4AC806
:1080280006CE2A843289AE849790FA1FE780C09ED4
:1080380019C538219307E00F5D456308F700631CF5
:108048000900A6852285EFA06FF2F2406244D2446F
:108058004249056182808A209305E10023170100C7
:108068009790FA1FE780009E2887EFF0CFD7AA8560
:1080780005462285EF20104269D5C1BF5945828047
:1080880013F7050201C7B2856FF02FD7411126C239
:108098004AC006C622C413F98500AA8463170900DA
:1080A800139785016187635B070232853684EFF099
:1080B8008FD3AA8505466313090001462685EF205C
:1080C800703D01E90145B240224492440249410110
:1080D80082801C34EDDB1C24F5F7F5B793F72500F7
:1080E800F5F30D45CDB77971AE8622D42A848A225C
:1080F8009305E10106D636C69790FA1FE78080946B
:1081080011C90C25B246B08722859D3FB250225432
:10811800456182800545DDBF13F7050201C7B285B9
:108128006FF0AFCD411122C426C206C693F4850074
:108138002A8491E413978501618763500702328589
:10814800EFF06FCAAA85054691E0014622852244D0
:10815800B240924441016F20F03393F72500014566
:1081680091E30D45B24022449244410182807971E5
:10817800AE8622D42A848A229305E10136C606D621
:108188009790FA1FE780008CB24609C90C25B08782
:1081980022855937B2502254456182800545DDBF9A
:1081A800797126D2AA842A25C16722D44AD04ECE14
:1081B80006D623170100FD173284B6890149630CDE
:1081C800F50005059420D04042051307E1004181E0
:1081D800EFF0DFB72A899420D04037E506008945BB
:1081E8001305C528EF909FA115C5A2242285EFF09D
:1081F8004FBE09C57D142A94420441806384090056
:1082080023908900B25022544A8592540259F24967
:10821800456182809420D04037E5060089451305E2
:108228008529EF90BF9D71F19420D04037E5060075
:10823800894513058526EF907F9C11C9E30809FA43
:108248003C87E39587FA0354A9007D1475B7A224E7
:1082580075B7397122DC26DA4AD84ED652D456D2AE
:108268005AD062CC06DE5ECEBE899C252A8AAE84B0
:10827800C18B328C36843A89C28A468B9DE783CB80
:1082880004008947638BFB046285EFF0CFA11DC111
:1082980083280500638008025A88D6874E87CA86D5
:1082A8002286A6855285829839A03285EFF06FA183
:1082B800AA8711ED3945F2506254D2544259B25945
:1082C800225A925A025BF24B624C21618280294603
:1082D800A6855285829745D5F9BFD8401C33182307
:1082E800A207D98FC2070D67C187930607906383DA
:1082F800D71E63CCF60693062780638ED70A63C021
:10830800F60213070780E3C1E7F82D45E39509FA5C
:10831800DC449023CC432310C9002285B9A213075B
:108328003780E393E7F62D45E39709F8854723104F
:10833800F900DC4481459C231CA0AA2405054205BC
:1083480041819780FA1FE780E06F83570900631027
:10835800051091072310F9001146814513051400F3
:108368009780FA1FE7804003F1A893062790638659
:10837800D71463C1D71093063790638DD7141307AA
:108388004790E393E7F02D45E39709F2DC441D4756
:108398002310E900982318A0983318B0BA2338A0FE
:1083A800BA23218338B0D82358A0FA2358B0FE2323
:1083B800A1837CA041A82D45E39F09EEDC446C0015
:1083C80083C917009823A209B3E9E90011472310CC
:1083D800E9009C234E851CA0DC449C331CB097808C
:1083E800FA1FE7802066AA8425C13086C1659306F6
:1083F800E100FD158329C500EFF09FDA09ED94200F
:10840800D04037E50600894513058529EF900FFF11
:1084180019E1FD577C8703C7090089476310F702F4
:1084280083A549000946130544009780FA1FE78091
:1084380000F08357090089072310F9003C873CA006
:10844800A1833CB0014585BD23173101C5BF182163
:108458008907BA972310F9003E251CB03E25A18351
:108468003CA010214C41130534009780FA1FE78087
:1084780000ECC9BFC8449780FA1FE780C0F493177F
:108488000501C1832A871D45E3E737E36399F900AE
:1084980023100900CC4403560900CE95BDBD420700
:1084A800B3863A01418363C7E600B3873741231097
:1084B800F900CDB723105901F1BF2D45E39D09DE21
:1084C800CC445285EFE07FDF2310790108A0218199
:1084D80008B08DBF2D45E39009DEDC4423107901F7
:1084E8009C231CA0DC449C331CB0A9BF1D71CAC8C6
:1084F8002A892A21A2CCCEC6D2C4D6C2DAC05EDE70
:1085080062DC66DA6ED686CEA6CA6AD8AE8AEF90E4
:108518001F83130CF5FF93170C01B72B0020C183A1
:108528002A8A814913840B743EC6372B0020B72C46
:108538000020C16D8357C90063F5F9001E2063CC84
:1085480087010355290093850B74EFA00F8E2A8DA0
:1085580015CD594D25A88327890013971900930530
:10856800E101BA9784339C23A204DD8C2685978089
:10857800FA1FE780204DAA8515E923909A00484004
:10858800054D09C59780FA1FE78040B8F640664454
:108598006A85D6444649B649264A964A064BF25B4E
:1085A800625CD25C425DB25D25618280324883485C
:1085B800490083A60C58B087035529008147130743
:1085C8006B57EFF01FC92A8D13880C5809C52390E3
:1085D8009A0048407DB75C4085E70355290051471C
:1085E80081461386FDFFBD45EFD0BFAEB7270020FB
:1085F80048C01388075809E523909A00454D79B774
:108608001E2003576B5793046B573E9763464701E9
:1086180013C7F7FF52979AA0484092208325080075
:108628003E9585099780FA1FE78060D01E209A2022
:10863800C20993D90901BA971EA0EDBD397122DC90
:108648002A842A2106DE26DA4AD84ED652D45AD0AF
:108658005ECE62CC66CA2E8B56D26AC8EF902FEED9
:108668002A8A54242E240A2478001306D400130CD2
:10867800BAFF651AEFF08FED420A37290020AA8960
:108688008144135A0A01B72B0020B72C0020130984
:1086980009746382090463D08405938A0C5883485B
:1086A800440083A60A0030862A205288814713870F
:1086B8006B57CE85138D6B57EFF0BFB91DC1814A3B
:1086C80030862E244E859306E100EFF07FADAA890F
:1086D80063990A065DFDF1E41E2429452310FB0079
:1086E80035A883570D001228E31BF6FC83A50A0062
:1086F80048489780FA1FE78080D471D183274900C2
:1087080095EF2A204166454781467D169D45EFD065
:108718005F9C1DE11E2445452310FB00F250625466
:10872800D2544259B259225A925A025BF24B624CC5
:10873800D24C424D216182802322A90083DAA9000C
:1087480041B783274900A6972380570193871400D0
:108758001397070183274900418393DA8A00BA9760
:108768002380570113872400832649009387340008
:10877800420791044183C207C204C183C18036976E
:1087880011C9348714A303274900BA97388721836E
:1087980098A301B7FD5614A303274900BA9794A3D9
:1087A8001DBF2A20B72500208980239095749385C2
:1087B8000574EF903FCF3DD159458DB7411122C483
:1087C80006C693F705012A84328585C3EFE0BFE129
:1087D800AA8505462285EF20E04B95476305F500FD
:1087E800BD47631DF502214515A893F7450099CBB0
:1087F800EFE07FDF0546AA8522852244B240410189
:108808006F20404993F7050489C7EFE0DFDD014693
:10881800DDB713F51500133515000605B2402244DF
:108828004101828079714AD04ECE52CC06D622D4EC
:1088380026D22A8AAE89014983D749006364F900A0
:10884800014581A083A7090013141900930414009B
:10885800338797001823A297882322079305E100FE
:10886800598D9780FA1FE780E01D05E583A7090069
:1088780005453E94182098A383A70900BE94982024
:1088880098B3B250225492540259F249624A45614F
:1088980082800C2530875285EFF05FF201CD83A7E7
:1088A80009003E94182098A383A70900BE94982035
:1088B80098B3C1BF0509420913590901B5BF011190
:1088C80022CC2A848A219305E10006CE9780FA1FDC
:1088D800E780401711C90C2530872285EFF01FEE7D
:1088E800F2406244056182800545DDBF1D71CAC83A
:1088F8002A892A2186CEA2CCA6CAD2C4D6C2DAC078
:108908005EDE62DC66DA2E8ACEC66AD86ED6EF9054
:108918000FC32AC68346C9008355A9000355890099
:1089280078081306D900EFF06FC2B247B7240020C9
:10893800416B938AA7FFC20AAA8B014493DA0A0102
:10894800372C0020B72C0020938404747D1B63828D
:108958000B18B08683C58B0003552900EFF01FE67E
:10896800AA8D631305168348490083A60C58B08660
:10897800035529005688814713076C57DE85EFF0A9
:108988005F8DAA8D93096C57138D0C58631E0512C1
:1089980015CC03D70900BE2011076397E7003247BB
:1089A800A2976D1763C7E706B7250020938705745C
:1089B800BA2303552900938505743354E40282A32E
:1089C800EF907FCAAA8D15C1D94D05A0035529007E
:1089D800494781465A86C545EFD0AFEFC8C015E56F
:1089E80083D7AB00C54D2310FA00F64066446E8568
:1089F800D6444649B649264A964A064BF25B625C1B
:108A0800D25C425DB25D2561828083D709009107FF
:108A1800BEA0DC4003D7AB009306E101A29798A360
:108A28009307140013970701DC4041835E85BA97CA
:108A380003D7AB00218398A3B0868355A900EFF034
:108A48002FF613072400D44093073400420711047B
:108A58004183C2074204AA8BC1834180369715ED32
:108A6800FD5614A3D84083250D00BA9794A3C84097
:108A780003D6090022959780FA1FE780408B83D799
:108A880009003E944204418005F083578900231071
:108A9800FA00E39C0DF4A94D89BFB48783250D0026
:108AA80014A3D840BA97B887218398A3C84003D69F
:108AB800090022959780FA1FE780608783D709000D
:108AC8003E944204418061B583D7AB002310FA007D
:108AD80065BF814D55BF5D71A6C2CAC0AA8403593E
:108AE80085002A21A2C44EDE52DC5AD85ED662D452
:108AF80066D286C656DA6AD06ECE2E8BEF902FA439
:108B0800930BD5FF7115131A0501B72900200144ED
:108B1800135A0A01372C0020B72C002093890974B6
:108B2800635B7413D424AE241307E1001386D400C6
:108B38004A85EFF0AFA12A8D630F05100359A500F0
:108B48000C253087AA20EFF07FC7631B051083C868
:108B5800440083A60C583087AA20528881471307FF
:108B68006C57EA85EFF0EFEE930D6C5713880C58AD
:108B780065E905C883D70D0003D72900890763086D
:108B8800F706B7250020138705743E23AA2093858E
:108B980005743354F40202A3EF909F990DC559450B
:108BA8001DA0AA2041664D4781467D16A545EFD0F8
:108BB8004FD2B727002023A2A900138807581DE128
:108BC80023102B014545B640264496440649F259E0
:108BD800625AD25A425BB25B225C925C025DF24DF1
:108BE8006161828083D70D0089072391F90083D7BB
:108BF8000D00A29763D1770783A749000357AD00FB
:108C0800930A2400A29798A305049317040103A4C8
:108C18004900C183C20A3E948357AD0083250800EA
:108C280093DA0A01A1831CA003A5490003D60D000D
:108C380056959770FA1FE780806F03D40D00C167BF
:108C4800FD17569442044180E30CF9EC05094209EA
:108C580013590901F1B529450DF423102B01A5B7C6
:108C68006DDC05B71E2181E789473E858280411169
:108C780026C2444122C406C64AC09420D0402A8451
:108C880037E5060089451305C528EF803FF711C968
:108C98003C202547E51793F7F70F6376F702E1477E
:108CA80021A89420D04037E5060089451305852979
:108CB800EF80DFF471FD8947B240224492440249B3
:108CC8003E8541018280372900208356494F8547D8
:108CD8001309494FF5D21A203697C166E3CEE6FC50
:108CE80091659385257031459770FA1FE7800035A7
:108CF800AA84CD4771D1314681459770FA1FE78024
:108D0800A0691E208355090001460147B386E50086
:108D1800C206C182636BF702AE97C207C18319C24C
:108D28002310F90023A004002146A28513854400DE
:108D38009770FA1FE780A05FB727002093874758EE
:108D4800984309EF84C3814785BF504013154700F6
:108D580005072A9636A6054655BF3E871C43F5FFEC
:108D680004C399BF011106CE22CC26CA4AC809E914
:108D78008944F240624426854249D2440561828092
:108D88002AC62A84280036896C845085EFF09FED26
:108D9800AA8465F1E30F09FC3E24F9DB916593850C
:108DA800557031459770FA1FE780402905C53E2464
:108DB80023200500232425015EA1B72700209387DF
:108DC8000759984301E788C36DB73E871C43F5FFF1
:108DD80008C345B7CD4471BFB7270020938787578D
:108DE80098230DE3054798A3058909CDB7260020E8
:108DF800372500209386464C414691451305454842
:108E08006FF05FF601458280B72700202384A74EC4
:108E18008280C167FD176315F5002E856FE04FB896
:108E2800411106C6EFE04FB209C5FD571EA1230147
:108E38000500B2404101828001114AC806CE22CC09
:108E480026CA85472A896392F5044A85EFE08FE2AE
:108E580031E9C16437E606009385F4FF1307E100A2
:108E680089461306C6260545EFE05FEE2A84FD1401
:108E780005C44C444A85EFF0DFF9308722858146E6
:108E8800A685EFF0EFB12A84E5B789476396F50028
:108E98008545EF20200055D9F2406244D24442492A
:108EA80005618280EFE04FD86DB7011126CAB7344B
:108EB80000209384849722CC88343724002013041C
:108EC8008458B72700203727002006CE4AC84EC648
:108ED8002320040023A60758232E075659C11389B7
:108EE800C7589307200C3305F502916593851570D3
:108EF8009309C7571905420541819770FA1FE78002
:108F0800E01390349307200C81453306F60208C01D
:108F180019069770FA1FE78020481C40983481454D
:108F28009386870B7D5563E8E5069306800BB306A9
:108F3800D7020146FD550507B6972320F900BE86DE
:108F48008EA2ACB2ACA22382060005069906E3699C
:108F5800E6FEF95696A399463307D702BA9723A097
:108F6800F9003775050013056579EFD04F903785FF
:108F780005001305A594EF807FCF3775050013050D
:108F8800A56FEF103068F2406244D2444249B249BA
:108F98000145056182802394A6F41386C6F4231044
:108FA8000600232406003106E31BD6FE85059386BA
:108FB800860B95BF411106C622C42A84EFC04FB361
:108FC800EFE02FA0B7270020A383874EB727002004
:108FD80003A5C757EFE0CF9CB7270020238B874E08
:108FE8002244B24037950500130505E441016F108E
:108FF800706193970501C18763D10730B7270020B7
:1090080003C5774E797122D45AC806D626D24AD0DB
:109018004ECE52CC56CA2E8B9770FA1FE780C026C8
:109028002A8429C518219307000B631EF702B72469
:109038000020854793840458DC849C402315010054
:10904800B9E3EF0080759165938535709770FA1FC5
:10905800E780C0FE88C005E99C8491C74C201305B1
:109068008400EFD08FDC2285EF70AFF2B25022542B
:1090780021653345AB0092540259F249624AD24AFB
:10908800424B45618280372A00206146814513059D
:109098000A749770FA1FE780203003494400894713
:1090A80093040A74D289930A0A74631AF904F52599
:1090B8008AA02A2093050A74EF90AFAF3A209E2029
:1090C800162401ED63E3F6001EA40E243A85EFC0D2
:1090D800BFFA2285EFC0FFCF41B763E3F6001EA4B5
:1090E8001E24D945938609740D463A852390FA00C3
:1090F800EFC0FFE38D4571DD1385097465A89947B5
:109108006319F9029305A1002285EFF02FD3AA84F1
:1091180069D1D947639EF40C05092A201379F90F00
:10912800D945938609744A86EFC07FE0CA8555D130
:10913800E1B7A1476318F9009305A1002285EFF074
:109148009F99F1B7A947631AF9060A246C0097801A
:10915800FA1FE780208F2A89630905122A204166B1
:109168009306E10055477D16AD45EFC09FF6C8C090
:10917800AA8625CD834844000358E10030862A207A
:10918800814713070A74CA85EFF0AF8CAA84631F5E
:10919800050C2A2093050A74EF902FBF1DD92A20A9
:1091A80093060A742D46D945EFC07FD81DD1AD4529
:1091B80013050A74EFD06FC729BFB147631BF90CB9
:1091C8000A246C009780FA1FE780C087AA8455CDCF
:1091D8002A2041669306E10059477D16B545EFC040
:1091E8005FEF23A2AA00AA8631E11E24C5447C852C
:1091F8001830D147E30FF7EC5C202A2093850974D7
:109208002380FA003C8523829A002391FA00EF809C
:109218007FC9E30005EC2A20938609740546D945E1
:10922800EFC0FFD0E30705EA8545F9B58348440058
:109238000358E1003E2430862A20A68513070A74C5
:10924800EFF02F81AA841DE12A2093050A74EF907C
:109258000FB9E30005E82A20D94593060A74354674
:10926800EFC0FFCCB545E30605E679B5D94763936A
:10927800F400814403A54A009770FA1FE78000E9CB
:10928800E38904E41E247C85A5B71E2485447C85D7
:1092980085B7B9476318F9009305A1002285EFF057
:1092A800EFA4B5B5C1476318F9009305A10022855D
:1092B800EFF0CFE3A9BDC947631AF900130691007F
:1092C8009305A1002285EFE07F9491B5D947631DEE
:1092D800F9009305A1002285EFE07F84AA84E31AB0
:1092E80005E2A3040100F5B3E147E314F9DE9305B1
:1092F800A1002285EFE0AFF119BD01458280F9CECA
:10930800011152C42E8A854522CC4EC656C206CEBD
:1093180026CA4AC8AA8AB6893284EF10B037D1471C
:109328001DC5B72700203727002083C7C7598346A4
:10933800D759814419E0B684BE8637270020032711
:10934800475993974400BA9763EDD400D547F24044
:109358006244D2444249B249224A924A3E85056152
:1093680082803E89C10703D727FF09C7850493F484
:10937800F40FD9BF31CC9565938525C0130500023C
:109388009770FA1FE78080CB2326A90061D11306C6
:1093980000028145938404049770FA1FE780C0FF98
:1093A8002311990023000900231359010DC43737ED
:1093B80000201C340326C78D2304F900118C832751
:1093C800C90011841180C0AF23A02901814741B78A
:1093D80023260900C1BF23044901FDB785473E85FF
:1093E8008280B727002083C5C759B727002003A765
:1093F800475981476395F500814636858280322337
:10940800BA8619C2E30BA6FE850793F7F70F410743
:10941800D5B7B727002003C6C759B727002003A729
:10942800475981476315F6008146368582802E2389
:10943800BA8681C54C23E38AA5FE850793F7F70F03
:109448004107CDB7B727002083C5F759B7370020A4
:1094580003A7C78D81476395F500814636858280CD
:109468001223BA8619C2E30BA6FE850793F7F70FF6
:109478004107D5B7B727002003C8D759B727002019
:1094880083A7475901476315E800814636858280DE
:10949800B223BE8609CAF2236317A600D04701C6C5
:1094A8003222E305B6FE05071377F70FC107E1BFC0
:1094B800411122C4404526C206C6AA8415C04844A4
:1094C80009C59770FA1FE78060C4484809C59770B6
:1094D800FA1FE780A0C322859770FA1FE78000C3B0
:1094E8002685414681459770FA1FE780E0EAB24039
:1094F8002244FD579CB4924441018280011122CC40
:109508002A842A2106CE2EC6EF10406732462285CD
:109518008145EF00F05622856244F24005616FF004
:109528003FF905C53A21411122C406C62A8411CB48
:10953800DD45EF00F05722852244B24041016FF02B
:109548003FF7B2402244410182808280411126C205
:10955800B1469304C5FFB386D402B73700201387FA
:10956800C78E06C622C4369736276397B602484385
:1095780005C51384C78E9307F00F6305F6001C21F9
:10958800639CC7009770FA1FE78040B8B147B3875C
:10959800F402A29723A20700B24022449244410158
:1095A8008280411122C42E8426C24946AA8481455C
:1095B800228506C69770FA1FE78000DE95CCDC2C62
:1095C80013974700B737002083A7C78DBA979A2308
:1095D8001AA0BA23FE233AA0372700200357A75919
:1095E8005AA09A207AA0BA201AA4DA203AA4FA201B
:1095F8005AA49A241EA87AA4B24022449244410153
:109608008280B727002083C5C759B737002003A831
:10961800C78DB727002003A64759014781476394A0
:10962800E5003E858280142299CA544689CAD42E00
:109638009206C2966315D500850793F7F70F0507BD
:109648001377F70F4106E1BF130600643386C5029E
:1096580093069500AA85379505001305A5526F70E6
:10966800EFFE411122C406C62A840835EF701F9800
:10967800FD571CB4B240224441018280011122CC22
:109688004AC84EC652C456C25AC006CE26CA2A89ED
:10969800AE890144372A0020B72A00201D4B834792
:1096A800DA596365F40463990902B7290020372A57
:1096B8000020930AF00F83C7C9596364F406114464
:1096C800A1442285050442041306F00FCA8541808F
:1096D800EFF0DFE7E31794FEF2406244D2444249D8
:1096E800B249224A924A024B0561828083A74A59AD
:1096F80093144400BE949C208DC3FE20639F2701D1
:1097080063956901AA20EF10604726854E8681453A
:10971800EF0010372685EFF0BFD905041374F40F56
:10972800BDBF83274A5993144400BE949C208DC31F
:109738009C34638F5701FE20639C27012685EFF038
:109748005FF22685D145EF00B0362685EFF05FD66B
:1097580005041374F40F85B741677917630BE502A5
:10976800411122C406C685472A846399F5002285DB
:109778002244B240814541016FF05FF0894763960A
:10978800F5008545EF1000717DD1B24022444101BA
:10979800828082809D456FF07FEEB727002003D539
:1097A800A7598280B727002003C78759011106CE21
:1097B80068876C8685476318F70070009305E10099
:1097C8000545EF502031F24005618280A947631DAD
:1097D800F6029C319821A207D98F1EA1BC31B8216D
:1097E800A207D98F3EA1DC31D821A207D98F5EA16B
:1097F800FC31F821A207D98F7EA19C359825A207B4
:10980800D98F1EA501458280054582809147631E38
:10981800F6009C319821A207D98F1EA1BC31B8212E
:10982800A207D98F3EA10145828005458280938792
:10983800C5FF93960701C1820D47636ED700314774
:10984800B387E702373700201307C78EBA97A8A354
:109858008EA30145828009458280930640203727E0
:109868000020AA8763F4A60093074020F117231D60
:10987800F758B7270020238FB758B7270020238031
:10988800B75A82801905956542054111938535C0FF
:10989800418106C69760FA1FE780407A01C9B24045
:1098A800E95541011773FA1F67008393B2404101DC
:1098B8008280B7270020238F0758B72700207971A7
:1098C8000547238C0758B73700202384E78E4ECEF0
:1098D800B7270020B729002022D426D24AD037241F
:1098E8000020B7240020A380075A37290020B72773
:1098F80000209389F95906D652CC2AC6230E04585B
:10990800A38E0458239D0758232A09582380090049
:10991800EF10402E3245B73700201306000323808E
:10992800A78E373500201305C58E81459770FA1F1D
:10993800E78080A6373A00200345CA911304C4592A
:109948009384D4591309495905CD9565938545C024
:1099580012059760FA1FE780606E37370020232EC4
:10996800A78C19CD0346CA919307CA919C332380CB
:10997800C900814512069CA09770FA1FE780C0A114
:10998800B737002003C507989C209565938555C077
:109998003E951375F50F08A012059760FA1FE7802A
:1099A800E0692320A90051C1102081451206977053
:1099B800FA1FE780609E03270900142081472507C6
:1099C8007D56639EF604EF104043B1473305F50218
:1099D8009565938565C0420541819760FA1FE780C8
:1099E800E065B737002023A2A78E2A8401CDEF10A7
:1099F800C04031463306C502814522859770FA1F5B
:109A0800E78080992254B25092540259F249624A2E
:109A1800379505001305057645616F10A03E85074B
:109A280010A393F7F70F410769BF230004002380B1
:109A3800040051BF41119397050126C206C622C4EE
:109A48004AC0C187AE8463DE070837390020034562
:109A5800098E9770FA1FE78020832A8429C9182164
:109A6800930700096312F7041831CD476319F70605
:109A7800B72600200348250003C5767E3727002037
:109A88008347E75913066400814581461307E75960
:109A9800AA886316D80291C11CA31C2391C7034549
:109AA800098E8545EF70EF872285EF609FCE21658F
:109AB800258DB240224492440249410182800C2201
:109AC800AE9793F5F70F93F7F80F63F4A50093F7A4
:109AD800F50F850693F6F60F090685455DBF092B38
:109AE800E1B793F715000145E9D7EF00305209CDEA
:109AF800B727002083C7E75981CBB737002003C5B4
:109B0800078E8545EF70EF8113C514005DB7854654
:109B18002A8763FFC6029C319021A207D18F1EA11C
:109B28006399D700BC31B421A207D58F3EA1014566
:109B3800828089460145639ED700BC31B421A207C3
:109B4800D58F3EA3DC31D421A207D58F5EA38280B6
:109B5800054582809147631EF6009C319821A20733
:109B6800D98F1EA1BC31B821A207D98F3EA10145CA
:109B78008280054582809147631EF6009C319821BA
:109B8800A207D98F1EA1BC31B821A207D98F3EA147
:109B98000145828005458280A1476318F6029C3101
:109BA8009821A207D98F1EA1BC31B821A207D98F4D
:109BB8003EA1DC31D821A207D98F5EA1FC31F82162
:109BC800A207D98F7EA101458280054582808947F9
:109BD8006319F6009C319821A207D98F1EA101456F
:109BE8008280054582803E2279714ECE06D622D4E7
:109BF80026D24AD01307F007AE896371F7020947E6
:109C08003AC47C86300093F5F50FEF001076B25019
:109C1800225492540259F249456182805A22D94607
:109C28002A89328463F7E6007E2263F4F6006379BA
:109C3800F70023140100300093F5F90F4A85F1B7B6
:109C48000A2202C4EFF01F80AA8435C5EFF07F9B7B
:109C58009C246369F5001146A246CE854A85EF002B
:109C6800906775B7340026869305F00F4A85EFF0A4
:109C78000FE975F1A2471A24DC479AA33A20BAA340
:109C88005A20DAA37A20FAA3DA209AA7DC4495C7E7
:109C980093F4F90F2286A6854A858297C167FD1736
:109CA8002A86E31BF5FA22459947F9451CA144A1E8
:109CB800EFF09F99A9BF094645B7014671BFA9476B
:109CC800631DF6029C319821A207D98F1EA1BC31D1
:109CD800B821A207D98F3EA1DC31D821A207D98F9C
:109CE8005EA1FC31F821A207D98F7EA19C35982569
:109CF800A207D98F1EA501458280054582809C2137
:109D08001CA19C311CB1BC31B821A207D98F3EA13E
:109D1800828023220500D82189476304F70005457E
:109D28008280F6210D47E37CD7FE9C45011106CEC3
:109D380022CC26CA4AC84EC684339023A204D18CAA
:109D4800138644006311D604A033BC23AE892204D1
:109D58005D8C9307C4FFC207C1832A896361F70238
:109D680003A589002311990023108900F1559760F4
:109D7800FA1FE780E0462322A900014531A0228589
:109D8800EFF02FE671FD0545F2406244D2444249A6
:109D9800B24905618280397122DC2E841C204AD8A0
:109DA80006DE26DA4ED619472A89B2856392E70677
:109DB80030202800EFF01FDAAA8405E92884EFF0A4
:109DC8004FE2AA890C3015C937B705002E8613074C
:109DD80067AC34009D454A85EF00702F4E850946D3
:109DE800814579294E85EFF0AFECF2506254268513
:109DF8004259D254B2592161828089477C803C847F
:109E08000A867C813C857C824A85EF001056F1BF2A
:109E180049476398E70232202800EFF0FFD7AA8469
:109E280069F5373500201305C58E5E2599E3814411
:109E38006DBF1830142068253C000146CA85CD2C1A
:109E48006DB75147639EE70032202800EFF01F9856
:109E5800AA8441FD0C3030004A85EFF0DFD871B795
:109E68005947639BE70432202800EFF03F9AAA8401
:109E78002DFD2C844A85EFF0EFDF05C95845348560
:109E88001E23B697C207C1831EA3D5D35C47C5D38B
:109E9800B727002083C7E759D9DBB737002003C5A8
:109EA800078E8545EF60FFC789B789473EC03C8468
:109EB8000A860C307C8289BF0C300A862310010088
:109EC800EF00B04AADB75D71A6C256DA86C6A2C425
:109ED800CAC04EDE52DCAA8A8831AE8432C6EFF0A0
:109EE8004FD3B24501ED8144B64026442685064944
:109EF8009644F259625AD25A61618280230205005F
:109F08002311050083C9040085472A846399F90051
:109F1800B0202808EFF0BFBFAA8405491DA09D47BF
:109F28006391F90418218D47E31FF7FAB020280838
:109F38000549EFF05FC4AA8409E5054681452285F5
:109F480081262285EFF0EFF108243C080147CE86F0
:109F58002686D685F12AE30909F82285EFF04FD540
:109F680061B7CD47639BF90018219147E31DF7F6C8
:109F7800B0202808EFF0BFC545B7D547E395F9F6F7
:109F8800034A05008947E310FAF6B0202808054976
:109F9800EFF0FFD2AA8455F583570102A1EBB884EC
:109FA8001306F0035C44930607FCC206C182636A89
:109FB800D600B085D94663F6C600B486D94563EDA8
:109FC800D5002A20BAA30549EF00503B03560102E9
:109FD800D2852285A92CB5B7AC87BAA3D2A38EA304
:109FE800F6A385471CA0014A0149CDB7014AF9BF2C
:109FF8007971AA8522D426D22221AA84280806D6D5
:10A00800EFF03FD1F24599E53DE185452285EFF036
:10A018006FF975A0BC8415476395E706B8858D4729
:10A0280063F7E7046800EFF09FCD3887DD4763FBEF
:10A03800E7008C86B70717008507100822853EC8F9
:10A04800EF00B0323C87B88591076305F700228599
:10A05800EFF04FF41C8672466C00858B1106228542
:10A0680091CFEFF05FE601C52285EFF0AFF28844AB
:10A0780049DD9760FA1FE780600941BFEFF0BFD163
:10A08800DDB711476389E7001387A7FF42074183BC
:10A09800854663EBE6023147F117B387E7023737A6
:10A0A80000201307C78EBA979A2371D3A8233008C4
:10A0B800A28505204DFDB8849147E318F7F4B25006
:10A0C80022549254456182802C082285FD2445F152
:10A0D800FDB701114AC82A89314526CA06CE22CCC5
:10A0E8002EC6B2849760FA1FE780A01421C1B2453A
:10A0F8009307000A1EA12EA12A84214611058DC0AE
:10A10800A6859760FA1FE7808022A2854A85EF60BE
:10A118002FED0145F2406244D244424905618280F4
:10A1280081459760FA1FE7802027C5B70545DDB749
:10A13800797126D2AA841305000206D622D42ECE1F
:10A1480032CC36CA3AC83EC69760FA1FE780600E1E
:10A1580029C56246F2454247D246B2472A841305CA
:10A1680020FA08A010B02EA058A054B013058400FF
:10A17800614691CFBE859760FA1FE780401BA28594
:10A188002254B2502685925445616F606FE581452F
:10A198009760FA1FE7804020DDB7B25022549254EE
:10A1A800456182805845797122D406D62A84AE86C4
:10A1B8002DC73E23FC85930720066397F504B72730
:10A1C800002003D6A7597E236373F600B28713F6DF
:10A1D800F70F2E2B1C2B8D8F93F7F70F81E589072F
:10A1E80093F7F70FB297FD17B3C7C702FC863E2057
:10A1F8006E200824FC8401473C080146EFF05FF319
:10A20800B250225445618280582FB737002083A767
:10A21800C78D1207BA97FE23D1BF2EC619468145AE
:10A2280028089760FA1FE7802017B246C9B77971E6
:10A2380022D406D626D22A8499CD8147014793068F
:10A2480000062E866E200824EFF09FEEB2502254AE
:10A25800925445618280B284280059469760FA1F5B
:10A26800E7808013648499E43E2048446C007C8530
:10A27800EFF02FB33C000147930600060146D9B71B
:10A28800797106D6814791E93E21584570867C84CC
:10A298003C0001C73E237C853C002E866E210825A4
:10A2A800014793060006EFF0BFE8B250456182808F
:10A2B800411122C406C61C2111472A846392E70271
:10A2C8002E866E21082581470147CD46EFF05FE6CF
:10A2D80049466E202244B240154541016FF00FA750
:10A2E80013F7B70F89466317D7000146EFF03FF41D
:10A2F8005146C5B70D476398E7002244B24001466E
:10A3080041016FF0FFF7B2402244410182809A2157
:10A31800B146B737002071173307D7029387C78E26
:10A32800BA97D84301EBD841AAA70145D8C3BA21A7
:10A338009AA7828059458280797122D4404526D2D5
:10A348004AD006D6AA842E8931C4484419C59760D4
:10A35800FA1FE780A0DB232604001E20EE208824B5
:10A368007C853E200147930640067C861E244A864B
:10A378007C871C483EC8BE207C843C00EFF05FDB35
:10A38800A30E240123280400B250225492540259E7
:10A39800456182802800314681459760FA1FE78031
:10A3A800A0FFBE20EE2088247C8401473C00930651
:10A3B80040064A86EFF0DFD7C1BF797152CC2A8AAE
:10A3C8008A2126D206D622D44AD04ECE56CAAE8488
:10A3D800EFF02F8119E1854795A84045AA8965DCEA
:10A3E8007E21E39A47FF1E2463890710542CB73A4D
:10A3F800002003A7CA8D9206FD173697C2077A2355
:10A40800C1831EA46316F70093053006EFF09FD9A9
:10A418005C48A5EFC840034915001C21220933698F
:10A42800F900BE2013072900631CF702F95597604D
:10A43800FA1FE780E0DAC8C02391240103C5890028
:10A448002686D285EFF0FFC8814721E1B250225419
:10A4580092540259F249624AD24A3E854561828045
:10A468009565938515C04A859760FA1FE78000BDFA
:10A4780048C8C840231C2401F9559760FA1FE78093
:10A4880020D6BE20C8C0F917BEA0484825CDB220A6
:10A49800362C1E2C3308D60063C80707582C83A710
:10A4A800CA8D95451207BA97BE2363C90705CC40E4
:10A4B80036959760FA1FE78080E73A2CBE20BA9756
:10A4C800C2071A2CC1833EACE397E7F003D72900F3
:10A4D80003C58900300078845848D2857C853AC6FF
:10A4E800EFF03FBF11C548489760FA1FE78000C2E8
:10A4F800232A0400232C0400F9BD99454E85EFE07A
:10A50800FFFFD1BDA545DDBF9145CDBFBA2171CBB8
:10A51800B727002083D6A759ED4763E5E60C01115C
:10A5280022CC2E8426CAAA844840914506CE97603C
:10A53800FA1FE780E0CA3E20AA861CA13E20A1831C
:10A548001CB11E203CA11E20A1833CB13220C16752
:10A55800F9171106420641826394F4042AC431456E
:10A5680032C69760FA1FE780C0CCAA85CD471DC1C7
:10A57800930700F91CA13246F957A2463EA1894724
:10A588005CA1B737002072A114C503C5078EEF6020
:10A598002FA58147F2406244D2443E8505618280FE
:10A5A80081452685EF406060AA8711E9B72600201B
:10A5B80003C7E65965D37D17238FE658E1BF0947DE
:10A5C8006304E5021D476303E50249476302E502A8
:10A5D8007D47E311E5FCB726002003C7E65981470C
:10A5E800D1BFED473E858280D1476DB791475DB7B2
:10A5F80089474DB701114AC831471309C5FF3307C9
:10A60800E902B737002026CA9384C78E06CE22CC2B
:10A61800BA94D84029C71384C78EB727002083C6A9
:10A62800E759854795C668849E24AA242C003AC613
:10A638007C85EFF0BFED11C5C8409760FA1FE78031
:10A64800E0ACB147B307F902A29723A207008547F8
:10A65800F2406244D24442493E8505618280814786
:10A66800C5BF797126D24445372700204AD0FE203D
:10A678000359A75952CC06D622D44ECE56CA2A8A96
:10A6880063F327013E89BA284209135909019E2814
:10A6980035CF998F4A8463D52701139407014180E8
:10A6A80089452285EFF00F9EAA89CD4A31C5BE2083
:10A6B8002AC660857C84BE2899EB9E2893092500CC
:10A6C8001CA19E28A1831CB1637424058228BE287E
:10A6D800CC4422864E85BE959760FA1FE78020C538
:10A6E80003556A002C00EFF07FE2AA8A15C54E8553
:10A6F8009760FA1FE78080A1B25022545685925481
:10A708000259F249624AD24A45618280890759B79B
:10A7180079144204418065BFBA289E203A94FD17F7
:10A72800C20742049A28C18341809EA0A2A86376EA
:10A73800E400F9F3FD57DCBCC1B781455285EFF061
:10A74800BFBF5DBF79714AD03729002052CC034A78
:10A75800195A22D456CA5AC85EC662C406D626D228
:10A768004ECE5284B72A0020054B930BF00F372C9E
:10A77800002083A74A5993144400BE9483C9040057
:10A78800639B6907DC44A5CBD84735C79A2329CBF7
:10A79800B727002083C7E75999CF2685EFF07FECCC
:10A7A800AA8515E9B727002083C7D759050463513F
:10A7B800F402A300895AB25022544E859254025989
:10A7C800F249624AD24A424BB24B224C45618280DE
:10A7D800A300095ACDB72685EFF01FB68149E1BF1E
:10A7E800DC3F639A7701930520062685EFF09F9B4F
:10A7F800DC44A38E07008347DC5905041374F40F67
:10A808006363F4000144E31644F7C9BF41111545D9
:10A8180006C6EFF03FDE09C50545B240410182801A
:10A828001945EFF03FDD6DF91145EFF0BFDC6DF52F
:10A838001D45EFF03FDC6DF1B727002083C7D759DE
:10A84800E9DFB24041016FF0FFEF9E210D47F1179C
:10A85800C207C1836363F706DC41A5C3411122C463
:10A868002E84854526C206C6AA842D2529C9268593
:10A878003D2BC167F917638FF40009ED3E2099CB92
:10A88800162019476393E604372700200357A75972
:10A8980063FDE702B727002083C7E759A28526850D
:10A8A80099C72244B240924441016FF03FC6224406
:10A8B800B240924441016FF09FA5094582805145FD
:10A8C800B24022449244410182806D45D5BF39711E
:10A8D80026DA4ED6AA84AE895D4589454AD806DE71
:10A8E80022DC328936C63AC4EFE0DFF935C12247A7
:10A8F8002A84014511C7B24613054400B68502975C
:10A908009357850023003401A30024013CB09547E8
:10A91800FC84B727002083C7E75928A01105E885DC
:10A9280022CE2C08268595C3EFF05FBEAA8411C5F8
:10A9380022859750FA1FE780607DF2506254268581
:10A948004259D254B25921618280EFF05F9CF9BF1D
:10A95800CD44E5B7797126D24AD052CC56CA06D62C
:10A96800BA8A22D44ECE19472E89B284368A639584
:10A97800E5062A220944EFE0DFA62AC635C55C456C
:10A9880083596500BE239EA0B247B73600201547FD
:10A998002380570103C6868EBAA3130716001377C0
:10A9A800F70F2384E68ED0A301E705472384E68EBC
:10A9B80051476317E9001547BAA0DC479A249AA7BC
:10A9C8005287A686CA854E85EFF07FF02A843245E5
:10A9D80015C4EFE0FFAD09A842867400BE85AA89B8
:10A9E800EFE0FF912A844DD12285B250225492542F
:10A9F8000259F249624AD24A45618280F945EFE03C
:10AA0800BFC4DDB79E211CA19E21A1831CB1BE211C
:10AA18003CA1BE21A1833CB1114582809E211CA18D
:10AA28009E21A1831CB1BE213CA1BE21A1833CB1C2
:10AA3800DE215CA1DE21A1835CB1FE217CA1FE2187
:10AA4800A1837CB1214582809E211CA19E21A183E6
:10AA58001CB1BE213CA1BE21A1833CB1DE215CA179
:10AA6800DE21A1835CB1FE217CA1FE21A1837CB102
:10AA78009E251CA59E25A1831CB5294582809A2167
:10AA88008546AA8718A19A21218318B19A216319AA
:10AA9800D700BA2138A1BA21218338B11145828063
:10AAA8000945631DA700BA211945B8A3BA21218316
:10AAB800B8B3DA21D8A3DA212183D8B382809E21C2
:10AAC8001CA19E21A1831CB1BE213CA1BE21A18352
:10AAD8003CB111458280797126D24AD04ECEB284DB
:10AAE8002A89AE8929468145480022D406D636846B
:10AAF8009760FA1FE780408A64868DE43E207C8256
:10AB0800B727002083D7A7597C845C4481CFD42FF2
:10AB1800373700200327C78D92069E2736973A239A
:10AB28007C85788337B705004A85130707A5540045
:10AB380013F6F90FD545EFF09FD92A8911C195E091
:10AB480085471CA023020400014681452285EFF0B9
:10AB58000FEEB25022544A8592540259F249456187
:10AB680082802285EFE0DF94EDB737B70500B28623
:10AB7800130767A82E8685456FF07FD50111688772
:10AB8800B7B605004165700001489307F00F0D47FF
:10AB98009386C6A099457D1506CEEFF0BFDBF2403F
:10ABA80005618280B7B60500B28701482E86114735
:10ABB800938646A2C9456FF0FFD9011122CC3734DC
:10ABC80000201304449226CA4AC84EC606CE2A89D3
:10ABD800AE89930404031C4081C7CE854A858297B9
:10ABE8001104E31A94FEF2406244D2444249B24945
:10ABF80005618280B727002003C5D77E411122C492
:10AC080037340020937735001304849709811CB4E6
:10AC1800AA9706C626C21CA4ADCB1305C00333856C
:10AC2800A702A5658505B73400209750FA1FE7806D
:10AC3800E04010249307C00381453306F60223A0A1
:10AC4800A4929750FA1FE780207583A704921424D2
:10AC5800014789077D566341D7022244B240924496
:10AC6800373500201306000381451305459241013D
:10AC78001753FA1F6700437292A32381070023A585
:10AC8800070205079387C703F9B7B24022449244E5
:10AC980041018280011122CC2EC632C406CE2A84FC
:10ACA8009760FA1FE780C0DE2246B24511E9C16706
:10ACB800F9176303F4005145F2406244056182804C
:10ACC80054555C218DC213F7270141456314A70031
:10ACD80015457DF2C18B3D45E5D3BC2E0145E3FD0D
:10ACE800B7FC3145D1BFC18B0145F9F71545E9B727
:10ACF800797126D24AD0B7340020416922D44ECE89
:10AD080052CC56CA5AC806D6AA8901449384849755
:10AD1800373A0020930AC0037D19054B9C246364CD
:10AD2800F400014525A8B307540303270A92BA97EC
:10AD3800BA236316270105041374F40FC5B7C83383
:10AD4800300093856700EF0011631946CE8528000F
:10AD58009750FA1FE780A06EE31F65FDB25022549A
:10AD680092540259F249624AD24A424B4561828062
:10AD7800B737002083C50798C166B737002003A7F7
:10AD88000792FD1681476395F5000146328582805A
:10AD9800035827003A866306D80003480700E307EC
:10ADA800A8FE850793F7F70F1307C703E9BF4111FB
:10ADB80006C69760FA1FE780A0CD09C54A29B240A8
:10ADC800410182800145E5BFB737002083C6079857
:10ADD800B737002003A707920145814711076393FE
:10ADE800F6008280102301C605051375F50F850747
:10ADF80093F7F70F1307C703DDB7B737002003C56D
:10AE080007988280373700209306479281471307B7
:10AE1800479231468C4291E58A07BA9788C3014523
:10AE2800828085079106E397C7FE4D4582804111D0
:10AE380006C622C49760FA1FE78080C50DCD2A8414
:10AE48002A218545EFF07FD7485409C59750FA1F46
:10AE5800E780C02B22851306C00381459750FA1F4F
:10AE6800E7808053FD573EA0230204000145B2400D
:10AE78002244410182800945DDBF411106C6976021
:10AE8800FA1FE780E0C009C54825B2404101828029
:10AE98000145E5BFC167F9176305F502411122C4F1
:10AEA80006C62E849760FA1FE78080BEAA870145F0
:10AEB80089C7C823698C33358000B24022444101D8
:10AEC800828005458280011106CE2EC69760FA1F42
:10AED800E78000BC854701C95A29B2458547630404
:10AEE800B7004EA98147F2403E850561828029CD91
:10AEF80001114AC84EC637390020C16922CC26CA7A
:10AF080052C456C206CE0144AA8413098997373A17
:10AF18000020930AC003FD1983478900634BF4009E
:10AF2800F2406244D2444249B249224A924A0561F7
:10AF380082803305540383270A923E953E2163831A
:10AF4800370182940504C9BF8280B737002003C641
:10AF58000798B737002083A70792C166014589077C
:10AF68000147FD1691456313E600828003D8070068
:10AF78006309D80003C8A7006315B8000505137551
:10AF8800F50F05071377F70F9387C703E9BFB7379F
:10AF9800002003C60798B737002083A60792014709
:10AFA800814791066310E602858393C7F7FFC207BE
:10AFB800C18305456362E50285473395A7004205CD
:10AFC800418182808C2299C1CE36CD8F05071377B7
:10AFD800F70F9386C603F9B793F61700F1FE050538
:10AFE80085831375F50FF9B7797156CAAA8A2E8524
:10AFF80026D24AD04ECE52CC5AC85EC662C406D6B5
:10B0080022D4AE84328B368CBA8B3E8AC28946896A
:10B018009760FA1FE780C0A73DED41657D159760F1
:10B02800FA1FE780E0A62A84554531C81946DE850F
:10B0380013056400A30284019750FA1FE780202FAC
:10B048008357010326A0230264013EA883574103C6
:10B0580023005401232604025EA823064401231773
:10B06800340123182401EFF09FF20AB8232A0402BE
:10B078002685232C04028145EFF03FB40145B250E8
:10B08800225492540259F249624AD24A424BB24B74
:10B09800224C456182804545DDB7B737002083C61D
:10B0A8000798B737002003A7079281476395F600F2
:10B0B80041657D1582803A861307C703835547FF8C
:10B0C8006394A5002A228280850793F7F70FF9BFBA
:10B0D800B737002003C80798B737002083A6079220
:10B0E800416601477D16954811436314E800014500
:10B0F8008280BE223685638EC702CC5A9DC9BC3178
:10B10800AC2189CD938597FD93F5F50FE372B3FED6
:10B118009387D7FA93F7D70F89EF82809385F7FD46
:10B1280093F5F50FE3F6B8FC9387D7FA93F7D70FA3
:10B13800E1D305071377F70F9386C6037DB7B737B3
:10B14800002083C507984166B737002003A70792F8
:10B158007D16814725486394F50001458280362392
:10B168003A85638BC600545B81CAB4329386E6FD88
:10B1780093F6F60FE374D8FE850793F7F70F1307D6
:10B18800C703D1BF011122CC2A84494506CEEF80DE
:10B19800EFB21DC12AC622859760FA1FE780408F4B
:10B1A80001CD6244B737002032460E39F24003C55C
:10B1B800B79705616F50DFB4F24062440561828041
:10B1C80039714ED652D4AE892A8A93053005414545
:10B1D80026DA4AD856D206DE22DC32C63689BA8A40
:10B1E8009750FA1FE78080E5CD4429C92A8489440D
:10B1F8006381090432468145F08241469750FA1F1F
:10B20800E78080195686CE8522859750FA1FE780F9
:10B2180000122146630E0902CA8528089750FA1FB2
:10B22800E780E010A28650082C085285EF30100EF7
:10B23800AA8422859750FA1FE78040EDF2506254A5
:10B2480026854259D254B259225A925A2161828093
:10B25800814528089750FA1FE7800014E1B741118B
:10B2680022C4405926C206C6AA8429CC085409C556
:10B278009750FA1FE78080E9285809C59750FA1FA8
:10B28800E780C0E8685809C59750FA1FE78000E8CA
:10B29800285C09C59750FA1FE78040E7685C09C534
:10B2A8009750FA1FE78080E60325040809C59750E0
:10B2B800FA1FE780A0E522859750FA1FE78000E58E
:10B2C80023AA04022244B73700208E38B2409244A1
:10B2D80003C5B79741016F50BFCA411126C206C6C0
:10B2E80022C4AE849750FA1FE780807A29C14C594E
:10B2F8002A8495CD83A8C50703A88507FC59B859A2
:10B30800F4219221AC212685EF804FA32285EFF00E
:10B318001FF5EFF0DFE201CD2244B7370020B2403D
:10B32800924403C5B797854541016F508FFFB240DE
:10B338002244924441018280011122CC06CE2A8403
:10B348002EC69750FA1FE780A0745C5989CF9E23B8
:10B35800B245639A870085476397F5006244F240D7
:10B3680005616FF0DFEFF2406244056182804111B0
:10B3780006C622C426C2EFF0BFD529C14059AA8407
:10B3880015CC3C209DC7B737002083A7879589C770
:10B39800DC4399C32285829738309307F002631FF4
:10B3A800F7002244AA20B2409244814541016FF03F
:10B3B800DFF2B737002083A74795D1BFB2402244B8
:10B3C800924441018280411126C24AC006C622C465
:10B3D800AA842E899750FA1FE780806B05CD4059C3
:10B3E80055C41E206394970A3C30130710026395D6
:10B3F800E7083C20ADCF7C5403270408DE2B15E377
:10B4080013F7170019CF18545A23058B19CB930734
:10B4180020023CB0B2402244924402490545410111
:10B42800828013F7270001CB18545A23098B01C7D0
:10B4380093074002F9BF918B81CB1C54DE23918B7B
:10B4480081C793076002F1B7B737002083A78795B4
:10B45800F1D3DC43E1D32285829738309307F00299
:10B468008145E319F7FA2685EFF03FE765B7B73767
:10B47800002083A74795E9BF1307A0026398E70058
:10B488006304090013092003CA85F1BF631C09007E
:10B4980026859750FA1FE780A05F09C55C2193E7CE
:10B4A80007015CA1A6854A85EF705FA4A5B77971ED
:10B4B80026D29947EC85AA842E858D4522D406D6B6
:10B4C80032C636C4FC84EFE0EFBB2ACE4D441DC122
:10B4D8003246A246AA85328582962A8419E52C0826
:10B4E8002685EFF08FB62A8411C572459750FA1F4A
:10B4F800E780C0C12685EFF0FFC82285B2502254EC
:10B508009254456182804111B7D6050022C42E8627
:10B518002E84938686C8894506C626C24AC02A89CB
:10B52800EFF0FFF80C20AA844A85EFF01FDBB24049
:10B53800224426850249924441018280B73700207F
:10B5480083A7479585CB9C4395C71D71A2CC86CE12
:10B55800984110082A843AC8D84185453ACA829742
:10B5680011C548862A206C00EFF0FFF9F6406644C2
:10B57800256182808280AE8711CD785501CF142352
:10B5880094A1143394B1342BB4A1142F584BB4B1F3
:10B59800D8C18280414681453E851753FA1F67000E
:10B5A800A3DFB737002083A7879591C703A3870038
:10B5B800630303000283094582803737002003278D
:10B5C80007B51DC75843AA8705450DC703A5070832
:10B5D800411106C6930605021306050C93050506D8
:10B5E800130505040297B2401375F50F41018280D7
:10B5F8000545828082804DC9357122CD2A840A2171
:10B6080026CB4AC94EC756C306CF52C55AC1DEDE3D
:10B61800B68AB2892E899750FA1FE7806047AA84B4
:10B6280031C50C182285EFF01FF53C20138A640001
:10B63800A9CBEF700FE62A8B014583CB5400EF703E
:10B648004FE3AA840C100818EF10204708542C1058
:10B65800EF104047D288268A56C05E88D2875A871C
:10B6680014103010CE854A85EF20606EFA406A4487
:10B67800DA444A49BA492A4A9A4A0A4BF65B0D61A2
:10B688008280EF700FE1AA8B014503CB5400EF7065
:10B698004FDE2ACE08540C10EF1020422C10081848
:10B6A800EF104042F2484DBF8280C14719C9145576
:10B6B800C14781CA785511C7BC32BD4663F3F6004D
:10B6C8001C2F3E858280894779C9F1C9411106C678
:10B6D80022C426C21C312E849CA13C219CB13C3141
:10B6E800BCA15C21BCB15C31858B93968700DE21BF
:10B6F80093F7F7EFD58FDEA1543193F7F7DFA20662
:10B7080093F60620DD8ED6A1583193F6F6BF2207B0
:10B7180013770740558FDAA15C31FD769386F67F63
:10B728008D87858B758FAE07D98FDEA17421F99B24
:10B73800858ADD8ED6A178219377270013F7D6FF67
:10B748005D8FDAA17C2193F647009377B7FFD58FF9
:10B75800DEA17821DD9B4D45218BD98FDEA1EF70CD
:10B76800FFD5AA845145EF707FD5383093F4F40F94
:10B77800C947636097021375F50F636CE5001420E1
:10B788001147E1476367D700143005476363D70063
:10B798008147B240224492443E85410182803E85E1
:10B7A800828015C1AA8709458DC141112E85414660
:10B7B8009385170006C69750FA1FE78040B7B24036
:10B7C80001454101828009458280828089470DC5F3
:10B7D80085C5411106C61831AE87194698A193054B
:10B7E8002500138517009750FA1FE78040B4B24030
:10B7F80081473E85410182803E85828015C1AA87A6
:10B8080009458DC141112E8541469385170006C60D
:10B818009750FA1FE780A0B1B240014541018280EC
:10B82800094582808280894705C99DC5411106C6A0
:10B8380038211431AE872207558F9AA121469305E6
:10B848003500138527009750FA1FE78040AEB240B5
:10B8580081473E85410182803E85828015C1AA8745
:10B8680009458DC141112E8541469385170006C6AD
:10B878009750FA1FE780A0ABB24001454101828092
:10B88800094582808280894709C981C91831BD4626
:10B89800E14763E4E60098A181473E85828015C1AF
:10B8A800AA8709458DC141112E8541469385170008
:10B8B80006C69750FA1FE78080A7B24001454101AC
:10B8C800828009458280828015C1AA8709458DC179
:10B8D80041112E8541469385170006C69750FA1FD9
:10B8E800E780E0A4B2400145410182800945828099
:10B8F80082801DC1AA87094595C141112E8513066D
:10B9080000049385170006C69750FA1FE78020A207
:10B91800B24001454101828009458280828015C17B
:10B92800AA8709458DC141112E8541469385170087
:10B9380006C69750FA1FE780809FB2400145410133
:10B9480082800945828082801D71A2CC2A840845A4
:10B9580086CEA6CA23060100042135479387F4FF43
:10B9680093F7F70F6364F70C37E706008A071307A6
:10B9780007C5BA979C4382870C08EFF0DFD4C94704
:10B988006310F50299475C862A206C00EFF0BFB778
:10B99800F6406644D644256182800C08EFF01FEC1F
:10B9A80031C51C86F5F32A20EFF0CFFDD5B70C087A
:10B9B800EFF0FFEEF5B70C08EFF0FFECD5B70C0889
:10B9C800EFF03FDEF1BF0C08EFF0FFE5D1BF0C0848
:10B9D800EFF0DFE2F1B70C08EFF05FDFD1B70C084A
:10B9E800EFF09FEE75BF1C312308F1002A20975015
:10B9F800FA1FE780E009A14705C15825631AF70235
:10BA0800B737002003A787959D4719C7184309C76B
:10BA18001008A6850297AA875C8661B70C08EFF024
:10BA28005FEDBDBF0C08EFF09FEF9DBF9D47A1BF25
:10BA3800B737002003A74795C1BF011122CC06CE16
:10BA480026CA4AC84EC61821930720092A846313B8
:10BA5800F7121C3139476393E70A562109676107D2
:10BA680081476391E610B739002003A58996CE84F3
:10BA7800630A050E0C4403C90500631E09001C2156
:10BA880085052146A9CF29059750FA1FE780208A06
:10BA980083A78496B5C349459740FA1FE780607924
:10BAA8002A840DC5930710FC1CA1A300250183A5BA
:10BAB80084960905414689059750FA1FE780208733
:10BAC80083A78496A2858833EF409FD103A58496E7
:10BAD8009740FA1FE780806323A4049631A80905DC
:10BAE8009750FA1FE780A084EF30000205494DF116
:10BAF80083A78996238027018547ADA01307E00314
:10BB08006398E70838219547631CF7024A21EFF04C
:10BB1800CFB69147E312F5FEB737002083A74795C4
:10BB2800E1DF03A38700E30903FC72244A2093059D
:10BB380064006244F240D2444249B249056102833A
:10BB4800A147631CF7006C204A206244F240D244AB
:10BB58004249B24905616FF01F8793060003814788
:10BB6800E303D7FEF2406244D2444249B2493E85DB
:10BB7800056182809306000A8147E315D7FEEFF03E
:10BB8800BFDC084435D99740FA1FE7802058ADB785
:10BB98008147C9BF011126CA06CE22CC89440DCDE2
:10BBA80085CDAA842E8468008D45EF601FE01C8730
:10BBB8002685228693F7F70393E707046C005C87D2
:10BBC800EF20E00FAA8409E90D466C001305340044
:10BBD8009740FA1FE780A075F24062442685D24458
:10BBE800056182805D714EDE86C6A2C4A6C2CAC047
:10BBF80052DC56DA5AD85ED6894945CD5DCA138BD0
:10BC08004500420B135B0B01AE8A2A8A9305300567
:10BC18005A85B2849740FA1FE78040422A84CD496A
:10BC280049C9EF70EF882A895686D285935A8900C8
:10BC3800135A0901937BF90F1305440093FAFA0F7D
:10BC4800137AFA0F135989019750FA1FE780A083D6
:10BC5800A301740123015401A3004401230024011A
:10BC6800EF706F84AA85414608089750FA1FE7804D
:10BC78008081214734005A86A2850808EF20A02A2F
:10BC8800AA891DE121462C0023807401A380540158
:10BC980023814401A3812401138544009740FA1F9E
:10BCA800E780607EEF708F8122859740FA1FE780DA
:10BCB800E045B64026444E8596440649F259625AF4
:10BCC800D25A425BB25B6161828001114AC82A89FB
:10BCD8002E8506CE22CC26CA2EC69750FA1FE7809C
:10BCE80020DB55CD405955CC5C300947B24593F619
:10BCF800B70F6386E60011474945639DE7061E2096
:10BD080009456399B706930484004146CA85268588
:10BD18009740FA1FE780A0614146CA851305840150
:10BD28009740FA1FE780A060383085469307F7FEF2
:10BD380093F7F70F63E6F6041306C4033285C1458B
:10BD480032C6EF609FC632469306C402A685228596
:10BD5800EFF07F8A3C2089CB22856244F240D244AE
:10BD6800424905616F00107A3830C947E306F7FE8B
:10BD78003CB00145F2406244D244424905618280A8
:10BD8800930710050145E317F7FE3C20E5D7228508
:10BD98006244F240D244424905616F00F07C094593
:10BDA800D1BF4945C1BF39C9011126CA06CE22CC27
:10BDB800AA8409459DCD0D4628002E848D059740FF
:10BDC800FA1FE780C0561C8570002C0093F7F70314
:10BDD80093E7070426855C85EF10706E19E90D4618
:10BDE800A28568009740FA1FE78060657D153335A6
:10BDF800A000F2406244D2440561828009458280F5
:10BE0800011152C42A8A32854EC656C25AC006CE7D
:10BE180022CC26CA4AC82E8BB28AB6899750FA1FF6
:10BE2800E78000C709ED8944F2406244268542490B
:10BE3800D244B249224A924A024B056182805C5937
:10BE48002A89C544F5F34D45EF704FE71374F50F94
:10BE58005145EF70AFE6E38809FC83C78901E3E445
:10BE680087FC1375F50FE360F5FC930530051305A2
:10BE780040089740FA1FE780601C232AA9022A84F9
:10BE8800CD445DD11306400881459740FA1FE780ED
:10BE9800A050A301040023014401230264012310DC
:10BEA80054012326340723240402A30204008144F6
:10BEB800E30C0AF62285EF00305FAA8435D54A855F
:10BEC800EFF0EFB995B7397122DC06DE26DA4AD8E9
:10BED8004ED652D456D25AD05ECE62CC66CA0944E7
:10BEE800630D0610630B0710AA8B3A89368BB28A4A
:10BEF8002E8C9750FA1FE780A0B92A8A5144630E06
:10BF0800050E9305300541459740FA1FE780001359
:10BF1800AA894D447DC18344190083472900A2049E
:10BF2800C207BE9483470900BE9483473900E207DD
:10BF3800BE9483278A0263E697007D570944639974
:10BF4800E70A63070C0083474A000544898BCDC381
:10BF5800930C4B00214681450A85C20C9740FA1F75
:10BF6800E780804393DC0C01930530056685974094
:10BF7800FA1FE780A00C2A8C4D443DC95A86D68505
:10BF880011059740FA1FE78000501146CA8562855F
:10BF98009740FA1FE780204F414693058A014E8556
:10BFA8009740FA1FE780204E21478A866686E285F9
:10BFB8004E85EF1050772A841DE521468A85280092
:10BFC8009740FA1FE780204C214693054900280036
:10BFD8009740FA1FE780A0468547631EF502A685AD
:10BFE8005E85EF707F8462859740FA1FE7800012B4
:10BFF8004E859740FA1FE78060112285F2506254FF
:10C00800D2544259B259225A925A025BF24B624CAC
:10C01800D24C216182800544F9B779719397050163
:10C0280022D406D626D24AD04ECEC1872E8463D5D6
:10C038000704B734002093848497A8309740FA1FE8
:10C04800E78080242AC609CDEFF03F9FB24511E56D
:10C05800A8209307F00F631EF5002E85EF406FF3BD
:10C068002165218DB250225492540259F2494561FA
:10C078008280EF40EFF6EDB793F7150091C7EFF028
:10C088000FAF13451400F9BFA1E10145E1BF8504D5
:10C0980093F4F40FEFE07FD6E3F9A4FE339599000B
:10C0A8001319050113590901B3772401EDD34A8502
:10C0B800EFE0BFFEC167FD176305F500DD45EFF052
:10C0C800CFA13345240179BF85448549E1B7B73706
:10C0D800002023A40796B737002023AC079437C75E
:10C0E8000500B73700201307876623AA0794B737D8
:10C0F800002023A6E79637C705009387C79613073E
:10C10800673BD8C337B705001307871C98C737D7CD
:10C118000500B73700201307E74E23AEE79437D75B
:10C1280005009387C7951307C709D8C337D70500F4
:10C138001307C73398C78280B737002083C7C797CC
:10C14800918B89C7B73700209387C7953737002069
:10C15800232AF79401458280011106CE2AC6EFF002
:10C168001FF73245B73700209945A38DA796EFD022
:10C178000FECF24037B505001305053405616FE093
:10C188007FC81C5581C7A1473E858280011122CCFA
:10C1980026CA2A84AE84130500049305300506CE0A
:10C1A8009740FA1FE78080E908D475C11306000498
:10C1B800A6859740FA1FE780801778543C2B93F6A2
:10C1C8008700F5CA1454B422A18AF5C68327040847
:10C1D800DDEF93053005130500109740FA1FE7803F
:10C1E800E0E52320A4088D4745C5A3020400785440
:10C1F8009C30143391EB91EABC20918BC5E33C2B26
:10C20800918BC9EF854701A881C6214758B089C7D6
:10C218005C3093E707015CB06C54BC29858B99CBE3
:10C228001C540547BC238D8B6396E7007C2093E75D
:10C2380017007CA08327040889C77C2093E7870020
:10C248007CA05C300547639AE70A93048400414662
:10C25800814526859740FA1FE780001441468145AD
:10C26800130584019740FA1FE78000131306C403DF
:10C278003285C14532C6EF604FF383270408324642
:10C28800B9CF2285EF00502E9307000525C5A14799
:10C29800F2406244D2443E85056182809C2014238A
:10C2A8001547B387E70237E70600130747CABA9767
:10C2B800B6979C238DB7943089C6143399C2E14749
:10C2C80099BFB420D58F918B95DF9C2014231547F7
:10C2D800B387E70237E70600130787C8C9BF930685
:10C2E800C402A6852285EFF00FB12285EF009021C8
:10C2F800C14751FD3CB0814761BF13F787012DCF7E
:10C30800C18B930484004146A9C7890526859740B7
:10C31800FA1FE780C0014146814513058401974013
:10C32800FA1FE78060077C201306C403328593E771
:10C3380047007CA0C14532C6EF602FE78327040879
:10C34800324699CF2285EF003022930720055DD130
:10C358003DBF814526859740FA1FE780E00365BF0A
:10C368009306C402A6852285EFF0EFA82285EF0088
:10C378007019CD4741D121BF09478545638AE70038
:10C38800114789456386E70019476396E7008D459D
:10C398000A20EF708FB37C2093E747007CA08327A7
:10C3A800040881C793071005B1B7C547A1B73C2159
:10C3B800638B0722797122D406D626D24AD03C3123
:10C3C800130750052A84639DE70603497500130681
:10C3D800C503C14593573900AA973285842732C6C9
:10C3E800EF60AFDCB737002083A707B5A1C79C472C
:10C3F800B1C30325040893767900B3D6D4403246F6
:10C40800858A93050504180893E6060813050508A8
:10C4180082971375F50F19ED41460C081305C402F0
:10C428009740FA1FE780A0F02285EF00B00D930730
:10C4380060053CB0B2502254925402594561828042
:10C44800130710026392E7021C5503270508DE2331
:10C4580061E313F707104DCF78555A2B1377071060
:10C4680045CB930770023CB03C30130770026397CA
:10C47800E70C3C5885E39305300571459740FA1F52
:10C48800E780C0BB28D819C5714681459740FA1F77
:10C49800E78080F02458B1C4BC2C89E72285EFF0EE
:10C4A800CFA0A8AC2858814541469740FA1FE7809D
:10C4B800A0EE28583D472C2D9387F5FF93F7F70FEB
:10C4C8006364F700EF606FCEEF408FCB3C58A14517
:10C4D8008AAB13852701EF604FCD2C580A20EF0057
:10C4E800B031930780020A203CB09740FA1FE780DA
:10C4F800205A414609C57E2513D617003E96B73700
:10C50800002003C5B79706068545EF406FFF1DB7A6
:10C5180013F7072009CB78545A2B1377072001C744
:10C528009307900289B793F707409DDF7C54DE2B71
:10C5380093F7074095DB9307B00235B713078002DE
:10C548006397E7023C5899C78E2B0A201386270168
:10C55800EF00F02F1C54DE2313F7072029CF78545F
:10C568005A2B1377072021CB93079002ADBF1307EF
:10C578009002639BE700EF606FF2AA850A20EF0044
:10C58800102C9307A00285B71307A0026390E70455
:10C59800EF602FF0AA85854701456384F500814542
:10C5A80005452EC6EF60EFEC2A86B2450A20EF005B
:10C5B800B0251C54DE2393F707409DC37C54DE2B23
:10C5C80093F7074091CF9307B00231BF1307B0022A
:10C5D8006398E700EF602FEDAA850A20EF00902A04
:10C5E8009307F002B9B58280411122C4405926C28E
:10C5F80006C67C54AA84DE2B13F7071011C71854FB
:10C608005A23137707100DE313F7072011C718549F
:10C618005A231377072009EB93F707408DCB1C5457
:10C62800DE2393F7074085C7930710023CB02285A5
:10C63800EFF0FFD738309307F002631EF70022446B
:10C64800AA20B2409244814541016FE01FC9930777
:10C65800F0023CB0EDB7B2402244924441018280DE
:10C66800397122DC405926DA4AD84ED606DEAA8924
:10C67800AE8432896302043A2A211E206384A7000B
:10C68800A14421A03C2091EB9D44F25062542685A0
:10C698004259D254B259216182809387E5FF93F7BA
:10C6A800F70F2D47E362F7FE37E706008A071307FF
:10C6B80007CCBA979C438287B2852285EFF07FAC7E
:10C6C800AA84E1B74146CA851305C4049740FA1FF6
:10C6D800E780E0C522858525AA8411C1A1443C30A4
:10C6E800130740056396E700930790053CB071BFB8
:10C6F800130760056395E7009307A005C5BFD147F9
:10C70800F5B79309C4054E854146CA859740FA1F77
:10C71800E780E0C10325040845C53C3013079005B0
:10C728006398E70022854D259307E0053CB079A082
:10C738001307A0056390E7087C3013D737002297CA
:10C7480014279D8BB3D6F640B737002083A707B5CB
:10C75800858A93E606F893F6F60F9DD39C478DD30A
:10C768009305050818084E861305050482979374E7
:10C77800F50FE39704F041460C081305C4049740ED
:10C78800FA1FE780C0CB7C304D47850793F7F70F3A
:10C798007CB06377F7002285052D9307E005B9B7CC
:10C7A800B737002003C5B7978545EF408FB7930784
:10C7B80050052DBF1307C005E386E7F68144F1B5A0
:10C7C800130984004E86CA8522851408EFE0BFE26B
:10C7D80041469305C40408089740FA1FE78020C61D
:10C7E800E30505EA8A861306C403CE854A85EF1059
:10C7F800206A05E12285EFE05FEBB73700202A8742
:10C8080083A747970A20814601468A858297AA848A
:10C8180011C1A14493072002D1BD0C22EFE0FFAB68
:10C8280071BF383093072002E310F7E67C5889EB94
:10C838009305300571459740FA1FE780208068D836
:10C848006858E30305E44146CA859740FA1FE78024
:10C8580000AE64582285EFE05FE5A8AC930730028C
:10C86800F1B5383093073002E310F7E21E2268581A
:10C878002146930529001EA949059740FA1FE7801C
:10C8880000AB7C54DE2B13F727002DC718545A230E
:10C89800098B2DC39307400251BD383093074002DE
:10C8A800E314F7DE3C5C81EB85455D459730FA1F64
:10C8B800E780C07828DC285CE30205F0834709009C
:10C8C8004146CA857CA99740FA1FE78040A693078E
:10C8D8005002A9BD383093075002E317F7DA285CF5
:10C8E80019469305190041059740FA1FE78020A4CF
:10C8F8007C54DE2B918B95CF1C54DE23918B95CBEA
:10C908009307600225B57C5C89EB9305300551459A
:10C918009730FA1FE780807268DC685CE30205D60E
:10C928004146CA859740FA1FE78060A07C5C7D5726
:10C9380098CB4E85EFF05FCB51B50325040813065D
:10C948000004CA85130505049740FA1FE780209E56
:10C958002285EFE09FC63C30130700056395E7008A
:10C9680093074005E1B313071005639CE700B73749
:10C97800002003C5B7978545EF40AF9A9307500548
:10C9880075B313072005E39BE7E2B737002083A7B9
:10C9980007B5E38707CE9C47E38407CE83250408C1
:10C9A80093048400180893850508814626862E85F9
:10C9B80082970A201008A685EF601FDA9307B00552
:10C9C800B5B338309307E005E310F7CC83250408A6
:10C9D80041464A859740FA1FE78060A6AD44E306C2
:10C9E80005CA032504084146CA859740FA1FE7800F
:10C9F80000942285EFE07FCBB73700202A8783A7F2
:10CA080047972C580A20814601468297AA8411C16B
:10CA1800A14493071002D9B9AD47E391F5DA14227E
:10CA28002E21130665000821EF602FDD41BB8947E1
:10CA380059C2D1C108A29C211CB29C313CA2BC2184
:10CA48003CB2BC31A30206005CA2DE21A183858B27
:10CA58005CB2DA211377072001C793E727005CB29D
:10CA6800DE2193F7074089C75C3293E747005CB241
:10CA7800DE2113974701635607005C3293E787006E
:10CA88005CB223030600DC21858B7CA2DA21098BAA
:10CA980001C793E727007CA2DE21918B89C77C22FE
:10CAA80093E747007CA2DA218147218B09C77822C6
:10CAB8001367870078A23E8582802E86AA85054561
:10CAC8006FF0FFF62E86AA8509456FF05FF6894755
:10CAD80085C51DC1411106C6AE870D47AA8598A315
:10CAE8001385170041469740FA1FE7804084B240FB
:10CAF80081473E85410182803E858280894785C580
:10CB08001DC1411106C6AE871147AA8598A3138592
:10CB1800170041469740FA1FE7806081B24081477D
:10CB28003E85410182803E858280894785C51DC139
:10CB3800411106C6AE871947AA8598A31385170021
:10CB480041469730FA1FE780807EB24081473E8594
:10CB5800410182803E858280894795C90DC941116E
:10CB680006C61D4798A11A21AE87214698B11A21F9
:10CB78002183B8A193052500138537009730FA1F44
:10CB8800E780E07AB24081473E85410182803E8558
:10CB98008280894785C51DC1411106C6AE872147D8
:10CBA800AA8598A31385170041469730FA1FE78096
:10CBB8000078B24081473E85410182803E8582806F
:10CBC80089479DC515C5411106C6254798A1182155
:10CBD800AE87194698B1930515001385270097303D
:10CBE800FA1FE780C074B24081473E8541018280C8
:10CBF8003E858280894785C51DC1411106C6AE871D
:10CC08002947AA8598A31385170041469730FA1F2C
:10CC1800E780E071B24081473E85410182803E85D0
:10CC2800828089478DC505C5411106C6AE87314743
:10CC3800AA8598A313851700130600049730FA1FD6
:10CC4800E780E06EB24081473E85410182803E85A3
:10CC58008280894785C51DC1411106C6AE87354703
:10CC6800AA8598A31385170041469730FA1FE780D5
:10CC7800006CB24081473E85410182803E858280BA
:10CC8800894799C511C595479CA11C219CB181472D
:10CC98003E858280894799C511C5AD479CA11C2155
:10CCA8009CB181473E8582800DC55D718A8586C6A7
:10CCB800A2C42A84EFE03F8C0A20B7D605000A8672
:10CCC800938626AC9D45EFE08FFEB6402644616111
:10CCD8008280054582800DC55D718A8586C6A2C49D
:10CCE8002A84EFE05F890A20B7D605000A86938672
:10CCF800C6AC9D45EFE0AFFBB6402644616182803B
:10CD0800054582805D71A2C49305C5022A84414607
:10CD18000A8586C69730FA1FE78060610A20B7D671
:10CD280005000A86938666ADC545EFE04FF8B64024
:10CD38002644616182805D71A2C49305C5032A847B
:10CD480041460A8586C69730FA1FE780405E0A206A
:10CD5800B7D605000A86938646B0C545EFE02FF59D
:10CD6800B640264461618280B737002083A707B5A3
:10CD7800A9CB9C435D71A2C486C62A841305E00F23
:10CD88008DCF032504089305050C13050508829724
:10CD980083250408130600040A859385050897303F
:10CDA800FA1FE780C0580A20B7D605009386A6C2A6
:10CDB8000A8693051004EFE08FEFB64026446161C0
:10CDC80082801305E00F8280317122DD2A840A21D6
:10CDD80026DB06DF4AD94ED752D556D35AD15ECF75
:10CDE80062CD9740FA1FE780A0CA3C58AA8489EB15
:10CDF8009305300571459730FA1FE780202428D81D
:10CE08002858CD4705C9714681459730FA1FE780F4
:10CE1800A058032904072285EFE03F89230DA900C4
:10CE28003C203739002063810712832709B585E341
:10CE38009307E00FFA506A54DA544A59BA592A5AF1
:10CE48009A5A0A5BFA4B6A4C3E852961828083AB09
:10CE58000701E38F0BFC032B0408EF509FE32A8C98
:10CE68000145EF501FE1DC303858130B0B029309D2
:10CE7800C403130AC405938A64003AC0B337F000A8
:10CE88002A87930801045688B33680015286CE85D6
:10CE98005A85829B1C54B8232307E1029833A306C2
:10CEA800E1029C232306F102832709B5D1D303AB02
:10CEB8004701E30F0BF6DC30B337F0003ECEEF50FE
:10CEC8005FDDAA8B0145EF50DFDA03270408F2473C
:10CED8002AC03AC2B3387001568878109306840085
:10CEE8004E86D2858800029B7C54B82B2305E1022C
:10CEF8009833A304E1029C232304F102832709B594
:10CF080003A94701EF50FFD82A8B0145EF507FD680
:10CF180083C854009C082A883EC2B3381001B3372E
:10CF280060013810930684015286CE8556C0880069
:10CF380002990A20B7D605009386A6C59008C5456C
:10CF4800EFE0EFD6AA87FDB5D430832709B5032BC8
:10CF58000408B336D00083AB070136CEEF507FD339
:10CF68002A8C0145EF50FFD03C58F246130B0B02B8
:10CF7800130AC4059309C403938A64002A88930892
:10CF880001044E86D2853EC05687B33780015A8544
:10CF9800829B1C54130B0103B8232307E102983327
:10CFA800A306E1029C232306F102832709B583AB7C
:10CFB8004701DC30B337F0003ECEEF509FCD2A8CCE
:10CFC8000145EF501FCBF2472AC0B338800156887D
:10CFD8007810930684004E86D2855AC28800829BB8
:10CFE8008325040841465A859730FA1FE780204573
:10CFF800AD47E31B05EE3DBDB7D605002E869386EB
:10D0080026B3C5456FE0AFCA5D71B287A2C44C8034
:10D018002A84BE8513051100194686C69730FA1F63
:10D02800E780E030B7D605000A862285938686BC5D
:10D03800A145EFE0CFC7B640264461618280B7D6EC
:10D0480005002E869386A6B9C5456FE04FC65D716B
:10D05800B287A2C46C802A84BE85130521002146AC
:10D0680086C69730FA1FE780802CB7D605000A8657
:10D078002285938606B6AD45EFE06FC3B6402644D9
:10D0880061618280B7D605002E869386C6BFC545E6
:10D098006FE0EFC1797122D406D626D23C3113074E
:10D0A80030052A846381E708130750056392E7086F
:10D0B8009307A0053CB17C31C14513D737002A97A7
:10D0C80014279D8B1305C503B3D6F640858A93E6CE
:10D0D80006F893F6F60F36C6EF503F8DB246B737CF
:10D0E800002083A707B59DCB9C478DCB032504085B
:10D0F80018081306C4039305050413050508829749
:10D108001375F50F01ED1305C40241460C0897305D
:10D11800FA1FE780C0212285EFF0DFBEB25022540B
:10D12800925445618280930790053CB1814645BF82
:10D13800130710026391E7027C5503270508DE2BCD
:10D1480061EF13F7170069CB18555A23058B69C788
:10D15800930720023CB03C30130720026394E70E8B
:10D168003C5889EB9305300571459730FA1FE780E5
:10D17800E0EC28D82458ADCC2285EFE00FD3A8AC3A
:10D188002858814541469730FA1FE780E020285803
:10D198003D472C2D9387F5FF93F7F70F636DF70243
:10D1A800B737002083C7B7B5D9CB414681450808B2
:10D1B8009730FA1FE780401EB7350020194693853F
:10D1C800C58408089730FA1FE780601630580C08A5
:10D1D8002E85EF801026EF30AFFA3C58A1458AAB78
:10D1E80013852701EF506FFC2C580A20EFF0DFE081
:10D1F800930730020A203CB09740FA1FE780408925
:10D20800414611C17225B737002003C5B7970606F6
:10D218008545EF30FFAE19B713F7270001CB185437
:10D228005A23098B01C7930740022DB7918B85D7E5
:10D238001C54DE23918B85D39307600221BFEF50E6
:10D24800CFF651BF130730026396E7023C5899C7DF
:10D258008E2B0A2013862701EFF07FDF7C54DE2B0C
:10D2680013F7270021CB18545A23098B21C793079A
:10D27800400249B713074002639BE700EF501FA223
:10D28800AA850A20EFF0BFDB93075002A5B7130762
:10D298005002639DE702EF50DF9F15E58145054584
:10D2A8002EC6EF501F9D2A86B2450A20EFF0DFD523
:10D2B8007C54DE2B918B8DC71C54DE23918B8DC340
:10D2C8009307600205BF85450145D9BF1307600272
:10D2D8006398E700EF503F9DAA850A20EFF09FDA98
:10D2E8007C5403270408DE2B09EF13F7071011CB32
:10D2F80018545A231377071009C7930770023CB0D4
:10D3080031BD13F7072009CB18545A231377072088
:10D3180001C793079002E5B793F7074089CB1C54E0
:10D32800DE2393F7074081C79307B002C9BF93076D
:10D33800F002F1B7397122DC26DA4ED652D406DE75
:10D348004AD8AE89328AAA849730FA1FE780407497
:10D358004059414681450A859730FA1FE780C00346
:10D3680035C4035904006313990638309307100233
:10D37800631FF7028327040899CF2C58A1C94A854F
:10D38800EF1080790545F2506254D2544259B2598F
:10D39800225A216182808A861306C4059305C40334
:10D3A80013058400EF00D02E15E18A85C9BF2C58DB
:10D3B80091CD9E29639C47012146C9054E8597302A
:10D3C800FA1FE780C00719C12C5855BF268597302A
:10D3D800FA1FE780E06B2A84054555D44C54B1C543
:10D3E8009E29639447052146C9054E859730FA1F43
:10D3F800E780E0048547631AF502B727002083C752
:10D40800F74F89C74C54BC3D639AA70CBD45268588
:10D41800EF10406BB737002083A7C7800145A5D719
:10D428001D45894582970145B9BFB737002003C715
:10D43800C7B5B72900209389897D058B3E8929C303
:10D44800B7370020583083C747B5631BF702B73595
:10D4580000201946938555B5130564009730FA1FC7
:10D46800E780E0FD8547631DF50083A7490381C771
:10D4780091451D458297BD452685EF10A06419B7D3
:10D48800373700200347B7B583A7490331CB034794
:10D49800C9B5098B09CB81C795451D458297268556
:10D4A800EF10C067C5B581C78D451D4582974146B8
:10D4B800814508089730FA1FE78000EEB73500204D
:10D4C80019469385C58408089730FA1FE78020E637
:10D4D8000C082E850A86EF80C0758A8526854DB58D
:10D4E8008545C5FF6DBF797122D440594AD04ECECB
:10D4F80052CC06D626D2AA892E8A328963060462BD
:10D508002A211E20638CA700A144B25022542685EC
:10D5180002599254F249624A45618280242099C096
:10D528009D44E5B79387F5FF93F7F70F3147E36914
:10D53800F7FE37E706008A07130707CFBA979C4319
:10D5480082871C54F1F393053005130500049730C6
:10D55800FA1FE780A0AE08D445D9034709009147D0
:10D5680063F4E7008D4455B7034719008547E3EB9B
:10D57800E7FE13060004CA859730FA1FE78020DB10
:10D588000C547054A3020400D4415C4A858AFD8E71
:10D598005E2AF99BD58F5EAAD841544AF59B05832C
:10D5A800058B8582F98E8606DD8E56AADC41584A9F
:10D5B800ED9A8983858B09837D8F0A07558F5AAA2F
:10D5C800D4415C4A5D9B8D82858A8D83F58F8E0759
:10D5D800D98F5EAAD841544A93F7F7EF2183058B78
:10D5E800A182F98EA206DD8E56AADC41584AA5838F
:10D5F800858B25837D8F9317970013F7F6DF5D8F53
:10D608005AAAD4415C4AA982858AA983F58F939640
:10D61800A7009377F7BFD58F5EAAD441584AAD8249
:10D62800858A2D83758FFD769386F67F2E07F58F75
:10D63800D98F5EAA3C2A03250408A18BF1CFBC210F
:10D64800A18BF9CBE31205EC930530051305001007
:10D658009730FA1FE780809E2320A40801D57C54C8
:10D66800A302040003471900943399E63DCF5C30C8
:10D6780093E707015CB021A0A1475CB06DFB228550
:10D68800EFF06FE56C54BC29858B89CB1C54BC2307
:10D698008D8B89C77C2093E717007CA0832704081B
:10D6A80089C77C2093E787007CA05C300547639896
:10D6B800E70A41468145130584009730FA1FE78041
:10D6C800A0CD41468145130584019730FA1FE780B4
:10D6D800A0CCC1451305C403EF502FAD8327040820
:10D6E800ADCF930700053CB00DB5B82B118B19E7EA
:10D6F80003472900118B19E38547ADBF9C231547C4
:10D7080083460900B387E70237E70600130747CACD
:10D71800BA97B6979C23B9BF19C59730FA1FE78007
:10D72800E09E232004087C54983311C7034719004E
:10D7380019C3E14781B7B82B118B09E703472900C3
:10D74800118B5DDB9C23154783460900B387E702ED
:10D7580037E70600130787C865BFC14769B713F7DE
:10D76800870131CBC18B1305840041468DCF8905D4
:10D778009730FA1FE780A0BB414681451305840115
:10D788009730FA1FE78040C17C20C1451305C403C8
:10D7980093E747007CA0EF504FA18327040891CB63
:10D7A8009307200589B781459730FA1FE780C0BEE7
:10D7B800E1B7CD470DBF09478945638AE70011479F
:10D7C80085456386E70019476396E7008D450A207B
:10D7D800EF50BFEF7C2093E747007CA08327040825
:10D7E80081C79307100501B7C547F5BD4146CA85EE
:10D7F8001305C4049730FA1FE78060B33C30130761
:10D808006005639CE700B737002003C5B7978545D7
:10D81800EF302FB193075005F9B545476383E70209
:10D828009306C4021306C403930584002285EFD02F
:10D838009FDC2285EFF00FCDAA8411C1A144D14706
:10D848005DB5C9474DB59309C4054E854146CA859E
:10D858009730FA1FE780A0AD0325040869C53C305E
:10D86800130790056398E7002285EFF0CFCC930764
:10D87800E00595BD1307A0056399E706B7370020B3
:10D8880083A707B5E38E07C803A88700E30A08C87B
:10D898007C30930505084E8613D737002297142746
:10D8A8009D8B0A87B3D6F640858A93E6060813054A
:10D8B8000504029841468A851305C4049730FA1F67
:10D8C800E780E0B711E1D2842285EFF0CFC67C3043
:10D8D800CD461307E005850793F7F70F7CB063E49F
:10D8E800F6001307600538B00DB11307C005E39EB5
:10D8F800E7C0B737002083A707B5E38307C29C4773
:10D90800E38007C293050508130984000A87814646
:10D918004A862E8582970A200A86CA85EF50DFE359
:10D928009307B005C9B38A864E869305840022857D
:10D93800EFD07FCC41469305C4040A859730FA1F7F
:10D94800E780E0AF8547D284E311F5BC2285EFF08C
:10D958008FBEAA84E31A05BA9307100269B3383058
:10D9680093077002E31EF7BA7C5889EB93053005DC
:10D9780071459720FA1FE780606C68D86858E30102
:10D9880005BACA8541469730FA1FE780409A0329AD
:10D9980044072285EFD07FD1230DA9009307800289
:10D9A80099B3383093078002E31CF7B61E226858F3
:10D9B8002146930529001EA949059730FA1FE780DB
:10D9C80000977C54DE2B13F7072035C718545A23C9
:10D9D800137707202DC39307900231B3383093078C
:10D9E8009002E31FF7B23C5C89EB930530055D4577
:10D9F8009720FA1FE780806428DC285CE30205B2E0
:10DA08004146CA859730FA1FE78060929307A002C3
:10DA1800D9B938309307A002E314F7B01C22285C68
:10DA28001946930519007CA941059730FA1FE7802C
:10DA380000907C54DE2B93F70740A1C71C54DE23CB
:10DA480093F707409DCF9307B00271B93830930719
:10DA5800B002E317F7AC7C5C89EB930530055145C0
:10DA68009720FA1FE780805D68DC685CE30E05A8F4
:10DA78004146CA859730FA1FE780608B7C5C7D57EA
:10DA880098CB03D529008145EFD03F85BDBC383000
:10DA98009307F004E3FAE7A603250408E30605A6BE
:10DAA80013060004CA85130505049730FA1FE7809A
:10DAB80000882285EFF04FABAA842285EFD0FFAF14
:10DAC8003C3013070005639FE700B737002003D6F3
:10DAD800E90003C5B79785450606EF306FA293079F
:10DAE800300511B1130710056395E700930760052A
:10DAF800DDBE13072005E39AE7A09307C005E5B646
:10DB080038309307E005E311F7A0032504084146E0
:10DB1800CA859730FA1FE78080812285EFF0CFAA67
:10DB2800AA841DBD0C228DB785478144E39FF59CCF
:10DB3800032846003C32382214322E211022014597
:10DB4800EF502FC2D9B28147C1463307F500B388D9
:10DB5800F500182383C808003308F6008507334703
:10DB680017012300E800E392D7FE82800147BD47F2
:10DB78001308F00F3306F5001422B388F500FD17DB
:10DB88008606558F2380E800182293F7F70F1D8328
:10DB9800E39207FF82808147930800F8414893F693
:10DBA800F70F3387F50063FAC600B306F500942231
:10DBB80014A38507E39507FF82806395C6002300B9
:10DBC8001701C5BF23000700EDB701114AC856C2A7
:10DBD8002E89AA8A93053005414506CE22CC26CA4D
:10DBE8004EC652C4328A9720FA1FE7802045AA847D
:10DBF8009305300541459720FA1FE78020442A8481
:10DC0800CD49A5C431CD414681459720FA1FE7800B
:10DC1800A0782686A2855685EF80A001AA8929E1E9
:10DC28008387040063D30706A2852685EFF01FF4D7
:10DC3800B7E506004A86938545D22285EFF0BFF006
:10DC48008307090063D80704A2854A85EFF01FF20D
:10DC5800B7E506005286938545D22285EFF0BFEEE0
:10DC680026859720FA1FE780604A11C422859720ED
:10DC7800FA1FE780A049F24062444E85D2444249E7
:10DC8800B249224A924A05618280CA852685EFF008
:10DC9800FFED7DB7D2854A85EFF05FEDD1B78147BB
:10DCA8004146B306F5003387F500182303C806007C
:10DCB80085073347070198A2E395C7FE82800111C3
:10DCC80026CA4EC6AE84AA899305300513050003FB
:10DCD8004AC806CE22CC32899720FA1FE780003640
:10DCE8002DC51306000381452A849720FA1FE78073
:10DCF800A06A4146CE8522859720FA1FE780A07842
:10DD0800A6850D461305D4019720FA1FE780A07752
:10DD180013060402930504012285EF709071AA840A
:10DD28000D469305D4024A859720FA1FE780A0750F
:10DD380022859720FA1FE780603DF24062442685DD
:10DD48004249D244B24905618280CD44FDB75D7134
:10DD58004EDE62D4AE892A8C930530051305000384
:10DD6800A6C2CAC052DC56DA5AD85ED686C6A2C443
:10DD7800B28B368BBA84BE8A4289468A9720FA1FAC
:10DD8800E780C02B630405101306000381452A842D
:10DD98009720FA1FE78040604146E2852285972058
:10DDA800FA1FE780406E414681450A859720FA1F91
:10DDB800E780805E1D46DE850A859720FA1FE7808A
:10DDC800806C1D46DA85130571009720FA1FE780DD
:10DDD800806B33392001B3349000414681450808EF
:10DDE80023072101C4879720FA1FE780E05A1946C4
:10DDF800D68548089720FA1FE780E0681946D2853B
:10DE08001305A1019720FA1FE780E0679304040136
:10DE18004146CE8526859720FA1FE780C0668A8509
:10DE28002685EFF0DFE7930904024E86A685228552
:10DE3800EF7030602A890DE94146CE852685972006
:10DE4800FA1FE780C04E0C082685EFF05FE54E8686
:10DE5800A6852285EF70F05D2A8946454146CE8524
:10DE68009720FA1FE780206222859720FA1FE78013
:10DE7800E029B64026444A8596440649F259625A32
:10DE8800D25A425BB25B225C616182804D49D5B750
:10DE9800011126CA52C4AA842E8A130500039305C9
:10DEA80030054AC84EC606CE22CC3289B68997209C
:10DEB800FA1FE780A01835C52A84A6854146972011
:10DEC800FA1FE780405C930404012146D285268529
:10DED8009720FA1FE780205BCA8521461305840135
:10DEE8009720FA1FE780205A13090402A6854A865C
:10DEF8002285EF701054AA844146CA854E85972022
:10DF0800FA1FE780405822859720FA1FE7800020F3
:10DF1800F240624426854249D244B249224A056108
:10DF28008280CD44F5B739715AD05ECE2A8BAE8B3C
:10DF380041459305300506DE26DA52D456D262CC26
:10DF480066CA6AC8368C328DBA8C22DC4AD84ED65C
:10DF58009720FA1FE780800EAA8A9305300541456D
:10DF68009720FA1FE780800D2A8ACD44638E0A081D
:10DF780059C52A86D6855A85EFF03FC5AA8441E15E
:10DF88009305300541459720FA1FE780200B2A8921
:10DF98009305300541459720FA1FE780200AAA8992
:10DFA800630A090E6306050E1304FD001184137637
:10DFB800FD0049C07D144204418035EE131544002C
:10DFC8004E86D6855E95EFF01FB8414681454A8555
:10DFD8009720FA1FE780403C014D93170D01C1833C
:10DFE80063F48708BDC04A859720FA1FE7800012AE
:10DFF800638709004E859720FA1FE7802011568510
:10E008009720FA1FE780801063070A00528597203F
:10E01800FA1FE780A00FF250625426854259D25465
:10E02800B259225A925A025BF24B624CD24C424D80
:10E03800216182800144131544008A855E95EFF0C2
:10E048009FB54E86D2850A85BDBF93154D000A86B9
:10E05800DE954A85EFF03FAF4A868A855A85EF708C
:10E06800503DAA84050D95BFBDFC0A86CE854A851C
:10E07800EFF07FAD4A868A855A85EF70903BAA8477
:10E088006686CA8562859720FA1FE780402AA1BF65
:10E09800CD4491BFCD44A9BF397162CC2A8C594572
:10E0A80026DA4AD84ED652D456D25AD05ECE06DE9A
:10E0B80022DCAE8B328BB68A3AC63E8AC289468942
:10E0C800834401049720FA1FE780A0162DCD91679D
:10E0D800938717E91EA185473CA12A843247210569
:10E0E800630A0C04930710033CB019468145972036
:10E0F800FA1FE780602A23036401A303540144A89C
:10E10800231274012317440123183401231924010D
:10E11800A285B73700206254F250D2544259B259FE
:10E12800225A925A025BF24B624C03C587972161CF
:10E138006F200FEBA30104001946BA859720FA1F38
:10E14800E780E01E4DBFF2506254D2544259B25992
:10E15800225A925A025BF24B624C21618280011171
:10E1680022CC2A84314506CE2EC632C436C23AC0E5
:10E178009720FA1FE780E00B15C99167938717E985
:10E188001EA1B2452246924602478D473CA120B1C6
:10E198006244B73700204EA172A116A53AA5F240F5
:10E1A800AA8503C5879705616F208FE3F240624413
:10E1B8000561828001114AC82A89394526CA06CED6
:10E1C80022CC2EC6B2849720FA1FE78080061DCD88
:10E1D800B2459167938727E91EA191473CA1A30106
:10E1E80025014EA12A84A685190521469720FA1FE4
:10E1F800E780E013A285B73700206244F240D2449A
:10E20800424903C5879705616F208FDDF24062445C
:10E21800D24442490561828001114AC82A89414590
:10E2280026CA06CE22CC2EC6B2849720FA1FE780D3
:10E23800400015CD9167B245938727E91EA1954700
:10E248002A843CA123122501214619059720FA1F8B
:10E25800E780E00DA28566A4B73700206244F2404B
:10E26800D244424903C5B79705616F206FD7F24082
:10E278006244D244424905618280011122CC2A8439
:10E28800394506CE2EC632C436C23AC09720FA1F88
:10E29800E78020FA15C99167938717E91EA1B2454F
:10E2A80022469246024799473CA142A1B73700202F
:10E2B80062446EA112A536A55AA5F240AA8503C5E7
:10E2C800879705616F20CFD1F24062440561828053
:10E2D800797122D406D62A842EC632C436C23AC0F0
:10E2E8009720FA1FE780C07A19CDB2452246924698
:10E2F8000247EC84F0852C081306F00F2285F4867B
:10E30800F887EFC03F8AB2502254456182800111DC
:10E3180022CC2A84394506CE2EC632C436C23AC02B
:10E328009720FA1FE780E0F015C99167938717E9EE
:10E338001EA1B2452246924602479D473CA142A1F2
:10E34800B737002062446EA112A536A55AA5F2403F
:10E35800AA8503C5879705616F208FC8F24062447C
:10E36800056182805D713EC2835701062AC6130586
:10E3780040024EDE52DC56DA5AD85ED662D466D2F5
:10E388006AD06ECE86C6A2C4A6C2CAC02E8DB28C72
:10E39800368C3AC4C28DC68B035B0105835A41058E
:10E3A800034A81058349C1053EC09720FA1FE780CB
:10E3B80040E861CD1166130616E9324312A113062F
:10E3C80090022A8930A19304E90021051304490128
:10E3D800924722476302030893071003A301F90039
:10E3E800194681459720FA1FE78000FB19468145A9
:10E3F80026859720FA1FE78020FA1946814522854D
:10E408009720FA1FE78040F9824723039901A30365
:10E41800890123004903A30039032311F902264483
:10E42800B73700202312A901231D7901231E690192
:10E43800231F5901B6409644F259625AD25A425B98
:10E44800B25B225C925C025DF24DCA8503C5879778
:10E45800064961616F20CFB8BA85A3010900194642
:10E468003EC29720FA1FE78080EC9247268519461E
:10E47800BE859720FA1FE78080EB1946EE85228536
:10E488009720FA1FE780A0EA41B7B6402644964491
:10E498000649F259625AD25A425BB25B225C925CDC
:10E4A800025DF24D61618280011122CC2A842145EE
:10E4B80006CE2EC632C436C29720FA1FE78060D730
:10E4C80005C9224692469167938717E91EA1B2456E
:10E4D800B1473CA120B170A174B16244B7370020A4
:10E4E8004EA1F240AA8503C5879705616F204FAFFB
:10E4F800F24062440561828041110D4506C69720AD
:10E50800FA1FE78000D315C1930710F91CA19307E0
:10E51800E0031CB1C5473CA1B7370020B240AA852B
:10E5280003C5879741016F20AFABB240410182809C
:10E53800011122CC2A84294506CE2EC632C436C201
:10E548009720FA1FE780E0CE05C9B2459246916749
:10E55800938717E91EA12246C9473CA14CA120B1C7
:10E5680014A56244B737002072A1F240AA8503C5FA
:10E57800879705616F20CFA6F240624405618280CB
:10E5880001114AC82A892D4526CA06CE22CC2EC694
:10E59800B2849720FA1FE780C0C929C1B245930702
:10E5A80010F91CA19307E0031CB1CD473CA1A301BE
:10E5B80025014CA12A84A685150519469720FA1F1E
:10E5C800E780E0D6A285B73700206244F240D24403
:10E5D800424903C5879705616F208FA0F2406244C6
:10E5E800D244424905618280011122CC2A84214506
:10E5F80006CE2EC69720FA1FE780A0C305C5B245F0
:10E608009167938717E91EA1D1473CA16CA142A14C
:10E61800B73700206244F240AA8503C58797056191
:10E628006F200F9CF240624405618280011122CC68
:10E638002A84214506CE2EC632C49720FA1FE780C9
:10E6480040BF1DC12246B245930710591EA120A103
:10E6580070A16244B73700204EA1F240AA8503C5D5
:10E66800879705616F20CF97F240624405618280E9
:10E67800011122CC2A84214506CE2EC632C4972009
:10E68800FA1FE78000BB15C522469167938727E9E3
:10E698001EA1B245A1473CA160A170B16244B73741
:10E6A80000204EA1F240AA8503C5B79705616F20E7
:10E6B8002F93F240624405618280011122CC2A84A2
:10E6C800314506CE2EC632C436C23AC09720FA1F4C
:10E6D800E78020B605C922468567B24592460247BB
:10E6E800938717C91EA120A170A16244B7370020E3
:10E6F8004EA116A53AA5F240AA8503C587970561DC
:10E708006F200F8EF240624405618280011126CA93
:10E71800AE844AC82A891385C40006CE22CC32C6E4
:10E728009720FA1FE780E0B00DCD8567938717E93A
:10E73800B2451EA124A1231225012A84310508C44B
:10E7480026869720FA1FE78080BEA285B73700206B
:10E758006244F240D244424903C5879705616F205D
:10E768002F88F2406244D2444249056182800111F7
:10E7780022CC2A84194506CE2EC69720FA1FE78098
:10E7880040AB05C58567938717F91EA1B245854734
:10E798003CB120A16244B73700204EA1F240AA85BF
:10E7A80003C5879705616F20AF83F2406244056116
:10E7B8008280411122C42A840D4506C69720FA1F7B
:10E7C800E78020A70DC1930710F91CA1E9471CB1E8
:10E7D80020A12244B7370020B240AA8503C58797F5
:10E7E80041016F10FFFFB2402244410182800111B4
:10E7F80022CC2A84214506CE2EC69720FA1FE78010
:10E8080040A30DC59167938727E91EA1B2459307D9
:10E8180000033CA160A16244B73700204EA1F2403A
:10E82800AA8503C5B79705616F109FFBF240624444
:10E83800056182800111214506CE2EC632C497207B
:10E84800FA1FE780009F05C58567B2452246938772
:10E8580007391EA185473CA1B73700204EA172A1F8
:10E86800F240AA8503C5078E05616F107FF7F24055
:10E8780005618280397122DC1304F5FF4AD852D42D
:10E8880056D25ECE420406DE26DA4ED65AD0894BE0
:10E898002A8A3289B68A418063937515B72B00207E
:10E8A80083C70B5A5E8B894495CF83C916009C2277
:10E8B8009144A209B3E9F900B727002083D7877EDE
:10E8C800F51763D1F9029307C6FF639DF90831452F
:10E8D8002EC69720FA1FE780C0952A84B24519ED05
:10E8E8009304F00FF250625426854259D254B2591B
:10E8F800225A925A025BF24B2161828042091359D3
:10E9080009014CA123132501930700F91509A165F5
:10E918001EA12311450185054A859710FA1FE78036
:10E92800E07108C415C983C70B5A9385EAFF1356CB
:10E938002900FD172380FB5A9720FA1FE780C0A201
:10E948001C44A28589071CC4B737002003C5078E5D
:10E95800EF101FE9814479B722859710FA1FE780E5
:10E96800E07ABDBF9307D6FFE3CCF9F6B14733048D
:10E97800F402B734002083A7448EA297B82719C79A
:10E98800884309C59710FA1FE78040781385490026
:10E99800A16542058505418103AA448E9710FA1F97
:10E9A800E780C06983A7448E229A2320AA00A297F1
:10E9B80088431DD50547B8A783470B5A4A86D6858D
:10E9C800FD172300FB5A9720FA1FE780409683A77C
:10E9D800448E3E942313240123123401A5BFB1476A
:10E9E8003304F402373B002083274B8EDA89A29741
:10E9F800FA2388435DC3DE23B306C700910763CEBD
:10EA0800D7083A95D6859720FA1FE78040920327C2
:10EA18004B8E814422977E23CA97C207C1837EA367
:10EA28005A231107E390E7EC31459720FA1FE78056
:10EA38004080AA850DCD930700F91EA183274B8E30
:10EA48002302750123114501A297FA239C437AA159
:10EA58001CC5B737002003C5078EEF107FD8832762
:10EA68004B8E3E942313040023050400A5BD832781
:10EA78004B8EA297884311C99710FA1FE780006947
:10EA880083274B8EA29723A0070083A7498E3E9425
:10EA9800231304002305040075BD11C99710FA1F3C
:10EAA800E780C06683A7498EA29723A0070083A7A3
:10EAB800498E85443E9423130400230504001DB5A4
:10EAC8006FA0201D6FA0401E6FA0004205458280E8
:10EAD80005458280411106C6EFA0401DB2400145A0
:10EAE800410182806FA0601F6FA020216FA0C0230A
:10EAF8006FA080256FA020276FA0E0286FA0A02A14
:10EB08006FA0602C6FA0002E6FA0C02F1C321022A7
:10EB1800A2075D8E6FA020316FA060326FA0C03455
:10EB28006FA020376FA080396FA0C03E6FA0A040B3
:10EB38006FA080426FA060446FA040466FA020483D
:10EB4800411122C60344C10226C48344010303437E
:10EB58000101030E4101834E8101034FC101834F1F
:10EB68000102834241028343810222D6324426D8DD
:10EB7800A2441ED416D27ED07ACE76CC72CA1AC8D7
:10EB880041016FA0204C6FA080456FA060476FA027
:10EB980040490545828005458280054582806FB0E1
:10EBA800103D05458280054582806FB07042B7E60A
:10EBB80006008147938646D31308F00F3387F60083
:10EBC80010231317060141836364E50063130601EC
:10EBD800828092216364C7009AA18280850793F797
:10EBE800F70FE9BF41119397050122C406C626C253
:10EBF800C1872E8463D607029710FA1FE780C06882
:10EC0800AA8401CD1C21054793C707086364F70050
:10EC1800EF50607B2685EF10DFB72165218D21A895
:10EC280093F7150091CFB737002083A7C79E91C3EC
:10EC3800829713451400B2402244924441018280D5
:10EC480093F7250091CBB737002083A7079F91C37F
:10EC5800829713452400C5B793F7850099CBB7373A
:10EC6800002083A7C79FFC5791C382971345840050
:10EC7800D9B793F7450099CBB737002083A7C79F2B
:10EC8800BC5791C382971345440075B793F70502A3
:10EC980081CFB737002083A707A183A7070991C3AE
:10ECA80082971345040241BF93F7050181CFB73717
:10ECB800002083A707A183A7C70891C3829713459C
:10ECC800040195BF939725010145E3D607F6B737A9
:10ECD800002093878798F433F023CC33C823EFA020
:10ECE800C045096525BF411126C2B7340020B73792
:10ECF800002013060012814522C42A8413858498B3
:10ED080006C623A607AA4AC09710FA1FE780C0685C
:10ED18000145EF10B0510145EF109058B72700207A
:10ED2800A3858778B707D70713848498B5075CC885
:10ED3800B7B70D0D938717131CCCB7B7D7079387B1
:10ED480017135CCCED77938717137D471EB0232CE0
:10ED5800E40C81470327840C232EF40CE167938786
:10ED6800F79F5D8F8327C40C8966938606B0372981
:10ED78000020D58F1309897D2326F40C232AF40C4F
:10ED88008347E9002324E40C2328E40CA30AF40AAB
:10ED9800A30EF40AF977FD17231FF40E2310F410BD
:10EDA800FD472301F41085679387F7F03EBC5EBCEE
:10EDB800A30C0402EF208FE49307C01C2319F40668
:10EDC8008547A30FF402835749000357090128B068
:10EDD800A983A30EF4068D472311F4042322040407
:10EDE8009306B00F9387849863F4E6001307B00F77
:10EDF80093150701BAB7FAB703C7C703C1811386CA
:10EE0800E500118B35CB1387A5080E0783C6D703FA
:10EE180042074183DAB7918ABDC29386A5088E0658
:10EE2800C206C18296BB6D4593848498AE8663F30F
:10EE3800A500ED46B6B093058014BA866374B70092
:10EE4800930680141307C01C2390E70437071600A5
:10EE58000E0613070790D6B3F2B396B7D8DBEF7058
:10EE6800205CEF30803BEF6010442244B240924473
:10EE7800024941016F50B0271317360041BF93165E
:10EE8800360079BF397122DC3704400026DA4ED6C5
:10EE9800AE84AA899305E4FF054506DE4AD8EF202B
:10EEA800CFDE498C13170401418321839317840013
:10EEB80013590401D98F231601001379F90F10088B
:10EEC8008A854E857C87A306210102C002C202C43E
:10EED80002C802CA02CC02CEEF60B0558347E101F6
:10EEE8000347D101A0B0A2074207BA970347F1012F
:10EEF8002180C0A0BA97F25062549CA013D7870013
:10EF0800C183A382240198B0BCA04259D254B259FB
:10EF180021618280B725002037350020011119466C
:10EF28009385057F130585A606CE22CC26CA4AC836
:10EF380091644EC69710FA1FE780603F9385F4FFEF
:10EF48000145EF204FD22A84FD550145EF20EFD32C
:10EF5800A287FD147D5933F79700B366E500D5CA3B
:10EF6800631425016307970A373400201307849830
:10EF78002308F70EA18393E707FC9169C164232650
:10EF8800A70EA308F70E13048498FD19FD14CE8567
:10EF98000145EF204FCD2A89FD550145EF20EFCEE1
:10EFA800B3672501EDD7FD576314F500E30139FF79
:10EFB80093570501230AF40E93578501A30AF40E0B
:10EFC8008317040E2319A40E230B240F420513598B
:10EFD80089001379F9034185A30B240F658DE58F0B
:10EFE8006312F5020317440F8317240E658FE58F0C
:10EFF800631AF7000317640F8317440E658FE58FB4
:10F00800E307F7F8F2406244D2444249B249056145
:10F018008280A6850145EF200FC52A84FD5501454C
:10F02800EF20AFC6A28705BF411126C2B734002022
:10F0380006C622C44AC09387849803C7E70383C7D8
:10F04800F703636AF70001442285B24022449244E0
:10F058000249410182802A899305102413058007FB
:10F068009710FA1FE78080FD2A8471DD1306800758
:10F078008145938484989710FA1FE780E0316314E0
:10F088000900C1575CA0BC48B1E3E0C4A0C8E0C80F
:10F09800232004008547238FF40285475CB093073B
:10F0A80000F97CB0B73700209387C7AC9853DC537E
:10F0B80038C47CC4FD573CA8B727002003C5C77EC9
:10F0C8002302A406EF60504408B8BDBFFC4880C3C3
:10F0D800E0C82320040083C7E40385076DBF3C2DE7
:10F0E800411122C406C699075CB53C45114758A58D
:10F0F80098A33C4558352A8498B383471503858BD4
:10F1080091E70347050389476317F70038441C2331
:10F1180093E707041CA3284493052403194609050B
:10F128009710FA1FE780A0202844322C0C542105A0
:10F138009710FA1FE780A01F930730F97CB0B24000
:10F1480022444101828041114AC037390020930787
:10F15800899883A7C70A06C622C426C299E305452B
:10F1680031AAAA8413098998EF6090678327C90A8E
:10F178008297EF20F0622A847DD19C50EC442324AE
:10F18800F508F8309307A0096310F71085472300A6
:10F19800F51483C7F4052303F514A303F514FC350C
:10F1A80098290148A2074207BA97F8251546F90594
:10F1B800BA9703C735FF130584136207BA97232C40
:10F1C800F40883C755FF03C765FFA2074207BA972C
:10F1D80003C745FFBA97232EF40883C775FFA30B0F
:10F1E800F40283C795FF03C785FFA207D98F1EBC0A
:10F1F80083C7B5FF03C7A5FFA207D98F3EBC83C746
:10F20800D5FF03C7C5FFA207D98F5EBC83C7F5FF2B
:10F2180003C7E5FF232E0413A207D98F7EBC8147BD
:10F22800232CF4129710FA1FE7806010F8448347E4
:10F238003702FD8BA30AF40203473702ED1793F751
:10F24800F70F15832308E4022D476365F7023E3C58
:10F2580005679306A7C7E917C207C18363ECF600E1
:10F26800563C9307301F63E7D7007E3C130707C857
:10F27800637BF7020A24EF20B0720145B2402244B2
:10F2880092440249410182808327090D139717018F
:10F29800E35707F0BC4498239C21F98F9583858B0D
:10F2A8002300F514EDBD8327090B22858297832758
:10F2B800890D0A24294693F7072091E3054693050B
:10F2C8000008EF50C0278327090D139717016358CB
:10F2D80007000A24514693050008EF50402683276B
:10F2E800C904BC4B13974700E35B07E6C820A38912
:10F2F8000400494693050008EF5060248DB5B737E0
:10F30800002083C79798411122C406C626C24AC066
:10F318002A8485EB582485476312F70E83479403A4
:10F3280003471404858B6319F70C194693052404C5
:10F338001305A4039710FA1FE7806010B334A000E8
:10F3480089A883471504D5C38347750413070004A8
:10F3580093F7070C639BE708485539C11309240440
:10F36800CA851305A502EF50002E8547AA846319A4
:10F37800F502485489472300F4043C311946CA85EC
:10F3880093E72700A300F40451059710FA1FE780BC
:10F3980000FAB24022442685024992444101828003
:10F3A800582485476303F7048347C405918B95EF79
:10F3B800834784039DEB130504049720FA1FE78015
:10F3C800004548D41DC189472300F4043C3119463F
:10F3D8009305240493E72700A300F404510597102C
:10F3E800FA1FE780C0F485446DB783478403898B8F
:10F3F80095D35C549C3399FF814461BF8347C4050E
:10F40800918B89FF1C3413F7170005C374340D471B
:10F41800639DE60028406C402244B2409244024971
:10F4280041011723FA1F67004346898BCDDF7834E3
:10F438009547E31AF7FAF9BF4111B737002022C4FC
:10F4480006C69387879823880706930710F97CB127
:10F45800B737002003A487AA0DC0B727002003C52B
:10F46800B7788545EF101FC0930710273305F502BD
:10F4780022832244B24041010283B2402244410126
:10F4880082807C2991C778216314F7006FF0DFFA36
:10F49800583901CF7421638FE60078A1B72700207F
:10F4A80003C5B77889456F10CFE7EDD3782179FF89
:10F4B8007CA1EDB7E1DFEDBF6C4531479C3193F797
:10F4C800F7037CA56386E700930700083E858280E2
:10F4D8009C210D47BD8B7CB5E398E7FE41114AC0DE
:10F4E8001309250322C419462A84A1054A8506C69C
:10F4F80026C29710FA1FE78080F491476309051226
:10F508006C441946130524049C2189059987858B29
:10F51800A300F4049710FA1FE78060E12285EFF05A
:10F528001FDEA1476305051024449D475CA49CA0E9
:10F538008547BCA0BCB01946CA85138544009710FE
:10F54800FA1FE780C0DEBC20B830990793F7F70FA1
:10F5580013678700BCA0B8B03844BA97035784062D
:10F56800B8B3BC2038448346D4053E9783578406F5
:10F578009206A183BD8BD58F5CA3B820814709076C
:10F588001377F70FB8A0322C8346C40501CA93F746
:10F598000604CDE7F957998F93F7F70F93F606040A
:10F5A80081CEB030344413660604B0B036971438B0
:10F5B80034B3B8200507B8A0322C014709CE63EC54
:10F5C800C700BC2028440C548D073E959710FA1F9D
:10F5D800E780E0D5382CB42093F7F60385073E97EB
:10F5E80058B4B4A083471403858B91E703470403F9
:10F5F80089476317F70038441C2393E707041CA3C3
:10F608003C444C348CB3930790F97CB00345F40523
:10F61800834774065D8DEF60807B014681450D450B
:10F628009720FA1FE780A06AEF60901B8147B240DD
:10F638002244924402493E8541018280F557A1BF88
:10F648006C45130720029C3193F7F7037CA5639C54
:10F65800E710411122C406C626C29C2115472A84F8
:10F66800BD8B7CB5639AE7021946A10513052503EE
:10F678009710FA1FE780A0DC914765C16C441946D2
:10F68800130524049C2189059987858BA300F4041C
:10F698009710FA1FE780A0C92285EFF05FC6A1473F
:10F6A8004DCDB727002083A7C77C82972444A14764
:10F6B80008D05CA49CA08547BCA0BCB019469305A3
:10F6C8002403138544009710FA1FE78040C6BC2026
:10F6D8009907BCA0BC3093E72700BCB0834714044B
:10F6E80091C738441C2393E707F81CA319469305D0
:10F6F80024041385A4009710FA1FE78040C3BC2098
:10F70800990793F7F70F13F7F703050758B4BCA049
:10F7180083471403858B91E70347040389476317DD
:10F72800F70038441C2393E707041CA33C444C34DB
:10F738008CB39307A0F97CB00345F405834774069E
:10F748005D8DEF60C068014681450D459720FA1F21
:10F75800E780E057EF60D0088147B24022449244E6
:10F768003E8541018280930700083E8582804111D1
:10F778004AC037390020832649AF22C426C206C6AC
:10F788009307000AFCD2B737002083A707ACB70558
:10F7980033002A84D857719B13671700D8D798432A
:10F7A8001377F7E798C398431377F7E713670710BA
:10F7B80098C337370020032787B410474D8E10C7EA
:10F7C8001306A005B0CA5057759A50D70347E505E8
:10F7D8001376F7079843137707F8518F98C3DC42DD
:10F7E8000D4793E71700DCC224459D475CA5854675
:10F7F8009CA0A3810400B4A08347B5056385E700F6
:10F808001947639EE7188547BCB01946930524033A
:10F81800138544009710FA1FE78060B1BC20990750
:10F82800BCA00347B4059947631FF702BC30138592
:10F83800A40093E72700BCB083471403898B638136
:10F8480007124C54BC29638D07101946D10597102F
:10F85800FA1FE780C0AD38441C2393E707F81CA3C0
:10F86800BC209907BCA0BC30B82093E78700BCB087
:10F878003C44BA9703578406B8B3BC20384483463F
:10F88800D4053E97835784069206A183BD8BD58FF6
:10F898005CA3B820814709071377F70FB8A0122C8B
:10F8A8008346C40501CA93F70604F9EBF957998F03
:10F8B80093F7F70F93F6060481CEB03034441366FD
:10F8C8000604B0B03697143834B3B8200507B8A08A
:10F8D800122C4DEA0147B0208347A4059376F6031E
:10F8E800850636979A07D18F58B4BCA0834714036E
:10F8F800858B91E70347040389476317F70038446A
:10F908001C2393E707041CA33C44583498B393077B
:10F9180060F97CB03844832749AFB8DBB73700209B
:10F9280083C7C78281EB3705060081451305254249
:10F93800EF100FFDB73700209387C7ACA3810700EE
:10F948008345F4058347740650342244B2409244F8
:10F958000249DD8D014541011723FA1F670023374E
:10F968008347940391C738441C2393E707F81CA3E3
:10F9780019469305A4039710FA1FE780409BCDB55D
:10F98800F55735B7E3E8C7F4BC2028444C508D0739
:10F998003E959710FA1FE7808099182C2DBF138782
:10F9A800E7FF1377D70F79EF93052503B4B019460E
:10F9B800138544009710FA1FE7806097BC20B83081
:10F9C8001146990793F7F70F13678700BCA0B8B0E3
:10F9D8003844BA9703578406B8B3BC2038448346E2
:10F9E800D4053E97835784069206A183BD8BD58F95
:10F9F8005CA3B820814709071377F70FB8A08345A0
:10FA0800B4058346C4056399C50093F70604ADEBB6
:10FA1800F957998F93F7F70F93F6060481CEB43010
:10FA280093E60604B4B034443697143834B3B82097
:10FA38000507B8A00346B405914601476310D602EE
:10FA4800122C09CE63ECC700BC2028444C508D070B
:10FA58003E959710FA1FE780808D182C0346B40551
:10FA68009146B7370020938787986315D61483C6C5
:10FA7800070793F6060F93E656002388D706A1BD1D
:10FA8800F55741BF93F7B70F0547E395E7E4BCB0D7
:10FA9800930525031946138544009710FA1FE7803C
:10FAA8000089BC209907BCA0BC3093E72700BCB0F4
:10FAB8008347940391C738441C2393E707F81CA392
:10FAC800834714031385A400898BF9C34C54BC29BC
:10FAD800E1C31946D1059710FA1FE78040853844DD
:10FAE8001C2393E707F81CA3BC20B83005469907E8
:10FAF80093F7F70F13678700BCA0B8B03844BA97DC
:10FB080003578406B8B3BC2038448346D4053E97CF
:10FB1800835784069206A183BD8BD58F5CA3B8203A
:10FB2800814709071377F70FB8A08345B4058346C3
:10FB3800C4056399C50093F70604BDEBF957998F7F
:10FB480093F7F70F93F6060481CEB43093E60604D4
:10FB5800B4B034443697143834B3B8200507B8A085
:10FB68000346B405854601476310D602122C09CE18
:10FB780063ECC700BC2028444C508D073E95970085
:10FB8800FA1FE780C07A182C0346B4058546D1BD14
:10FB98008347940391C738441C2393E707F81CA3B1
:10FBA80019469305A4039700FA1FE78040782DBFF4
:10FBB800F55771B783C6070793F6060F93E66600F5
:10FBC8006DBD011152C4373A002056C2930A8A9873
:10FBD80083A7CA0906CE22CC26CA4AC84EC6639550
:10FBE800071C2A840945EF60C047373900200326DF
:10FBF80049AF9307000AB73900207CD283A709AC24
